:1000000000400020816F0000C16F0000C36F00003E
:1000100000000000000000000000000000000000E0
:10002000000000000000000000000000C56F00009C
:100030000000000000000000C76F0000C96F000052
:10004000CB6F000051510000FD730000CB6F00002A
:10005000CB6F000000000000CB6F0000CB6F0000F2
:10006000CB6F0000CD760000C1300000CB6F0000E8
:10007000CB6F0000CB6F0000CB6F0000CB6F000098
:10008000CB6F000065780000CB6F0000CB6F0000E5
:10009000CB6F0000CB6F0000CB6F0000CB6F000078
:1000A000CB6F0000CB6F00000000000000000000DC
:1000B0000000000000000000000000000000000040
:1000C00010B5064C2378002B07D1054B002B02D02E
:1000D000044800E000BF0123237010BD640200202B
:1000E0000000000090E20000044B10B5002B03D08C
:1000F0000349044800E000BF10BDC04600000000F6
:100100006802002090E20000164B002B00D1144B37
:100110009D46402292029A1A924600218B460F4633
:100120001348144A121A0BF045F90F4B002B00D05C
:1001300098470E4B002B00D0984700200021040068
:100140000D000D48002802D00C4800E000BF0BF065
:10015000F1F82000290007F06FF90BF0C5F8C04650
:100160000000080000400020000000000000000027
:1001700064020020B42F00200000000000000000F6
:1001800002000120104011D1042A0ED91368180969
:1001900080B2002809D001388000031D11180979A8
:1001A000002902D001309842F8D170470020FCE7C6
:1001B0000378002B03D05AB2002A01DB01307047CC
:1001C0003F229343C03B59424B41C01803789343AD
:1001D000802BF4D10130F9E710B500240378002B0F
:1001E00001D1200010BDFFF7E3FF0134F6E770B541
:1001F000002204000D00411C092003F07DFA0028B4
:1002000006D001236200134343600023A34200DBB6
:1002100070BD9A00A958821891600133F6E770B555
:10022000012803DC1C2001F043F870BD01230D6898
:1002300011201D42F7D04868184206D1042804D97D
:100240000F2302681340042B01D00E20EBE703F0CC
:10025000B1F86D100400002D03DDFFF7BDFFA842CB
:1002600006DA1220DFE72000FFF7A2FF0400013DBD
:10027000012DF8D120787F2809DDDF280BDCF82359
:100280003F22DB00800118406378134018430123AC
:1002900040001843C9E7EF280BDCFC226378120109
:1002A0009B0113403F220007000C0343A07810403D
:1002B000ECE7F72812DCFC22637892021B03134060
:1002C000E0228004520310403F221843E378134099
:1002D000FC220343A07812018001E8E7012040429C
:1002E000D5E7F8B54D680F00EB0706D4042D04D907
:1002F0000F232E683340092B03D00B2000F0D8FFCA
:10030000F8BD6B683609B6B25C10731EA3420FD8F5
:100310000321200008F00AFF6421642803DC0100A7
:10032000032800DA03212800891903F017FA0500D1
:100330002B6800201B099BB2013B9C42E0D23A682B
:10034000A31C9B005A510123013464001C436C60C0
:10035000D6E7F0B585B0012803DC1C2000F0A8FF2B
:100360002CE001274B683A000093022806D08B68E6
:100370003B4203D05F10002F00DC17000124009BDC
:10038000234200D0B2E0042B00D8AFE01B680D6818
:100390000F2619003140042925D1254205D1042D0D
:1003A00003D92B681E40042E01D00E20D6E70098FA
:1003B000FFF7E6FEB84203DA0120404205B0F0BD87
:1003C000009802F0F7FF0600280002F0F3FF01009A
:1003D000781E30180BF0A4FB0028EDD0801B0130F4
:1003E00040002043EAE709293DD1009B5B685B1090
:1003F00001939F42E0DC25422CD1042D2AD92B68A1
:100400003340042B26D1280002F0D4FF039602903B
:100410007E1C009AB300D058854201D17800E0E7F5
:1004200020420ED104280CD90368039A1340042BF0
:1004300007D102F0BFFF010002980BF03BFB002840
:10044000ECD0019B37009E42E2DDB5E71F00019B27
:100450009F42B1DC7B1C00999A008A58AA42F5D1D0
:1004600078000124BDE7032940D11A0992B25B0F3D
:1004700092000B40D31A01939F429DDC254229D163
:10048000042D27D92A681640032E19D1100980B2ED
:10049000520F800032402C1D801A019B26181B1A17
:1004A0000193009B781E0433019A904200DD83E79C
:1004B00022001918B2420FD316D101304000D0E704
:1004C000042E07D1280002F075FF04002800FFF772
:1004D00057FEE2E70F2041E70D78AC461578AC45B2
:1004E00002D101310132E5E70130DDE7212035E7B6
:1004F00010B502F043FF43000120184310BD000077
:10050000C30711D404280FD90F2302681340032B0B
:100510000AD119400133591AC0234907DB05194094
:10052000024B1A40114301607047C046FFFFFF9F16
:10053000F7B507000E001C20012F06DD4C680123D3
:1005400022001A40009203D10D2000F0B1FE53E0CA
:10055000022F02D08A681A42F6D0012335681D4264
:1005600000D0A9E0042D00D8A6E01C41002C00DC3E
:100570001C000F2029680840092828D16B685B10EF
:100580000093022F05D0B368009A5B109A4200DDF9
:100590000093009B01221D1B0135EB43DB171D401F
:1005A000691C092003F0A8F8071E09D001236D007B
:1005B0001D4303003268083345600099A14201DA07
:1005C0003800FEBD0134A100515802C3F5E70428EC
:1005D00045D1280002F0EEFEFFF7FEFD0190022F4C
:1005E00004D0B3685B10984200DD0193019BA342E5
:1005F00004DA002003F0F2F80700E1E7280002F037
:10060000D9FE0700009BA34221DB2800009702F0DF
:10061000D1FE05003800FFF7CBFD019B0134070038
:10062000A342F7DA009BC41A200003F0D7F8071E94
:10063000C6D002F0BFFE0190306802F0BBFE22007F
:10064000009B591B411801980AF098FEB8E7380042
:10065000FFF7AEFD009B070001330093D2E70328AC
:100660002AD10B099BB2490F9B000140591A022F56
:1006700004D0B2685210914200DD1100A14205DAA7
:1006800000220320110003F037F8B5E703200E1B0A
:10069000331DD9170140C9188910002203F02CF826
:1006A000071E00D18CE7013631000334FFF728FF25
:1006B000381D29193200C7E7212046E7F8B5002880
:1006C00005DC1C2000F0F4FD05002800F8BD012623
:1006D0000C6826400FD06410E343DB171C40E11C7C
:1006E00089100022032003F007F8051EEDD0210039
:1006F000FFF706FFE9E7042C01D80025E5E70F2303
:1007000022681340042B1BD12000FFF739FDC31CC6
:1007100007000320D9170140C9188910320002F0E0
:10072000EBFF051ED1D03900FFF7EAFE200002F0F2
:1007300041FE2B1D01003A0018000AF01FFEC4E71D
:10074000092BDAD10320636832005F10FB1CD91734
:100750000140C918891002F0CFFF051ECDD0390025
:10076000FFF7CEFEFF20BE42AFDA0122B300E3184E
:100770009B68134208D01341FF2B00DD0300D943CF
:10078000C917AA190B4013710136ECE710B57F2980
:1007900002DC0170013010BD1A4B99420CDC402381
:1007A0008A115B42134303703F230B40802149426F
:1007B000194341700230EEE7134B994210DC2023BD
:1007C0000A135B4213433F24802203708B11524271
:1007D0002340214013430A43437082700330DAE719
:1007E0000A4B9942D7DCF0230370603B4370113B06
:1007F0008A11FF3B1A4382703F2211401943C17096
:100800000430C8E7FF070000FFFF0000FF0F0100F2
:10081000F0B50D0085B0002803DC1C2000F048FD79
:100820000DE009680122080010400AD002AC114115
:100830002000FFF7ABFF011B200002F0DBFF0400EC
:100840001AE004293FD90F230C682340092B3AD121
:100850004B685B10019303239C46019B9A420EDD7B
:1008600002F0BCFF041E07D02E68012502F0A2FD95
:100870002F00019B9D421DDD200005B0F0BD01321F
:100880009300CC580123234001D10D20C6E764100A
:100890007F2C0DDD0D4E0223B44209DD0C4E634664
:1008A000B44205DD00270B4EE30FA6427B419B00BF
:1008B000C018D2E70135AB00F1583942E5D04910F4
:1008C000FFF764FFD5E72120A8E7C046FF07000037
:1008D000FFFF0000FF0F010010B5040001200840D9
:1008E00010D104290DD90F230A681340042B08D115
:1008F000080002F05FFD010020000BF0DBF843422E
:10090000584110BD0020FCE7F7B50F00012803DCBB
:100910001C2000F0CDFCFEBD01264D682E4006D106
:10092000042D04D90F222B681A40092A01D00B206C
:10093000EFE76A681B099BB25410A34200D85C1E03
:1009400039681E48FFF7C8FF01230190002813D122
:1009500039681B48FFF7C0FF002811D0002C0DD0CC
:100960000123621C013C9C409200535123436B6065
:1009700004E00136B200AB50B442FADA0020CAE714
:100980003B680D20DA07C4D55B10002B11DD9C42BB
:100990000FDB9B00A200291DEB1889180433994234
:1009A00009D10123013C9C40AA181C4353606C6090
:1009B000E4E71220ADE758681860EFE747CA000087
:1009C0004BCA0000002310B50C000B70C30705D5FF
:1009D0000D49421020000BF031F808E00B490028C7
:1009E00002D0042804D10A4920000BF047F810BDBA
:1009F0000428FCD90F2302681340042BF7D102F01E
:100A0000D9FC04490200E5E744D4000050CA0000C4
:100A100056CA00005BCA0000F0B593B00600029110
:100A20001C20012E1DDD029B01251B681C002C4093
:100A300000D0ADE0042B00D8E6E01A680F231A407E
:100A4000092A4AD10394039A029992008A581700FE
:100A50002F4005D1042A03D910681840092806D070
:100A6000222000F025FC0190019813B0F0BD5268DF
:100A70005210A418039A013203929642E3D1611CEA
:100A8000012202F039FE0190002802D100230193D7
:100A9000EAE7019B6400190025435D600831029A72
:100AA000BB00D05802684368120992B25B109A42A8
:100AB00000D8531E0022934209DCDA43D2171340B8
:100AC0009B00C918039B01379F42E8DBCCE79400E9
:100AD0000519AD6801320D51EDE72700032A59D100
:100AE0000193029ABB00D3582B42B9D1042BB7D93A
:100AF000186801990140032939D1020992B2430FC4
:100B000092000B40D31A1C190137BE42E9D10320D1
:100B1000E31CD9170140C9188910002202F0ECFD2E
:100B200001900028B2D000252100FFF7E9FC019BCD
:100B30001E1D029AAB00D45801231C421FD1042C65
:100B40001DD90F2123681940032918D1180980B233
:100B50005B0F80000B40C01A0023834213DBC343AA
:100B6000DB17184001353618BD42E2DB7CE704296B
:100B700000D075E71800FFF703FB2418C4E7200036
:100B8000FFF7FEFAE8E7E2181279F2540133E4E7DE
:100B900000273C000F25029ABB00D35801221342C4
:100BA00034D1042B32D9186801002940042935D1E9
:100BB0001800FFF7E5FA24180137BE42EBD12000F8
:100BC00002F00CFE0190002800D15FE7029FB60002
:100BD000BB19041D029301233D681D4229D1042D38
:100BE00027D90F262B681E40042E37D12800FFF787
:100BF000C7FA0600280002F0DDFB010020003200E9
:100C00000AF0BCFBA41922E02700C3E7180005A9DD
:100C1000FFF7D8FE05A80AF057FFCCE7032900D05C
:100C20001EE7020992B2430F92000B40D31A1C191F
:100C3000C2E705A92800FFF7C5FE05A80AF044FF92
:100C400005A90500020020000AF098FB6419029B28
:100C50000437BB42BFD10023237005E7032EF6D132
:100C60001A0992B25B0F92001E40961B291DC5E720
:100C7000F0B50D0095B0002806DC1C2000F018FB34
:100C80000400200015B0F0BD0C68012123000B40CA
:100C9000009306D1042C04D922680F331A40092A84
:100CA00001D00B20EAE7626852100392002A03DCAD
:100CB000009802F093FDE3E73F4A019201280BD030
:100CC0006868084208D1042806D902681340042B3A
:100CD00002D102F06FFB019001980AF0F5FE0600C8
:100CE0000F27039B0834013B04935E43039B029050
:100CF0009B001B19059301232068184251D1042839
:100D00004FD903683B40042B52D1FFF739FA059BBA
:100D100004343618A342EED1300002F05FFD041E09
:100D2000AFD02B680593029B002B03D0686802F0BC
:100D300041FB0190200002F03DFB0500009B059A5D
:100D40009B00D3189F68380002F034FB0123060093
:100D50001F4201D1042F04D807A93800FFF732FE43
:100D600007AE30000AF0B0FE070002003100280094
:100D70000AF004FB029BED19002B0AD0049B009A99
:100D8000934206DD2800029A01990AF0F7FA029BC5
:100D9000ED18009B01330093009A039B9342CDD141
:100DA0006FE707A9FFF70EFE07A80AF08DFEAEE772
:100DB00002F000FBF9E7C046E8CE000010B50024C1
:100DC000A04207DD0B6801341C4003D05C10E343F4
:100DD000DB171C40611C0122092002F08DFC002859
:100DE00003D0012364001C43446010BD0A6870B541
:100DF00010000125284034D1042A32D90F24136869
:100E000049681C40092C17D154681B099BB22C411E
:100E1000A34200D85C1E844205DC022001339842C4
:100E200006DB00200FE085005519A9600130F2E7CC
:100E3000840011510130F2E7032C12D1294203D171
:100E4000132000F035FA70BD4910FF29F8D81B09AE
:100E50009BB204329B00D3189342E2D91170013245
:100E6000FAE70B2000F024FADBE700000123F7B5D6
:100E700000254E680F0033400093AB420ED11D0099
:100E8000042E0BD90F2233681A40092A10D1726838
:100E90001B099BB25510AB4200D85D1E3968CB07C9
:100EA00017D54C10002C01DDA5421DDA122032E0CE
:100EB000042A04D13000FFF763F90500EEE7009D36
:100EC000032AEBD11D09ADB25B0FAD001340ED1A43
:100ED000E4E72E48FFF700FD002814D00AF04AFD91
:100EE000290008F009FA4C1C009B002B4CD1042E61
:100EF0004AD932680F331340092B10D10134A400B2
:100F0000A4592000FEBD39682148FFF7E5FC2C00FC
:100F10000028E9D1113000F0CBF90400F1E7042BEF
:100F20002AD1300002F046FA0500FFF755F9A04239
:100F3000BCDB012C1ADC300002F03CFA00902800E7
:100F4000FFF736F9461B300002F048FC041ED8D0EB
:100F500002F030FA0190786802F02CFA009B32001F
:100F6000E91A411801980AF009FACAE72800FFF7C0
:100F70001FF9013C0500DCE7032B05D13419E478A7
:100F8000023B64001C43BCE70B20C4E740CA0000DE
:100F90004BCA0000F7B54D680F002A0001210A4036
:100FA0002FD1042D2DD90F242B68BE681C40092C8D
:100FB00014D169681B099BB24C100192A34200D85E
:100FC0005C1E39682A48FFF787FC00282DD00F23C4
:100FD0002A681340092B1DD1012317E0032C10D1DF
:100FE0000E4203D1132000F063F9FEBD721001928E
:100FF000FF2AF7D81A0992B25B0F92001C40141B0B
:10100000DFE70B20EFE701339A00AE509C42FADA9B
:101010000020EAE7032BFBD12B0001335A1BA2422D
:10102000F6DC6A461279DA70F7E73968CB0706D53D
:101030004910002901DD8C4209DA1220D3E70D485E
:10104000FFF74AFC2100002801D11130CBE70F2324
:101050002A681340092B03D1013189004E51D7E78B
:10106000032BD5D16B461B796D18EB70D0E7C046CA
:1010700047CA00004BCA000010B50124086820428E
:101080001AD1042818D90F2102681140092901D169
:10109000406810BD032908D113099BB2500F9B0073
:1010A0000840181A40002043F3E7042904D102F055
:1010B00081F9FFF791F8F5E70B2000F0F9F8E8E780
:1010C00010B5034A0B21034804F03AF910BDC0469D
:1010D000E8C90000E0C90000002070470020704708
:1010E00000207047002070470020704700207047A4
:1010F0000020704700207047002070470020704794
:10110000002070470020704710B5034A0C210348A7
:1011100004F016F910BDC046D0CA000030CB000064
:1011200010B50124044002D04410200010BD042852
:1011300010D90F2302681340042B07D102F03AF9AB
:1011400021000A220AF088FD0400EEE7032B01D1FA
:101150000430F5E70D22014B1A70E6E7A4020020E7
:10116000012210B5024018D1042802D903681A09D7
:1011700092B201230B4012D1042902D90B681B093A
:101180009BB20024934206D104309B000431C31863
:10119000984206D30124200010BD0022E9E7002375
:1011A000EFE704780A78002C01D1002AF2D0013050
:1011B00001319442ECD00024EDE70000F7B50700C0
:1011C000009101933049314B002A02D002220A706B
:1011D000013A00261A601B68CE54BE4200DBF7BD00
:1011E000009AB300D058294B274D1C68C8239B0098
:1011F00065191C1B0123184206D0254A4310210003
:1012000028000AF0E9FB09E0224A002802D004285D
:101210001BD1214A210028000AF0DEFB1A4C2000D5
:101220000AF052FC194A019B1060002B0BD07B1E68
:10123000B34208DD194B984205D8431C13602022A5
:1012400022540022E2540136C7E7042819D90F239B
:1012500001680B40042B04D102F0ACF8104A0300E3
:10126000CDE7092B03D143680E4A5B10C7E7032B78
:1012700008D10A0992B2490F92000B40D31A0A4AC8
:10128000BDE70123094ABAE7A5020020C8050020EE
:1012900044D4000050CA000056CA00001F030000DA
:1012A0006FDA0000A0CD0000AFCD0000BACD000085
:1012B000014B187000207047A402002070B501F0A7
:1012C000EDFD094C0100251D1F2228000AF014FC29
:1012D00028000AF0F9FB04230430800800011843B9
:1012E0002060200070BDC04680020020C368F0B5B9
:1012F0009D00836889B05D19030018330693036964
:10130000069A9F00069B0290DF19436901939B0098
:10131000D3180393CD4B1B78002B26D17F222B684B
:10132000CB491C1213409B005B58043501929F4629
:10133000029B587804F020FC0023029A137027E0E7
:10134000C24B1B78002B10D12B68019A1C12134042
:10135000BF4A9B009B580435E9E7069B3A1DD11A0A
:10136000BA4BD82928DD1A221A70029BB74C9B6809
:1013700021780193EA1A029B92109B7812021A4379
:10138000029B587804F000FC0023029A237013702B
:10139000029B069A9B680193ED1A029BAD10DD60DB
:1013A000069BFE1A029BB6101E61039B9B1A029AB3
:1013B0009B10536109B0F0BD1B783C60002B01D03D
:1013C0001700D2E72B6801991C120B40A0499B0023
:1013D0005B5817000435AAE7069B3A1DD11A9B4BB0
:1013E000D82902DD1A221A70BFE728681B78291D48
:1013F0003860002B02D017000D00B6E76B6801992A
:101400001C120B4092499B005B58170008358EE771
:10141000069B3A1DD11A8D4BD82902DD1A221A706B
:10142000A3E7A4001B782C193C60002B01D0170007
:101430009BE72B6801991C120B4085499B005B5868
:101440001700043573E7069B3A1DD11A7F4BD82944
:1014500002DD1A221A7088E77E49A40061581B78C1
:101460003960002B01D017007FE72B6801991C120F
:101470000B4077499B005B581700043557E7043F42
:10148000744B3A68A400E250704B1B78002B00D0DC
:101490006BE72B68019A1C1213406D4A9B009B5806
:1014A000043544E76B4BA400E058FFF739FE043FD6
:1014B00006003868FFF734FE36180120654B7600C9
:1014C0000643E650614B1B78002B00D04DE72B689C
:1014D000019A1C1213405E4A9B009B58043526E774
:1014E000069B3A1DD11A594BD82902DD1A221A70CF
:1014F0003BE70698039C0121A04202D221000C394F
:1015000009681B783960002B01D017002DE72B6884
:1015100001991C120B404E499B005B581700043583
:1015200005E7069B3A1DD11A484BD82902DD1A223D
:101530001A701AE70699039881420FD203000C3BF8
:101540001B6845495B106418E41AA40023583B60EB
:101550003E4B1B78002B05D0170006E718211970A9
:101560000023F4E72B6801991C120B4038499B00BB
:101570005B5817000435DAE6069B039A934219D2AA
:1015800013000C3B1B68344A043FA4185B10E31A99
:10159000039A39689B0099502C4B1B78002B00D084
:1015A000E3E62B68019A1C121340294A9B009B58C2
:1015B0000435BCE61822254B1A70EDE7069B039A0A
:1015C00093422DD2244B3E1FE31814000C3C04938D
:1015D0002368049A5B10D31A039A9B009858FFF76C
:1015E0009FFD07903068FFF79BFD2468049B641003
:1015F0001C1B079BA4001F1801207F00039B0743AF
:10160000E7503700114B1B78002B00D0ADE62B685C
:10161000019A1C1213400E4A9B009B58043586E623
:1016200018220A4B1A70EDE7069B3A1DD11A074B98
:10163000D82902DD1A221A7097E60399A40061588E
:101640001B783960002B09D017008EE6A402002019
:10165000A0CB0000802D0020FDFFFF3F2B680199EB
:101660001C120B40D9499B005B58170004355EE6FD
:10167000043F039B3A68A400E250D54B1B78002B33
:1016800000D072E62B68019A1C121340CF4A9B00CF
:101690009B5804354BE6039BA4001C192368043FA8
:1016A00038685E10FFF73CFD36180120C84B760005
:1016B0001B7806432660002B00D056E62B68019A63
:1016C0001C121340C14A9B009B5804352FE6069B11
:1016D000A4003F1BBE4CBB420CD82378002B00D08B
:1016E00043E62B68019A1C121340B84A9B009B5892
:1016F00004351CE6B74801F04DFE2378002B00D0DE
:1017000033E62B68019A1C121340B04A9B009B5889
:1017100004350CE6A300ED18002C00DA38E6AC4BDB
:101720001B78002B00D020E62B68019A1C12134076
:10173000A64A9B009B580435F9E5043F3B68042BFF
:1017400004D1A300ED18002C00DA21E6A04B1B7891
:10175000002B00D009E62B68019A1C1213409B4A0B
:101760009B009B580435E2E5043F3B68042B04D002
:10177000A300ED18002C00DA0AE6954B1B78002B2D
:1017800000D0F2E52B68019A1C1213408F4A9B008F
:101790009B580435CBE53A1F13685B10013B002BC7
:1017A00006DD01215B00A4000B432D191360EFE55A
:1017B000874B17001B78002B00D0D6E52B68019AC9
:1017C0001C121340814A9B009B580435AFE53A0038
:1017D000069B0C32D31AD82B03DD1A227C4B1A70CD
:1017E000C3E5FF2361005B001940FE3BFF3B19434B
:1017F0003960029906988968241204916D1A029939
:10180000AD1089782D020D4303999D40091A891066
:1018100099401D430B43BB60029B7D609C70E4B20A
:101820006D4BE4000392E358029A9360684A127881
:10183000002A03D008331D00039F96E51D00019A7E
:101840009B680C351C121340604A9B009B58039FF9
:101850006DE53B1F1C68039A069B93422DD10A201D
:10186000E3070CD4042C13D90F2322681340042B54
:1018700011D1200001F09EFD0AF026F906306430F7
:1018800003F098FD00280FD1043D069B03937FE5EC
:101890000720042CF3D02000431E9841FA23404235
:1018A000FF3318400730EAE7029B2100587804F024
:1018B0007DF90023029A1370E7E7039B039A0C3B20
:1018C0001B6802995B109B00D31A0C3B1C601F1D08
:1018D0001300083B1B685A108A70D2B23E49D200EE
:1018E0005B0055589B0A029A9B009560ED18039B7C
:1018F000069A043B1B685B109B00D3180393344B80
:101900001B78002B00D030E52B68019A1C12134085
:101910002E4A9B009B58043509E53B1F1868FFF7CA
:10192000FFFBA40006003F1B1E2827DC00280DDC5F
:10193000274B1B78002B00D017E52B68019A1C124F
:101940001340224A9B009B580435F0E401F094FABE
:10195000033E361801F090FA204B801B9842F9D8CC
:101960001B4B1B78002B00D0FFE42B68019A1C1244
:101970001340164A9B009B580435D8E40123029A71
:10198000137001F079FA029B0A3886195E60FFE451
:101990003B1F1868FFF7C4FBA40006003F1B00288C
:1019A0000DDC0B4B1B78002B00D0DEE42B68019A7A
:1019B0001C121340054A9B009B580435B7E4084BA2
:1019C00098420FDD1D22024B1A70CEE4A0CB00001E
:1019D000A4020020CCCD0000882500203F420F004B
:1019E00080EE36000123029A137001F045FAFA23C3
:1019F0009B005E43029B0A3E30185860C8E4A30077
:101A0000FF1A002320001A003900FFF7D7FBCC4E45
:101A1000CC4C3168200001F0EDFECB4B31681860F2
:101A2000200003F077FF3168200004F0C6F8C74BB0
:101A30001B78002B00D098E42B68019A1C121340ED
:101A4000C34A9B009B58043571E4C04BA4001B782B
:101A50003F1B002B00D088E42B68019A1C12134016
:101A6000BB4A9B009B58043561E4029803F006FDD5
:101A7000B64B1B78002B00D077E42B68019A1C1220
:101A80001340B34A9B009B58043550E43B1F1B682E
:101A9000002B3ED13B000C3B1B68DA072CD53900EC
:101AA00001225B105800083902430A60002B44DD14
:101AB000012259001143381F0160390008390968B3
:101AC0001141CB1A39000C390968114224D09B18F6
:101AD0009340A4001343039AA3509C4B1B78002B04
:101AE00000D042E42B68019A1C121340984A9B00D4
:101AF0009B580435FFF71BFC042B06D90F211A68ED
:101B00000A40092A01D15B68C9E719228F4B1A7074
:101B10002BE45B10013BC9E7042909D90F200A68AF
:101B20000240092A04D102339B005B58A400D2E78B
:101B30001922864B1A70FFF718FC0435CDE7A30075
:101B4000069AFB189B1AD82B13DC0122631E002C6B
:101B500014DC7E4B1B78002B01D0FFF706FC2B68B2
:101B6000019A1C1213407A4A9B009B580435FFF7D8
:101B7000DEFB1A22754B1A70FFF7F7FB3A601C0068
:101B80000437E3E7069A3B1D9B1A704ED82B03DD02
:101B90001A233370FFF7E9FB069B039AA4009342D4
:101BA0002AD23B1F1868FFF7BBFA011E21DD039BF9
:101BB0000C3B1A68521082421BDB9007801A654B5F
:101BC0004018C018039B8000C2583B1B1A605F4B33
:101BD0003F1B1B780437002B01D0FFF7C6FB2B6897
:101BE000019A1C1213405A4A9B009B580435FFF778
:101BF0009EFB20233370EAE71823FBE7524BA40037
:101C00001A683B1B1F001A60504B04371B78002BCF
:101C100001D0FFF7AAFB2B68019A1C1213404C4A13
:101C20009B009B580435FFF782FBA3009C46FE1ADD
:101C3000002C17DC1C22454B1A70002333606346CE
:101C4000FF1A424B04371B78002B01D0FFF78DFBA6
:101C50002B68019A1C1213403D4A9B009B58043587
:101C6000FFF765FB002033685A108300F158012309
:101C70000B4003D10D21354A1170DFE749108A422C
:101C800000DD0A0001308442EFDC012352001343DF
:101C9000D4E7A3009C46FE1A002C17DC1C222B4B19
:101CA0001A70002333606346FF1A284B04371B78F1
:101CB000002B01D0FFF759FB2B68019A1C1213402F
:101CC000234A9B009B580435FFF731FB0020336803
:101CD0005A108300F15801230B4003D10D211B4AF8
:101CE0001170DFE749108A4200DA0A0001308442AD
:101CF000EFDC012352001343D4E73B00083B186894
:101D0000FFF70EFA3B1F06001868FFF709FA0023D9
:101D1000864200DA0433A4003A1B170013600B4B11
:101D200004371B78002B01D0FFF71FFB2B68019AAB
:101D30001C121340064A9B009B580435FFF7F7FA24
:101D4000C8050020A502002008000020A4020020F1
:101D5000A0CB0000FCFFFF3F3B00083B1868FFF7EB
:101D6000DFF93B1F06001868FFF7DAF9F30FC21717
:101D7000B0425341A4003A1B17009B001360E34B91
:101D800004371B78002B01D0FFF7EFFA2B68019A7C
:101D90001C121340DE4A9B009B580435FFF7C7FA1C
:101DA0003B00083B18683B1F1968A600BE1B0423B4
:101DB000814202D0042802D80023336018E00123B6
:101DC0009C461842F8D10F2302681A40042AF3D126
:101DD00063461942F0D10429EED90B680B32134047
:101DE000042BE9D1FFF7BCF9431E98418000306015
:101DF000C64BA4001B783F1B0437002B01D0FFF714
:101E0000B4FA2B68019A1C121340C14A9B009B58DC
:101E10000435FFF78CFA3B00083B18683B1F196834
:101E2000A600BE1B0023814202D0042802D804234E
:101E3000336018E001239C461842F8D10F23026852
:101E40001A40042AF3D163461942F0D10429EED98D
:101E50000B680B321340042BE9D1FFF781F94342A1
:101E6000584180003060A94BA4001B783F1B043709
:101E7000002B01D0FFF779FA2B68019A1C1213404E
:101E8000A34A9B009B580435FFF751FA3B00083BDF
:101E90001868FFF745F93B1F06001868FFF740F97F
:101EA000F317C20F86425341A4003A1B17009B0050
:101EB0001360964B04371B78002B01D0FFF755FABF
:101EC0002B68019A1C121340914A9B009B580435C1
:101ED000FFF72DFA3B00083B1868FFF721F93B1F7D
:101EE00006001868FFF71CF90023864200DD043362
:101EF000A4003A1B17001360844B04371B78002B97
:101F000001D0FFF732FA2B68019A1C121340804A65
:101F10009B009B580435FFF70AFA3B1F1B68A4007F
:101F2000043B5A1E93413A1B17009B001360774BEA
:101F300004371B78002B01D0FFF717FA2B68019AA2
:101F40001C121340724A9B009B580435FFF7EFF9AF
:101F50003B00083B1868FFF7E3F83B1F06001868D2
:101F6000FFF7DEF832180120A4003B1B1F005200CF
:101F700002431A60654B04371B78002B01D0FFF732
:101F8000F4F92B68019A1C121340614A9B009B587C
:101F90000435FFF7CCF93B00083B1868FFF7C0F8A1
:101FA0003B1F06001868FFF7BBF8321A0120A40097
:101FB0003B1B1F00520002431A60544B04371B782E
:101FC000002B01D0FFF7D1F92B68019A1C121340A6
:101FD0004F4A9B009B580435FFF7A9F93B00083B8B
:101FE0001868FFF79DF83B1F06001868FFF798F880
:101FF00002000120A4003B1B1F0072435200024359
:102000001A60424B04371B78002B01D0FFF7ADF963
:102010002B68019A1C1213403D4A9B009B580435C3
:10202000FFF785F93B1F1868FFF77AF8061E17D1EE
:102030001F23364A1370A4003B1B1F001E60334B46
:1020400004371B78002B01D0FFF78FF92B68019A1A
:102050001C1213402E4A9B009B580435FFF767F96A
:102060003B00083B1868FFF75BF8310007F05EF8AB
:10207000012640000643DEE73B1F1868FFF750F8D3
:10208000061E17D11F23214A1370A4003B1B1F00FB
:102090001E601E4B04371B78002B01D0FFF765F93B
:1020A0002B68019A1C121340194A9B009B58043557
:1020B000FFF73DF93B00083B1868FFF731F83100A6
:1020C00007F01AF9012649000E43DEE73B1F1868A6
:1020D000FFF726F8C217801850400122A4003B1BCE
:1020E0001F00400010431860084B04371B78002B7A
:1020F00001D0FFF73AF92B68019A1C121340044AE9
:102100009B009B580435FFF712F9C046A40200203B
:10211000A0CB0000A300FE1A3068012C24D1FEF7EA
:10212000FFFF0494079009F025FC0799002900DCC3
:10213000012107F0E1F8049BA400C918012349001C
:102140001943EA4B3F1B1B7831600437002B01D049
:10215000FFF70BF92B68019A1C121340E44A9B000D
:102160009B580435FFF7E3F8FEF7DAFF0490706838
:10217000FEF7D6FF049B0130C31A0793D3E7A300F1
:10218000FE1A31002000049301F0BAFC049B306079
:10219000FF1AD64B04371B78002B01D0FFF7E5F868
:1021A0002B68019A1C121340D14A9B009B5804359E
:1021B000FFF7BDF83B00083B1868FEF7B1FF3B1F77
:1021C00006001868FEF7ACFF02000120A4003B1BCC
:1021D0001F003240520002431A60C44B04371B7880
:1021E000002B01D0FFF7C1F82B68019A1C12134095
:1021F000BF4A9B009B580435FFF799F83B00083B0A
:102200001868FEF78DFF06003B1F1868FEF788FF71
:10221000320002430120A4003B1B1F005200024376
:102220001A60B24B04371B78002B01D0FFF79DF8E2
:102230002B68019A1C121340AD4A9B009B58043531
:10224000FFF775F83B00083B1868FEF769FF0600CA
:102250003B1F1868FEF764FF320042400120A400D3
:102260003B1B1F00520002431A60A04B04371B782F
:10227000002B01D0FFF779F82B68019A1C1213404C
:102280009B4A9B009B580435FFF751F83B1F186889
:10229000FEF746FFC0430122A4003B1B1F00400085
:1022A00010431860914B04371B78002B01D0FFF7C7
:1022B0005CF82B68019A1C1213408D4A9B009B58B6
:1022C0000435FFF734F83B00083B1868FEF728FF99
:1022D00006003B1F1868FEF723FF320082405100C2
:1022E0000122A4003B1B1F000A431A607F4B0437E6
:1022F0001B78002B01D0FFF738F82B68019A1C12CD
:1023000013407B4A9B009B580435FFF710F83B00B5
:10231000083B1868FEF704FF06003B1F1868FEF72D
:10232000FFFE3200024151000122A4003B1B1F00AE
:102330000A431A606D4B04371B78002B01D0FFF75E
:1023400014F82B68019A1C121340694A9B009B5891
:102350000435FEF7ECFF3B000C3B1868FEF7E0FE8F
:102360003B00083B06001868FEF7DAFEF117020092
:10237000C317300007F012F83B1F0490059118684E
:10238000FEF7CEFE02000498059906F0BBFF43005D
:102390000120A4003E1B37001843544B30601B78CB
:1023A0000437002B01D0FEF7E0FF2B68019A1C12C6
:1023B00013404F4A9B009B580435FEF7B8FFA3001B
:1023C000FE1A310020000493FEF7F8FC049B3060F5
:1023D000FF1A464B04371B78002B01D0FEF7C5FFD0
:1023E0002B68019A1C121340414A9B009B580435EC
:1023F000FEF79DFFA300FF1A39002000FEF7F6FC50
:102400003A4B1B78002B01D0FEF7AFFF2B68019AE7
:102410001C121340364A9B009B580435FEF787FF79
:10242000A300FE1A310020000493FEF71FFD049B59
:102430003060FF1A2D4B04371B78002B01D0FEF7BC
:1024400094FF2B68019A1C121340294A9B009B5849
:102450000435FEF76CFFA300FF1A39002000FEF7D9
:1024600099FD224B1B78002B01D0FEF77EFF2B68D5
:10247000019A1C1213401E4A9B009B580435FEF71C
:1024800056FFA300FE1A310020000493FEF7F4FD6E
:10249000049B3060FF1A154B04371B78002B01D0CA
:1024A000FEF763FF2B68019A1C121340104A9B0031
:1024B0009B580435FEF73BFF3B1F186800F07AFF7E
:1024C0003A00083A12680300A400D1072DD4042A68
:1024D00010D910680F2210400138082813D806F0D0
:1024E00087FD09242A26121212122800A4020020B5
:1024F000A0CB0000F149180009F0DCFA4342584132
:102500003B1B80001860EE4B3F1B1B780437002BF1
:1025100001D0FEF72AFF2B68019A1C121340E94AEA
:102520009B009B580435FEF702FFE749E3E7E749C4
:10253000E1E7E749DFE7E749DDE7069B3E1DF31AE0
:10254000DF4CD82B03DD1A232370FEF70EFF00F0BB
:102550009DFC43000120184323783860002B02D0F3
:102560003700FEF702FF2B68019A1C121340D54A70
:102570009B009B5837000435FEF7D9FE069B3E1D95
:10258000F31ACF4CD82B03DD1A232370FEF7EDFE90
:1025900000F072FCD04B4000184001231843237810
:1025A0003860002B02D03700FEF7DFFE2B68019A5F
:1025B0001C121340C34A9B009B5837000435FEF79A
:1025C000B6FE0123A600BE1B20001A003100FEF754
:1025D000F5FDC24C2068643002F0ECFE002802D108
:1025E000043DFEF7D5FE029B21685A78BC4803F0F3
:1025F000F2FA0123029A3700137000F03DFCB94B48
:1026000022681B68063253431818029B5860FEF775
:10261000BFFEA600BE1B2000012300223100FEF7F2
:10262000CDFDAE4C2068643002F0C4FE0028D7D047
:10263000AB4803F05FF8DCE7A4003E1BFEF73EFE6C
:1026400037009F4B30601B780437002B01D0FEF71A
:102650008CFE2B68019A1C1213409A4A9B009B58CF
:102660000435FEF764FEA4003E1B300000F03DFC84
:102670003700934B30601B780437002B01D0FEF7F6
:1026800074FE2B68019A1C1213408E4A9B009B58C3
:102690000435FEF74CFEA4003E1B300000F027FC82
:1026A0003700874B30601B780437002B01D0FEF7D2
:1026B0005CFE2B68019A1C121340824A9B009B58B7
:1026C0000435FEF734FEA300FE1A31002000049307
:1026D00000F010FC049B3060FF1A794B04371B7824
:1026E000002B01D0FEF741FE2B68019A1C1213400B
:1026F000744A9B009B580435FEF719FEA4003F1B4B
:10270000380000F029FC6E4B1B78002B01D0FEF73F
:102710002CFE2B68019A1C1213406A4A9B009B589E
:102720000435FEF704FEA300FE1A310020000493D6
:1027300000F03AFC049B3060FF1A614B04371B78B1
:10274000002B01D0FEF711FE2B68019A1C121340DA
:102750005C4A9B009B580435FEF7E9FDA4003F1B33
:10276000380000F063FC564B1B78002B01D0FEF7BD
:10277000FCFD2B68019A1C121340524A9B009B5887
:102780000435FEF7D4FD0121200000F037FC4C4B4E
:102790001B78002B01D0FEF7E8FD2B68019A1C1274
:1027A0001340484A9B009B580435FEF7C0FD0021AA
:1027B000200000F023FC424B1B78002B01D0FEF7D9
:1027C000D4FD2B68019A1C1213403E4A9B009B5873
:1027D0000435FEF7ACFDA4003E1B300000F048FCC1
:1027E0003700374B30601B780437002B01D0FEF7E1
:1027F000BCFD2B68019A1C121340324A9B009B5867
:102800000435FEF794FDA4003E1B300000F044FCAC
:1028100037002B4B30601B780437002B01D0FEF7BC
:10282000A4FD2B68019A1C121340264A9B009B585A
:102830000435FEF77CFDA4003F1B380000F006FCC9
:102840001F4B1B78002B01D0FEF78FFD2B68019AE0
:102850001C1213401B4A9B009B580435FEF767FD72
:10286000A4003F1B380003F0D1FC154B1B78002B54
:1028700001D0FEF77AFD2B68019A1C121340114A11
:102880009B009B580435FEF752FDA4003E1B300010
:1028900003F054FD37000A4B30601B780437002BDF
:1028A00001D0FEF762FD2B68019A1C121340054A05
:1028B0009B009B580435FEF73AFDC046DCCD000076
:1028C000A4020020A0CB0000E4CD0000EBCD00006E
:1028D000F2CD0000F7CD0000FEFFFF7FC80500200D
:1028E000A502002004000020A4003F1B380003F0D4
:1028F0003DFCC24B1B78002B01D0FEF736FD2B6848
:10290000019A1C121340BE4A9B009B580435FEF7E7
:102910000EFDA4003E1B300003F03EFC3700B74B19
:1029200030601B780437002B01D0FEF71EFD2B68AA
:10293000019A1C121340B24A9B009B580435FEF7C3
:10294000F6FCA300FF1A3900200001F0F7FBAB4BA7
:102950001B78002B01D0FEF708FD2B68019A1C1292
:102960001340A74A9B009B580435FEF7E0FCA300E8
:10297000FF1A3900200001F017FAA04B1B78002B3A
:1029800001D0FEF7F2FC2B68019A1C1213409C4AFE
:102990009B009B580435FEF7CAFCA300FF1A3900C0
:1029A000200001F003FB954B1B78002B01D0FEF7B4
:1029B000DCFC2B68019A1C121340914A9B009B5827
:1029C0000435FEF7B4FCA300FF1A3900200001F023
:1029D00015FB8A4B1B78002B01D0FEF7C6FC2B6839
:1029E000019A1C121340864A9B009B580435FEF73F
:1029F0009EFCA300FE1A31002000049303F043FD67
:102A0000049B3060FF1A7D4B04371B78002B01D0EC
:102A1000FEF7ABFC2B68019A1C121340784A9B000E
:102A20009B580435FEF783FCA300FE1A31002000FA
:102A3000049303F030FD049B3060FF1A6F4B0437A2
:102A40001B78002B01D0FEF790FC2B68019A1C121A
:102A500013406B4A9B009B580435FEF768FCA300AB
:102A6000FE1A31002000049303F01DFD049B30602A
:102A7000FF1A624B04371B78002B01D0FEF775FC60
:102A80002B68019A1C1213405D4A9B009B58043529
:102A9000FEF74DFCA300FE1A31002000049303F062
:102AA0001DFB049B3060FF1A544B04371B78002B2E
:102AB00001D0FEF75AFC2B68019A1C121340504AB1
:102AC0009B009B580435FEF732FCA300FF1A390027
:102AD000200001F0A1F9494B1B78002B01D0FEF733
:102AE00044FC2B68019A1C121340454A9B009B58DA
:102AF0000435FEF71CFCA300FF1A3900200001F08A
:102B0000A5FA3E4B1B78002B01D0FEF72EFC2B685C
:102B1000019A1C1213403A4A9B009B580435FEF759
:102B200006FCA300FE1A31002000049301F00AFA0B
:102B3000049B3060FF1A314B04371B78002B01D007
:102B4000FEF713FC2B68019A1C1213402C4A9B00C1
:102B50009B580435FEF7EBFBA300FF1A3900200059
:102B600001F0B8F9254B1B78002B01D0FEF7FDFBD7
:102B70002B68019A1C121340214A9B009B58043574
:102B8000FEF7D5FB069B029AFB1A9B101361A3006C
:102B9000FF1A3900200002F0EBFD184B1B78002BC8
:102BA00001D0FEF7E2FB2B68019A1C121340144A75
:102BB0009B009B580435FEF7BAFB069B029AFB1A52
:102BC0009B101361A300FE1A31002000049302F051
:102BD000CFFD049B3060FF1A084B04371B78002B95
:102BE00001D0FEF7C2FB2B68019A1C121340044A65
:102BF0009B009B580435FEF79AFBC046A4020020B8
:102C0000A0CB00000023F7B55A1E0192002B07DA73
:102C100001F0AAFA02F0DCFE03F03CF8192301935C
:102C200000263000194B1968B14212DD184B1A68A2
:102C300001328A420FDAF0241A601D68154F6C4386
:102C4000E35D002B1FD0E419022B06D12000FEF714
:102C50004DFB019BD8E70022EDE7012B0DD10028A9
:102C600001D100F009F9F0226A43BB185B680A49F8
:102C7000C31A8B4201D80223BB54F0235D43054B9A
:102C8000EB5C022BE2D00136CCE7C046CC0500203D
:102C900000000020281C00203F420F0001220021DC
:102CA0000A4B0B481A61195004301950A221042014
:102CB000C9005850C121C0208900800258501A60B4
:102CC000044BFC311960044B1A70704700A000409F
:102CD0000405000000E100E0F30500200420704737
:102CE000F8B550C9012322001A40101E2DD03340E0
:102CF000181E2AD0641000201C2C26D81D4B7610DC
:102D000035009E4200DD1D001B4F3B5D012B05D0B1
:102D10000121200004F026FD01233B55174B1B78B1
:102D2000002B01D1FFF7BAFF0023154A9E420DDCAC
:102D3000FF2514491448D65CB44202D15E0070529B
:102D4000D5540133042BF6D10420F8BDD15C8C425C
:102D500003D10C4A5B009D52F6E70133042BF5D1F9
:102D60000023D15CFF2901D1D454F2E70133042BB5
:102D7000F7D1E9E788130000D4050020F30500200F
:102D80001C0000200E000020DC050000F8B530C952
:102D9000012623003340181E1BD02B003340181E81
:102DA00017D0344100201C2C13D8174F3B5DB34281
:102DB00004D03100200004F0D5FC3E556910080015
:102DC000124A1038124B904204D9012252421A6022
:102DD0000420F8BD1C600F4806F0A8F90E4B1880BF
:102DE0000E4B1B78002B02D1FFF758FFF0E70122B2
:102DF0000B4B9A64A922D2009A588018A82280B25C
:102E0000D2009850E4E7C046D40500209086010027
:102E10001800002020A107000C000020F30500206E
:102E200000A00040030010B50120002B02DC1B3085
:102E3000FEF73EFA10BD0420704710B5002803DCF1
:102E40001C20FEF735FA10BD0B680020DB07FAD412
:102E50000D30F6E701220020054B06491A61585053
:102E60000431033058500831801858501A607047A8
:102E700000800040040500000122034B1A64A822D0
:102E8000D20098587047C0460080004010B5FFF748
:102E9000F3FFFA21890006F0BFF810BD0048704723
:102EA00054CE00001D20704770B5054E0400335C01
:102EB0000D008B4202D004F055FC355570BDC04664
:102EC000D405002070B50024064D635D012B05D1AB
:102ED0000021200004F046FC0023635501341D2C22
:102EE000F2D170BDD405002070470D2070473B2003
:102EF00070470000F8B501240B6806000D0023425E
:102F000004D10D20FEF7D4F92000F8BD5B1020009D
:102F1000052BFAD80E4A9B009C580E4F3B5D002BA8
:102F200005D00021200004F01DFC00233B55012E9C
:102F300006DD6B68042B03D10221200004F012FC93
:102F4000200004F0BDFA012440002043DDE7C04624
:102F50003CCE0000D4050020F8B5012605683542B6
:102F600002D04468344203D10D20FEF7A1F9F8BD28
:102F70006D101C2DFBD80A4F7B5D012B04D0310056
:102F8000280004F0EFFB7E55064964108C4202DCF9
:102F9000E143C9172140280004F018FBE7E7C046C9
:102FA000D4050020FF03000070B501240D68254200
:102FB00004D10D20FEF77CF9200070BD6D101C2D92
:102FC00017D80024012804DD4C68043C63425C41AE
:102FD0006400094E735DA34204D02100280004F070
:102FE000C1FB7455280004F0F1FB03000420012B01
:102FF000E3D00020E1E7C046D405002070B504000E
:103000000D001C280ED8084E335C012B04D0012182
:1030100004F0A8FB01233355290020004D1EA941CF
:1030200004F0BEFB70BDC046D4050020036810B597
:10303000DA0703D40D20FEF73BF910BD41685810A4
:1030400004394A425141FFF7D9FFF6E737B56946DF
:103050000A00064B30CB30C203680220042B02D199
:1030600000F0A4FF37BD00F0C9FFFBE704CE00006D
:1030700010B5084C6379002B05D00021052004F021
:1030800071FB00236371052004F0A0FB434258410B
:10309000800010BDD405002010B5084CE37A002B49
:1030A00005D000210B2004F05DFB0023E3720B2010
:1030B00004F08CFB43425841800010BDD405002031
:1030C000F7B5304D304E6B6C002B15D0A824002383
:1030D000E40037596B642D4B186800280CDB2C4B2F
:1030E00019784A425141C9B2197004F059FB294B71
:1030F0001B88DF19BFB23751AB6C002B39D00021D0
:10310000254B264FF458A9643A780C340193244D8A
:103110008A4206D02B68032B03D8224AD05C04F0E5
:103120003FFB2B68204A0133134004D50422013BA6
:103130005242134301331B4900228C462B60042B5F
:1031400018D06046C05C591CFF2802D10B00012238
:10315000F5E7002A00D02B60012104F021FB0123B8
:103160003B702B68114A5B009B5AE418019BA4B288
:10317000F450F7BD01235B422B6000233B700C4BE6
:10318000F3E7C046FCA0004000A00040180000206B
:10319000F20500200C00002044050000F10500208D
:1031A000D00500201C000020030000800E0000203D
:1031B00050460000084B094AFF201A805A809A8026
:1031C000DA800023064A07491370074A08704870DE
:1031D0008870C870136070470E000020DC05000086
:1031E000F10500201C000020D00500200122024B28
:1031F00052421A607047C0461800002010B5034ABA
:103200000621034802F09CF810BDC0460CCE000019
:1032100076D50000E12170B54902144803F048FF5B
:10322000FFF718FE0A2004F045F90023FF21104A99
:10323000995401331D2BFBD1012200200D4B0100BD
:103240001A6004230C4A0D4D1468002CFCD02C6825
:103250000002013B20431160002BF5D10122084BF5
:103260001A6004F0E1F801F0CBF870BDB01B00204B
:10327000D405002000D0004000D1004008D5004017
:1032800004D00040F8B50B4E070030000D0003F0ED
:1032900057FF0400A84200DD2C003D00EB1B9C42C0
:1032A00005DD300003F056FF28700135F6E72000F9
:1032B000F8BDC046B01B002010B50100014803F066
:1032C000FFFE10BDB01B002010B5054C200003F020
:1032D00005FFE1212000490203F0EAFE10BDC046CF
:1032E000B01B0020C3070CD4064B1B68834208D8D0
:1032F000054B1B68984204D8031F1B68002B00D0A5
:1033000018007047FC050020F8050020002301226A
:1033100010B50A48990001334250642BFAD1084C89
:10332000084B00211A602000074A08F043F8074BB9
:10333000074A6360074B1A6010BDC046802D00200D
:103340000006002008000020D409000030270000FB
:1033500004060020F405002010B5044B044A1A604E
:10336000044B054A1A60FFF7D1FF10BDFC05002091
:1033700000060020F8050020D40F0020044B1B6835
:103380001868000980B20238C343DB171840704741
:10339000F405002000B59BB00200054901A808F023
:1033A0004DFB01A802F0C2F902F074FCFCE7C04634
:1033B000D8CE00000B4BC20704D4042804D80A4B13
:1033C00000D00A4B180070470F2203681A40031DF3
:1033D000042AF7D0064B092AF4D0064B032AF1D071
:1033E000054BEFE7B2CE000056CA000050CA0000FD
:1033F000BCCE0000CCCE0000C3CE00000020064AA8
:103400000649131F186013681B099BB202339B0007
:10341000D2188A42F5D3704704060020D40F00204A
:10342000F7B50F240126314B314A1968314B324D23
:10343000186813681F002740072F26D813681B0938
:103440009BB202339B00D218AA42F2D300242B4E27
:10345000A500AD192868FFF745FF01342860642CEA
:10346000F6D1274C2068FFF73DFF2060254C2068EF
:10347000002802D0FFF736FF20600025224B1B6892
:103480000093009B9D4214DBF7BD1B099BB29B0080
:10349000D3189A42D2D01F68374208D1B94206D217
:1034A000B84204D3043F3F68002F00D01F60043BA4
:1034B000EFE7F0236B43154A9B181A78002A01D1D5
:1034C0000135DEE71F693C2300266B43DB199B00B7
:1034D00001930136BB1BF3D4019BB4001C1B0B4BA7
:1034E0001C19A069FFF7FEFEA061F2E7FC050020B1
:1034F00004060020F8050020D40F0020802D0020B5
:1035000008000020D40F0020CC050020281C00203B
:10351000F7B50124204246D1234B1B689C469842B4
:1035200041D3224B1B68019398423CD8031F1B6870
:10353000002B38D10200036800941B099BB2002BBA
:103540000FD10099131F196090422CD015682B1FC2
:103550001B68990069180C68013B14600A602A0016
:10356000EDE79D0055192968009C214219D18C4531
:1035700017D8019C8C4214D30E1F3468002C10D134
:103580000F680F343C40072C08D92F60151F2B60A3
:103590000B680A601B099BB20A00D0E700993160F2
:1035A000CDE7013BCBE7F7BDFC050020F805002087
:1035B0000D4970B50A000D4D1368141F1B092668CC
:1035C0009BB2981C002E0BD000238A4200D00B0027
:1035D00023608300C91880001218AA42ECD370BD82
:1035E0001B011360F7E7C04604060020D40F00203B
:1035F000F8B5124C27000F223B681D09ADB21342EB
:103600000DD06E1CB600A74204D032003900200055
:1036100007F0BDFE0022A3190436A4191A60023572
:10362000AD00074B7F199F42E5D31B1B9B10013B4D
:103630001B012360034B1C60F8BDC046040600203C
:10364000D40F0020F4050020F0B59BB0FFF714FC68
:1036500000240700214AA300D0580134FFF758FF87
:10366000642CF7D11E4B1868FFF752FF1D4B1868EA
:10367000002801D0FFF74CFF00261B4B1B689E4221
:1036800017DBFFF795FFFFF7CBFEFFF7B1FFFFF763
:10369000F3FB164BC21B1B6815491B6801A81B09CD
:1036A0009BB2023B08F0CAF901A802F03FF81BB038
:1036B000F0BDF02575430F4BED182B78002B01D191
:1036C0000136DAE72B695C1E002CF9DBA300EB184E
:1036D0009869FFF71DFF013CF6E7C046802D0020EA
:1036E00008000020D40F0020CC050020F4050020A5
:1036F00092CE0000281C0020F7B5174D4F1C2B68F8
:1037000006001B680C001B099BB201929F420BDB59
:10371000FFF79AFF2B681B681B099BB29F4203DBD4
:103720000A20FDF7C5FDFEBD2868A71CBA00DB1BFB
:1037300081181B010B6029600021031F19600F23F2
:103740001E4003002401264340C3083A9A189A42B7
:10375000E9D9019902C3FAE7F4050020F7B503009F
:103760000122134004000D000193002B2BD1174BB5
:103770001B68834227D8164B1B68834223D90F232B
:10378000144F386000681840FFF7B6FF019B3C6893
:10379000061E3B6017D0236804301B099BB29D4274
:1037A00000DD1D00AA00211D251F07F0E7FDFFF722
:1037B00025FE2E60FFF734FE00232B602268064BA7
:1037C0001340236034002000FEBDC046FC050020ED
:1037D000F8050020D40F0020F0FF0F000323043071
:1037E00010B5C11719400918891000220420FFF7ED
:1037F00083FF10BD70B5050008000C00FFF7EEFF59
:103800000023002804D170BDE95CC2181171013396
:10381000A342F9DBE343DB171C40002304192371A7
:10382000F1E7F0B50C009BB0022804DC1C20FDF78A
:103830003FFD1BB0F0BD01230868184206D10428E3
:1038400004D90F2601683140042901D00E20EEE78B
:1038500061680D001D40F9D10429F7D90A6832408A
:10386000042AF3D1A2681A4201D10D20DFE7FFF745
:10387000A1FD06006068FFF79DFDA768010001AC8F
:103880007F103000257002F0BEFF39006423220053
:1038900003F01EF8200008F017F901002000FFF7E0
:1038A000A9FFC6E710B51C4CA544041E02D1FFF7C2
:1038B00095FF0BE002F0C0FE0138062828D805F07D
:1038C00097FB090911182904240000208023DB003C
:1038D0009D4410BD200002F02BFF011B2000FFF7CC
:1038E00089FFF3E7200002F0D1FE430001201843D6
:1038F000ECE780226946D200200002F0DEFE684636
:1039000008F0E2F801006846E9E704210348E6E729
:103910000020CCE70420D9E700FCFFFF20CF000007
:1039200070B50C00022803DC1C20FDF7C1FC70BD43
:1039300001230868184206D1042804D90F2501681C
:103940002940042901D00E20EFE761681942FAD11D
:103950000429F8D90A682A40042AF4D1A2681A4234
:1039600001D10D20E1E7FFF725FD05006068FFF7B5
:1039700021FDA46801006410280002F044FF21002A
:1039800002F081FFFFF78EFFD1E770B50D0001282F
:1039900003DC1C20FDF78CFC70BD0124086820426C
:1039A00006D1042804D90F2102680A40042A01D054
:1039B0000E20EFE76A682242FAD1042AF8D9136888
:1039C0000B40042BF4D1FFF7F5FC06006868FFF705
:1039D000F1FC0100300002F016FF02F098FF4000F9
:1039E0002043D9E7F8B507000C001C20012F0BDDA0
:1039F00001250868284206D1042804D90F2102684D
:103A00000A40042A03D00E20FDF752FCF8BD62687C
:103A10002A42F8D1042AF6D913680B40042BF2D1BC
:103A2000FFF7C8FC06006068FFF7C4FC0100022F26
:103A300014D0A4682C4211D06410300002F0E3FED0
:103A4000050002F0F9FD012811D1002C02DD01353D
:103A5000012C06D12800FFF725FFD7E70124644297
:103A6000EBE7280002F070FE013C0500F0E70228B9
:103A7000F0D1002CEEDD0135012CEBD00022280026
:103A8000110002F093FE02F05FFE013C0500F3E737
:103A900010B501240868044016D04410200005F039
:103AA000D9FD154905F0A4FC07F08AFB03F0D2FF0D
:103AB0000022124B06F03EFD03F074FF07F010FBEE
:103AC00043000120184310BD042810D90F230268B9
:103AD0001340042B07D1FFF76DFC21000A2208F0E8
:103AE000BBF80400DAE7032B01D10430F5E70D2021
:103AF000FDF7DEFBD2E7C046D30237390000D040E5
:103B0000086870B501240500254006D1042804D9B1
:103B10000F2302681340042B03D00E20FDF7C8FBCF
:103B200070BDFFF747FC03782900233B5A425341FD
:103B30001022C01808F090F880239B05C218044B8F
:103B40009A4201D91420E9E740002043E8E7C04643
:103B5000FFFFFF3F10B5034A0621034801F0F0FBC9
:103B600010BDC046F0CE0000E9CE00000020704736
:103B700010B51E20FDF79CFB10BD10B51E20FDF7F3
:103B800097FB10BD10B51E20FDF792FB10BD10B5C0
:103B90001E20FDF78DFB10BD10B51E20FDF788FB24
:103BA00010BD10B51E20FDF783FB10BD10B51E2003
:103BB000FDF77EFB10BD10B51E20FDF779FB10BD93
:103BC00010B51E20FDF774FB10BD10B51E20FDF7CB
:103BD0006FFB10BD10B5034A0B21034801F0B0FB89
:103BE00010BDC0465CCF0000B4CF00000120034BE5
:103BF0001860034B1B68834018437047F80F002080
:103C0000D80F0020F0B5EFF310810123194083F3A2
:103C10001088134C134AA4461268134E013A93407D
:103C2000124F134A002B17D0146803420FD03D687F
:103C30002C60C046C046C046C046C046C046C046CE
:103C4000C0460C4C1568246825605B08EAE76546A9
:103C50002C6014683460F8E781F31088F0BDC0462A
:103C600008050050200000200C050050E40F002043
:103C7000EC0F0020E00F002030B585B001AD0C2224
:103C80000649280007F07AFB0024285D0121013451
:103C9000FFF70AF90C2CF8D105B030BD49D000006F
:103CA000F7B56A46394B01AD13801C239370384B2E
:103CB0002B800A23AB70FFF7DFF8364B364CC01869
:103CC0002368984201D2002323602668002E3DD14C
:103CD0006B469F5D01213800FFF7E6F801360021B1
:103CE000380003F05DFD032EF2D10026AF5D012107
:103CF0003800FFF7D9F801360121380003F050FDF4
:103D0000032EF3D1C8200138C046C046C046C04685
:103D1000C046C046C046C046C046C046C046C04673
:103D2000F1D100212878FFF7BFF868780021FFF76C
:103D3000BBF8A8780021FFF7B7F8FFF79DF8FA2342
:103D400000251B01C01820602800FEBDFFF794F875
:103D5000236800259842F7D3032003F0B1FB060047
:103D6000042003F0ADFB36180A2003F0A9FB0B4B2F
:103D70009B1B181A0A4BA84206DB18600023094A4D
:103D8000236013600125DFE71D60F7E71A1B0000C1
:103D90000304000010270000F00F0020E3030000E0
:103DA000D80F0020F80F00200022054B10B51A6034
:103DB000044B1B68934201D002F0DEFB002010BDD3
:103DC000F40F0020D41A002010B5041E10DA0024CD
:103DD0000A4BA400E25801239340094A09491360A1
:103DE000094A1160094A0A4911600A4A136010BD64
:103DF000FFF758F8A042EADDEAE7C0464CDD0000D4
:103E0000EC0F002008050050E40F0020E00F002018
:103E10000C050050180500502B4BF7B51B680C0023
:103E2000002B03D101204042FFF7CEFF246801267A
:103E3000250035401AD0FF22631012026012104094
:103E4000DAB21043FF221B021204134018431F4B27
:103E50001B68202B06D1B4401D4BA40EA400E358D0
:103E600000021843FFF7CEFE0020FEBD042CFBD954
:103E70000F2322681340092BF6D1FF2763683F0206
:103E80005B100193019B9D42EEDAAB00E3189B6847
:103E9000334216D05A105812D1B238400843FF218D
:103EA000120209040A401043084A1268202A06D167
:103EB0005B009B0E06499B00020258581043FFF717
:103EC000A1FE0135DEE7C046EC0F002020000020F7
:103ED00030D200000200086810B5C3070FD54010AB
:103EE0001823012A03DD4A68042A00D10833054A51
:103EF0001360FEF7F9FFFFF767FF002010BD0120F8
:103F00004042EDE72000002010B50124044002D01B
:103F10004410200010BD042810D90F23026813405C
:103F2000042B07D1FFF746FA21000A2207F094FE7E
:103F30000400EEE7032B01D10430F5E70D20FDF777
:103F4000B7F9E6E70868F8B5C3071AD5FFF7DCFF4D
:103F50000300203B5E2B25D80520434301221D187A
:103F60000020114E9D4219D005211024F75C3C42DF
:103F700000D080180139520064100029F7D10133B4
:103F8000F0E704280ED90F2203681A40042A09D149
:103F90001B099BB2002B05D00379DAE7012340000F
:103FA0001843F8BD0120FCE755D0000070B5086843
:103FB0000D00FFF7A9FF04006868FFF7A5FF621E68
:103FC0000100042A14D8451E042D11D805236B4383
:103FD0009B18012215009D402B00064805682B43C5
:103FE0000360054B1B68002B02D0200002F0C5FACD
:103FF000002070BDF40F0020D41A002070B50868AE
:104000000D00FFF781FF04006868FFF77DFF621E67
:104010000100042A13D8451E042D10D805236B4334
:104020009B1801229A400748036893430360064B9C
:104030001B68002B03D00022200002F09EFA002013
:1040400070BDC046F40F0020D41A0020F0B5050062
:1040500089B008680C00FFF757FF0690022D36DD87
:104060006068FFF751FF0190A068FFF74DFF040063
:104070000127231D661E0793731C0293079B9E4214
:1040800035D0052373430593019B019D05330493AC
:10409000049BAB421ED0042E16D86B1E042B13D8E3
:1040A0000122059B2349013B5B199A409446224A11
:1040B0000B681068069A3A4003920DD062461A4384
:1040C0000A60012200280DD17F000135E0E70124BC
:1040D0000194CDE7029ECFE7624693430B60002830
:1040E000F2D0039A0299280002F047FAECE7019B0C
:1040F0001E1D042E1AD8012C18D1002505273B00BF
:1041000021006B439B1999400B000A4A0135116845
:104110009943094B11601B68002B05D0019B0022BD
:10412000581D290002F029FA052DE8D1002009B018
:10413000F0BDC046F40F0020D41A0020086810B566
:10414000C30703D5FFF7E0FE054B1860054B1B685E
:10415000002B03D0024B186802F010FA002010BDAB
:10416000F40F0020D41A00207FB5A04C2368002B48
:104170000AD19F4A1268002A06D19E4B1B68002B69
:1041800001D0FFF78DFD7FBD9B4D2A68002A26D107
:10419000984A1268002A1BD0FFF782FD0028F2D04F
:1041A000FFF76AFD924B24681A681C60002A16D03B
:1041B000002C14D101AD0C229049280007F0DEF844
:1041C000285D00210134FEF76FFE0C2CF8D1DAE7F0
:1041D000874A1268002AE5D1002BE3D0E0E70021EE
:1041E0001A2003F0DDFA00211B2003F0D9FA002188
:1041F0001C2003F0D5FA2E68012E5CD0022E00D1CF
:10420000A2E0002E50D101363100794C0320236802
:10421000994303F0C5FA0420216801404B425941FB
:1042200003F0BEFA102123680A2019404B4259417D
:1042300003F0B6FA80212368090119404B42594125
:10424000062003F0ADFA80212368090219404B4291
:104250005941072003F0A4FA80212368490219403C
:104260004B425941092003F09BFA802123688902BF
:1042700019404B425941192003F092FA80212368DA
:10428000C90219404B425941182003F089FA802392
:1042900021681B0319404B425941172003F080FA53
:1042A00031001A2003F07CFA2B680321581C05F01A
:1042B00023F8296067E702214D4C17202368194035
:1042C0004B42594103F06CFA082123681820194029
:1042D0004B42594103F064FA80212368C900194018
:1042E0004B425941042003F05BFA802123684901C5
:1042F00019404B4259410A2003F052FA80212368A9
:10430000C90119404B425941032003F049FA802169
:104310002368890319404B425941092003F040FAB0
:10432000802321681B0419404B425941192003F096
:1043300037FA3100062003F033FA3100072003F08A
:104340002FFA31001B20ADE72021294C17202368CC
:1043500019404B42594103F023FA402123681820A9
:1043600019404B42594103F01BFA80212368192060
:1043700019404B42594103F013FA80212368490048
:1043800019404B425941092003F00AFA8021236861
:10439000890019404B425941072003F001FA80215E
:1043A0002368890119404B425941062003F0F8F96E
:1043B00080212368490319404B4259410A2003F0E8
:1043C000EFF980212368C90319404B42594103206A
:1043D00003F0E6F9802321685B0419404B42594100
:1043E000042003F0DDF901211C205BE7F40F00201D
:1043F000E80F0020F80F0020DC0F002049D000005B
:10440000012010B54042FFF7DFFC10BD10B5034A94
:104410000921034800F094FF10BDC04630D30000CE
:1044200078D3000030B502248025094B094AED00FD
:104430009C505C59002CFCD0A124E400884202D39B
:104440000021995030BD8025ED0018514019F5E745
:1044500000E001400405000010B5002806D1C0208E
:10446000B02140028902FFF7DDFF10BDB02080219E
:104470008002C902F7E7000043425841064B404220
:104480001840B0239B02C018036800201A0E532A5C
:1044900001D11B02180A704700C0FEFF30B501248D
:1044A0008025054B054AED009C505C59002CFCD042
:1044B00001600021995030BD00E00140040500007A
:1044C00043425841074B40421840B0239B02C0185A
:1044D000A62310B50902DB05090A1943FFF7DEFF21
:1044E00010BDC04600C0FEFF70B5012480250D4BF5
:1044F0000D4EED009C515C59002CFCD0002902DCD3
:1045000000229A5170BD557814782D022543947875
:10451000013924042543D478043224062C4310C0E6
:10452000ECE7C04600E001400405000070B505005E
:104530004B680A009C1C2100A400FFF7D5FF281936
:1045400070BD0000134B1B68002B0CD08022B023E1
:10455000D2029B0200280BD11A1D5B681B0E522B46
:1045600000D110007047B022C02392025B02F1E735
:1045700082420DD903681B0E522B09D143680233C6
:104580009B00C018824203D903681B0E522BE9D04E
:104590000020E7E7FC100020F0B50020B7B00024B1
:1045A000FFF7D0FF270005002600002D2ED1284D53
:1045B0002868FFF761FF32003B0001900094254915
:1045C00004A807F03BFA04A801F0B0F8224B6420DD
:1045D0001C682B68A0215A425341204A5B42134079
:1045E000B02292029B18E41A6043490204F09EFD37
:1045F000A0225202030000921949220004A807F0E9
:104600001DFA04A801F092F837B0F0BDFF226B68E4
:1046100029689C460233FF180B12013613409C4256
:1046200000DA1C00FF200A14024003926246014097
:1046300001920091039A0B4904A807F0FFF904A81E
:1046400001F074F82800FFF77DFF0500ADE7C046D4
:10465000FC10002082D400000011002000C0FEFFEA
:104660002CD400006ED4000070B50020FFF704FFCA
:1046700004000120FFF700FF844200DA04000A4B27
:104680001D686A42554128001D60FFF7E5FEA02223
:104690006B4252021340054A28009B18044A611CD1
:1046A0001360FFF70DFF70BDFC10002004800100B7
:1046B00000110020F8B50020FFF7DEFE0700012002
:1046C000FFF7DAFE3E00204D0643204C0DD180213D
:1046D000C020C9024002FFF7A5FE01213000FFF70C
:1046E000EFFE1B4B2E6023601DE0874209DD002397
:1046F000B0212B60164B890223602368002001251E
:1047000017E0012380212B60124BC9022360F4E7DC
:10471000120E522A08D0002800D023600E4801F063
:1047200005F8FFF7A1FFF8BD28005A680232920091
:104730009B188B4205D21A68561CE9D10028F2D08A
:10474000D1E72160EFE7C046FC10002000110020F7
:104750000480010004C0020047D4000070B50020AE
:10476000FFF7F0FEFF260500002801D1280070BDEC
:1047700003681C143440FFF7E5FEDA2CF4D1050081
:10478000F2E700008022F0B55200A1B00021674896
:1047900006F010FE802200215200654806F00AFE55
:1047A000644BFF271B681A00049353425A411000C0
:1047B0000592FFF751FE049C0020631E9C415E4B56
:1047C00064421C405D4BE418FFF7C8FF0600002E52
:1047D0002DD10498FFF750FE411C0598FFF770FE9D
:1047E000059A574D534B2C601A60FEF76DFD514BE7
:1047F00064201B68A0215A4253414F4A5B42134038
:10480000B0222C6892029B18E41A6043490204F01B
:104810008DFCA0225202030000924A49220007A800
:1048200007F00CF907A800F081FF21B0F0BD326855
:10483000131412123A403B4003921A000A3A092A12
:1048400049D83A4B039A995C002931D110223E484D
:1048500006F0B0FD35002B6803991A123A409142D8
:1048600009D11A143A400B2A27D0132A2DD00A2A2C
:1048700001D1354B1D602800FFF764FE051EEAD10B
:10488000314B196800290FD02000FFF74FFE0400BC
:104890002D4B5B195968002903D02000FFF746FE15
:1048A000040004350C2DF3D1204B0121039A9954B7
:1048B0003000FFF747FE060089E73B40022BDADCB9
:1048C000214A9B00D3185D60D5E7102200211E48C5
:1048D00006F070FDCFE71A00153A082AE8D8144A06
:1048E0000399525C002AE3D13500152B00D0150046
:1048F000300003681A143A40152A0FD01D2A00D13F
:104900000025FFF71FFE0028F3D1002D04D0200062
:104910002900FFF70BFE0400054BC6E7039A1B12A4
:104920003B409A42EDD10500EBE7C046FC0F00206A
:1049300004110020FC10002000C0FEFF04C0020093
:104940000011002011D40000102F002010B5FFF737
:1049500019FF10BDF0B585B0039203220333DC17B5
:10496000294D1440E4182B68284F5A4253418022A5
:104970005B42D202A4103B409B18A21C0291244E21
:10498000910000910190316800980A18934215D265
:10499000FFF7F8FE2B685A42534180225B421F40CA
:1049A000D202BF183368009A9B189F4206D219485A
:1049B00000F0BCFE0025280005B0F0BD029B356864
:1049C00019066B461A7BA423DB051343FF222F0035
:1049D000090C1943019B12041B04134019432800BE
:1049E000FFF75CFD0837281D21003760FFF756FDF3
:1049F000002C04D00A9A21003800FFF775FD009BB7
:104A0000083BFF183760D6E7FC10002000C0FEFF0F
:104A100000110020EBD3000070B59AB0FFF74AFEFA
:104A2000FF221E4CD2000021200006F0C3FCFF250F
:104A3000FFF794FE0026002814D10200C300E358BB
:104A40000130591E8B41D218FF28F7D1144901A813
:104A500006F0F4FF01A800F069FE124800F066FEBF
:104A60001AB070BD03681A142A400A2A0AD11A1211
:104A70002A40FF2A03D0D200A1180B71A050FFF7E3
:104A800061FDD8E7132AFAD11B122B40FF2BF6D079
:104A9000DB00E2181671E650F1E7C04688250020D9
:104AA000B7D40000CBD400000021094B094A59605B
:104AB0000131516059680029FCD00021196101239E
:104AC00093600222044B8131FF315A501A607047C3
:104AD000FC1000400010004000E100E00222064B04
:104AE0000121DA670022054B5A61054A11615A69B2
:104AF000002AFCD07047C04604E100E0FC100040F2
:104B00000010004010B5044C2378002B01D0FFF7B3
:104B1000E5FF0020207010BD051200208023012039
:104B20005B055B6E5B001843704700000120024B81
:104B30001B685B0018437047881200200120024B5D
:104B40001B685B0018437047240000200120024BC3
:104B50001B685B00184370478C12002070B504007E
:104B60000D001600FEF792F9802301215B055A6EB5
:104B70002670002653006170E1706272010A5A0AC1
:104B80006071A171A272010C5A0C000E5B0EA6702E
:104B90002571E1712072E272237370BD10B5044C6F
:104BA000200006F091FF01002000FEF723FE10BD5B
:104BB000911200200E4B10B51B680E4C5A1C0FD0E2
:104BC0000D4C002B0CD00D4C012B09D00C4C022BA2
:104BD00006D0094C042B03D00A4C052B00D1074CFE
:104BE000200006F071FF01002000FEF703FE10BD5B
:104BF000280000205CD50000E4CD000067D500004F
:104C0000EBCD000061D5000070B5214C2278002A60
:104C10003DD1204B01215A608022D20511605A6893
:104C2000002AFCD0002207201B4B1C4901255A50AA
:104C30000439585008315A5019481A4958501A49DD
:104C40001A485A501A495A50A622D2009D5008229A
:104C500018495A50043158500220174958501749E2
:104C600017485850174804395850182016495850BA
:104C7000C12189005A500539FF395858921802430A
:104C80005A501249124A9950FFF70EFF257070BD15
:104C900005120020FC000040001000400C05000040
:104CA000746962751C0500002405000020000402E0
:104CB0002C05000014050000340500003C05000030
:104CC000FFFF000021100100540500000612002023
:104CD0000405000070B50E4B06001B78002B01D1B7
:104CE000FFF792FF00200B4D2C7884420ED00A4B28
:104CF000202219780323091B1940084B4901C918C0
:104D0000300006F03BFB0120013C2C7070BDC0461A
:104D1000051200209012002004120020061200202C
:104D2000002370B588B0984235DD0D6801262C004F
:104D300034409C422FD12300042D2CD90F222B6804
:104D40001A402300092A26D16A683F2A23DD6846D3
:104D5000FFF7C0FF230000281DD06B4619783300F1
:104D6000A14203DB6B461B5D5B003343A200AA1824
:104D700001349360202CF2D1092169444A780B78E0
:104D800012021A438B781B041A43CB781B06134379
:104D9000024A13600423180008B070BD8C12002072
:104DA00070B5454B8AB01B78002B01D1FFF72CFF63
:104DB00002AC2000FFF78EFF002802D100200AB0CD
:104DC00070BD23780B2BF9D96378012BF6D1E378EA
:104DD000012BF3D100231120384E394D33602B7055
:104DE00068442379374A41781360027809021143F5
:104DF000827812041143C27812060A4332490A60CB
:104E0000002B0ED1152169444A780B7812021A43FF
:104E10008B781B041A43CB781B06134333600023A3
:104E200018E0012B1AD1152169444A780B78120237
:104E30001A438B781B041A43CB781A211B061343A1
:104E400033600E23627C6944934200DD130000222C
:104E50009A422CD100220420EA54B0E7022B03D15D
:104E6000627B10331621EEE7042B0DD115210822A9
:104E70006944684606F082FA0098019902F002FD42
:104E800006F02EF93060CAE7052BC8D1152108229B
:104E90006944684606F072FA0098019902F0F2FC43
:104EA00006F01EF93060627D0A231E21CBE7885C84
:104EB000A8540132CCE7C046051200208812002019
:104EC00091120020280000208C12002010B5134BF6
:104ED00004001B78002B01D1FFF796FEFFF7FEFDC3
:104EE00000200F4A0F49104B545058600130106099
:104EF00058680028FCD000201861013090601869C3
:104F00000028FCD0094B0A481B785B011B18535042
:104F1000FFF7E4FDFFF7C8FD10BDC04605120020F5
:104F20000010004004050000FC10004004120020A6
:104F30000612002010B588B000281DDD0A68012186
:104F400013000B4018D1042A16D90F2014682040F2
:104F5000092811D150683F280EDD9800101880688C
:104F60000024084201D04010C4B26846C454013342
:104F7000202BF2D1FFF7AAFF002008B010BD0000DF
:104F800010B5002813DD0C68E30710D56410532C0E
:104F90000DD8084B1B78002B01D1FFF735FEFFF72A
:104FA0009DFDA123044ADB00D450FFF77DFD0020C6
:104FB00010BDC046051200200010004010B50028AA
:104FC0000EDD0C68E3070BD56410FF2C08D8054BE9
:104FD0001B78002B01D1FFF717FE034A034BD45077
:104FE000002010BD05120020001000402405000024
:104FF00013B5002814DD0C68E30711D5094B6410C4
:105000000093094B0193072C0AD8084B1B78002BFF
:1050100001D1FFF7F9FD6B46054A1957054BD150F1
:10502000002016BDE2ECF0F4F8FC000405120020AC
:10503000001000400C05000070B588B0002820DD8D
:105040000124086804401CD104281AD90F230268DF
:105050001340042B15D1FEF7ADF9060006F034FD20
:105060000500122800D912252A0002210D326846B7
:10507000FFF774FD6B465D73A54205DC6846FFF7DC
:1050800025FF002008B070BD2300325D6B449A7389
:105090000134F1E7F0B50D008BB0012832DD08686E
:1050A0000122040014402DD104282BD90F230168BC
:1050B0000B40042B26D16B68134223D0FEF77AF9FC
:1050C0006E6807007310019306F0FEFC05000E28C1
:1050D00000D90E252A000121113202A8FFF73EFD5A
:1050E0006A46127902AB5A7302AA73129373019B38
:1050F00076141B0ED67313745574A54205DC02A8F2
:10510000FFF7E4FE00200BB0F0BD3A5D02A9631882
:105110009A740134F1E730B589B0002814DD0C68C9
:10512000E30711D5102268460021FFF717FD6B46F3
:105130006A4665105D73684663122D0E641493739E
:10514000D4731574FFF7C2FE002009B030BD000013
:10515000174B184A5968002903D0002159600131C2
:105160009160196900291FD0002018618023DB009D
:10517000D3581149012B18D1A923DB00D3585B4226
:105180000B600E490B78032B01D801330B70032001
:105190000B490B78013303400B700A495B015B1824
:1051A000094953500123936070470860FAE7C046ED
:1051B000FC1000400010004024000020901200204D
:1051C00004120020061200200405000010B5034A56
:1051D0001021034800F0B4F810BDC046DCD4000034
:1051E000D3D40000044A05491368C85401339B0511
:1051F0009B0D13607047C046C0160020C0120020EF
:1052000070B5114C114A2368834202DC00232360ED
:1052100016E0155C411C2E00FA3E012E05D899427D
:105220000FDA555C013D1F2D01D90800ECE70100A4
:10523000151A565C6E5401318B42FADC181A206044
:1052400070BD1570FAE7C046CC1A0020CC160020BD
:1052500010B5FDF711FE064B1A68824201D90022F3
:105260001A601B68C31A034898428041404210BD2F
:10527000BC120020204E000010B5094C094A2368DA
:105280001268934200D110BD074AD05CFEF714F8B3
:105290000028F8D0236801339B059B0D2360ECE7C1
:1052A000C4160020C0160020C012002010B5040053
:1052B000064B074A1B6812689B1ADB439B059B0D34
:1052C000A34200DB10BDFFF7D7FFF1E7C0160020B7
:1052D000C4160020F7B5050056680191B000441CC3
:1052E00006301700FFF7E2FFFB20FFF77BFF1C20D3
:1052F000FFF778FFE8B2FFF775FFE0B22412FFF77F
:1053000071FFE0B2FFF76EFF6B461879FFF76AFF97
:105310000025AE4200DCF7BDAB00FB189C680135F0
:10532000E0B2FFF75FFF2012C0B2FFF75BFF20146F
:10533000C0B2FFF757FF200EFFF754FFE9E7000068
:1053400070B5074E33680B2B08DC0C255D43054C0C
:105350000133285164196160A260336070BDC0469A
:10536000C8160020202F002010B5FBF7A9FEFFF77C
:105370004DF8FBF7C9FEFDF741FFFEF7EBFBFEF72B
:1053800029FCFFF723FF00F015FF01F0F9F801F009
:1053900043FB10BD962210B512010021034806F010
:1053A00009F80022024B1A6010BDC046281C0020DC
:1053B000CC050020064B074A1B6812689B1ADB438A
:1053C0009B059B0D0122834200DC002210007047E8
:1053D000C0160020C4160020F8B505000C00160009
:1053E0001F1E0ED10320FFF7E5FF002808D0FA208A
:1053F000FFF7F8FEE8B2FFF7F5FEE0B2FFF7F2FEC6
:10540000F8BD501DFFF7D6FF0028F9D0FB20FFF7AD
:10541000E9FEE8B2FFF7E6FEE0B2FFF7E3FEF0B226
:10542000FFF7E0FE3012C0B2FFF7DCFE3C00E31BEA
:105430009E42E5DD2078FFF7D5FE0134F7E7000056
:1054400070B50024F0250B4B1B68A34202DCFFF76C
:10545000A1FF70BD2B006343074A9B181A78002AEE
:1054600005D05978002311201A00FFF7B5FF013449
:10547000E9E7C046CC050020281C0020F8B507004D
:105480000024F0252B0063430C4A01349E18B742D8
:1054900011D0317800290BD00133D15C00231120C9
:1054A0001A00FFF799FF2A000021300005F082FF63
:1054B0000A2CE7D1F8BD024B1C60F9E7281C00203C
:1054C000CC050020F0B5150001222F00754C1740C7
:1054D000A54401900291002F11D005AB1A706A10FB
:1054E0005A70120E1A710522691299706D14029980
:1054F000DD70FFF771FFCF239B009D44F0BD042DAD
:105500001ED90F202A681040042826D1022304AA9D
:1055100028001371FDF74EFF040006F0D5FA624B28
:10552000984200D91800B84204DC421C05AB02992D
:105530000198DEE701377B1EE35C05AAD355F2E74D
:10554000042D00D0A9E0032304AA043D13716B428B
:105550005D4105AB55710222E9E709287ED104229D
:1055600005AB1A706A6851100091694652120978A9
:105570009A70009A59701F2A01DD202200926A4613
:10558000127806ACDA70009BBB4202DC05ABE21A73
:10559000CDE70126BB00EB189868064006D1042829
:1055A00037D90F210368194002290CD10123237038
:1055B0004310637042121B0E4014A270E0702371FE
:1055C00005340137DFE7042921D102232370FDF7D9
:1055D000F1FE039006F078FAA31C0C2809D860703D
:1055E000864201D19C19ECE7039A925D9A550136E7
:1055F000F6E70C226270039A925D9A550136092EE5
:10560000F9D12E23E372237363730E34D9E7012992
:1056100007D1032304382370434258416070023499
:10562000CFE7092909D10423237043685A10627017
:105630005B12A370E6700434C3E703290BD1052382
:1056400023700068020992B2430F92000B40D31AF4
:1056500063701B12EDE726700134B2E7032800D017
:1056600049E7052105AB1970110989B2520F89006C
:1056700002408A1A111299705A701100642A00DDD2
:1056800064210420D970C9B2041FA14201DC043294
:105690004DE72C5C1C540130F6E7002D00D02AE7C2
:1056A00051E7C046C4FCFFFF2303000070B50200B1
:1056B0000024F0210D4E0800604380194578954282
:1056C00003D001340A2CF6D170BDF022002105F080
:1056D00071FE074A1368013BA34200D11460002306
:1056E00029001A001120FFF777FEEDE7281C0020A3
:1056F000CC05002010B5B2B002236A460400137036
:1057000006F0E2F9C72800D9C7200023984207DC39
:10571000421C6B46FE211420FFF75EFE32B010BD26
:10572000694601335A1EA25CCA54EFE730B5B3B0E4
:1057300002236A460500137006F0C6F90400C72864
:1057400000D9C72400239C420BDC20003230FFF735
:10575000ADFD621C6B46FF211420FFF73DFE33B008
:1057600030BD694601335A1EAA5CCA54EBE70000FB
:10577000F0B5BBB004900C00012803DC1B20FBF744
:1057800097FD51E02A4B08680293C30709D4042807
:1057900007D90F2302681340042B02D1FDF70AFE3C
:1057A0000290234B60680393C30709D4042807D9E8
:1057B0000F2302681340042B02D1FDF7FBFD039079
:1057C00000271C4B1B680693069BBB420BDC039B0C
:1057D000194A0093C821029B08A806F0FDF808A802
:1057E000FFF7A4FFCAE70C267E43144B0299F61874
:1057F000306806F05FF9051E05D17368B668079337
:10580000079B9D4201DB0137DEE73068039905966F
:1058100006F050F90836002808D121000498059BAD
:10582000083102385B6898473BB0F0BD0135E7E7C7
:10583000E8CE0000C816002038D60000202F002037
:10584000F7B5234B06001B68F02100930023009A54
:105850009A4211DC0024F0231A006243019201995C
:105860001C4A55182F78002F12D001340A2CF3D17E
:105870001948FFF75BFF29E00A005A4315488218D0
:105880005078B04202D11278002A1FD10133DEE7EE
:10589000F0223900280005F08DFD02230D4A019900
:1058A000EB6053540D4AF1008A58009B6E70AE7045
:1058B000AA602F616F61A34202DC054B01341C60BA
:1058C000002331001A001020FFF786FDF7BDC04607
:1058D000CC050020281C002081DA0000882500204B
:1058E00010B5FFF7ADFDFF24084AE3005B429B18AB
:1058F000074AD35C043B012B03D8E043C0B2FFF757
:105900009FFF013C002CEFD110BDC046FC070000FA
:1059100088250020F7B50F00FF247F2501901E4A3F
:10592000E300D31A1D4A9A181278062A01D0032AD6
:1059300020D1FF22D2009B18186883682B401C2BB3
:1059400018D1C3681A002A40042A13D102692A40D8
:10595000192A0FD11B0A01339B000C30C018FDF728
:1059600029FD03780600002B10D006F0ADF80023C7
:10597000B84209D0013C002CD1D1F7BD019AF15CAD
:10598000D25C9142F6D101339F42F7DCE043C0B2D2
:10599000FFF756FFEEE7C04688250020FC07000011
:1059A00070B50500FF24084AE3005B429B18074AD4
:1059B000D35CAB4203D1E043C0B2FFF741FF013CEF
:1059C000002CF0D170BDC046FC07000088250020E7
:1059D000F7B5FDF751FA514B1A68824201D90022FE
:1059E0001A601A684E49821A8A4200D883E0186009
:1059F000FDF74CFA071E00D101370020FDF738FBF8
:105A000001900020FDF748FB019B0090454C464D5E
:105A1000002B14D02368002B00D07AE02B6827607D
:105A2000002B00D171E0414B01261B78002B63D184
:105A30000920FFF7B5FF3E4B1E703C4B1E70009BCC
:105A4000002B12D02B68002B0FD123682F60002B66
:105A50001ED0374B01261B78002B52D10920FFF7AF
:105A60009FFF334B1E70314B1E702368002B0FD0ED
:105A70002F4E3278002A0BD19F4200D22760236834
:105A8000FB1A312B04D90720FFF78AFF012333705B
:105A90002B68002B0FD0254E3278002A0BD1BB4249
:105AA00000D92F602B68FF1A312F04D90820FFF787
:105AB00077FF012333702368002B0CD0019B002B50
:105AC00009D11B4E3378002B02D10720FFF768FF66
:105AD0000023236033702B68002B0CD0009B002B1D
:105AE00009D1124C2378002B02D10820FFF758FF70
:105AF00000232B602370F7BD0720FFF751FF0C4BED
:105B00009CE70820FFF74CFFADE7009B002B9CD1E2
:105B1000ABE7009A002A95D1AAE7C046B812002048
:105B20000F270000A8120020B0120020B41200209D
:105B3000AC12002037B500240500FFF781FC01A856
:105B40000194FDF783FA21002000FEF72DF9FEF7FE
:105B50000BFBFDF72FFBFDF749FBFEF751FCFDF7B3
:105B6000B1F9A54204D0FDF7D1FB0248FFF7DEFDF5
:105B700037BDC04672DA0000002310B501001A00DC
:105B80001120FFF729FC10BD07B56B461970694657
:105B90005A7013128B701314120ECB700A716B466D
:105BA000010005221320FFF717FC07BD10B50A00FE
:105BB00001001220FFF786FC10BD70B5050008003B
:105BC0000C003230FFF772FB2B00220000211B205B
:105BD000FFF702FC70BD10B50C000300110014208B
:105BE0002200FFF7F9FB10BD012370B5FF24084A1E
:105BF00041185B42884201D3D84370BD06781D0A24
:105C0000234073409B009B5801306B40F2E7C04635
:105C100054D60000002313B501930B4BC2000400BF
:105C2000D058002805D0436808309900FFF7DCFF02
:105C300001900920FFF73AFB01AB04222100172055
:105C4000FFF7CAFB13BDC04688250020F7B50190B9
:105C5000FEF784FD01250400FF276D42002C01D1D1
:105C60002800FEBD266833143B40152B0DD12100C2
:105C70000198083105F01EFF002801D135123D4082
:105C80002000FEF75FFC0400E8E71D2BF8D101259A
:105C90006D42F5E7F0B580279DB0FFF7EDFAA54C12
:105CA000A54D2068FF00391A4019FDF7EBFA23686B
:105CB0000600C3182360002B0ED11DB0F0BD206874
:105CC000391A2818FDF7DEFA236806001B1823602E
:105CD000FDF7D2F8994B1860002EF0DC2B78FA2BE8
:105CE00000D037E12368022B07DCFFF7B1FA002868
:105CF000E3D00120FFF784FADFE76878AC78023858
:105D000018282BD803F07EF919002C00300034003D
:105D1000370040002A004A007C0086008A00A0006C
:105D2000F10002012A002A002A002A002A002A0083
:105D30002A002A002A002A001001FF2C0ED0200081
:105D4000FFF7B4FC00227E4BE100CA505B181A71C9
:105D50002100009213001320FEF7FCFD0320C9E789
:105D60002000FFF76DFDF9E72000FFF79FFCF5E746
:105D7000FFF7B6FDF2E7FFF763FB0020FFF7DAFE5F
:105D80007048FFF7D3FCE9E7632CE7D86E4BA2001D
:105D9000D25821001520FFF795FBDFE7FEF7DEFC68
:105DA000FF270400002CD9D025682B143B40152B6D
:105DB00004D02000FEF7C6FB0400F3E72000083003
:105DC00005F082FE06000530FFF770FAFB20FFF7B2
:105DD00009FA2D121D20FFF705FAE8B2FFF702FAC3
:105DE000F0B2FFF7FFF93012C0B2FFF7FBF9250060
:105DF0002B1B9E42DDDD287AFFF7F4F90135F7E72A
:105E000000211D2000910B000A00FEF7A3FDFDF705
:105E10007DFAA3E72000FFF7FDFE9FE7FDF73EF8C0
:105E200003AC4A4A64210090494B200005F0D4FDA0
:105E300002232000237005F047FE2300020000210A
:105E40001620FFF7C9FA89E700243D4AE300D55838
:105E5000002D27D06B689E00701DFFF727FA2B00DE
:105E600000253200083321000120FFF7B5FA2F008A
:105E7000FEF774FC2E00002818D1002F04D03A0041
:105E800001212000FFF726FA002D04D02A0002216C
:105E90002000FFF71FFA002E04D03200002120005E
:105EA000FFF718FA0134FF2CCFD157E7FF21036821
:105EB0001A120A40A24209D11A140A400B2A08D128
:105EC0000B400CD0012B0CD0022B0CD0FEF73AFB70
:105ED000D1E7132AFAD100252F002E00F6E706009D
:105EE000F4E70700F2E70500F0E70024FFF7A8FA5F
:105EF0002200210000942300DA20FEF72BFDFF2270
:105F00002100D2000E4805F055FA80E7012C02D19D
:105F1000FEF742FB22E7022C02D1FEF717FD1DE738
:105F20000120FFF707FE19E7002321001A001A20BD
:105F300087E7C046CC1A0020CC160020BC120020F7
:105F40008825002054DA0000802D00206BDA000044
:105F500066DA0000FB2B00D0CBE62268042A00DCC6
:105F6000C3E62E79E878574B360206439E4200DDA1
:105F7000BFE6331D9A4200DCB7E6EB5CFE2B00D097
:105F8000B7E66B78AC78771E1B2B61D019D8072B3E
:105F900047D0082B1CD0012B18D1FF2C16D0200085
:105FA000FFF784FB6D79484AB31E009221002A0056
:105FB0000A20FEF7CFFC454BE400E0501B191D7191
:105FC00004E01D2B56D048D31E2B6AD0701D91E6DD
:105FD000632CFBD86A79022A13D0032A1BD0012A2A
:105FE000F4D1E979AB79090219432B7AA4001B0497
:105FF00019436B7A1B060B435B001343344AA350CF
:10600000E4E7002FE2DDB11E2F48FDF7F3FB304B34
:10601000A400E050DAE7AB79A4005A1E93419B003C
:10602000ECE7632FD2DC03AD3A002A49280005F0E3
:10603000A5F900232800EB55FFF708FE0028C5DB73
:10604000234B8000C25821001520FFF73BFABDE723
:1060500039002048FFF75EFCB8E7FF2CB6D06A791C
:10606000022AB3D818490B2000912100B31EFEF775
:1060700071FCABE7632F00DD6327002303A99F4278
:106080000ADCFB430022DB173B40CB181A701520BB
:1060900000917B1C2100EAE7EA185279CA540133C7
:1060A000EDE7012C92D1002F90DD6B79002B03D00E
:1060B0001C00322B00DD322464235C43064B1C6041
:1060C00084E7C046F6030000D21600208825002091
:1060D000802D0020D1160020040000200122094B51
:1060E0001A60094A1368002BFCD00322074B1B6877
:1060F000D8171040C01801238010063840001843FC
:106100007047C04600C0004000C1004008C50040C4
:106110000120704710B5064C200000F0B3FD054982
:10612000200000F0D7FD0122034B1A6010BDC046CD
:10613000F81A0020801A0600D01A002010B501219C
:106140000D20FCF7B1FE01210E20FCF7ADFE002171
:106150000F20FCF7A9FE044C200000F0CFFC10211A
:10616000200000F0E7FC10BDD81A002010B504682C
:106170000D20E30703D56410FF2C03D91720FBF78C
:1061800097F810BDFFF7DAFFE1B2024800F0F4FC27
:106190000020F6E7D81A002010B5FFF7CFFF002146
:1061A000034800F0E9FC43000120184310BDC0463D
:1061B000D81A002010B5034A08210348FFF7C0F899
:1061C00010BDC04698DA0000D8DA00000D4B70B55B
:1061D0001B6804000E001500002B01D1FFF79AFF89
:1061E000E1B2094C200000F00CFEF1B2200000F0FA
:1061F0000FFDE9B2200000F00BFD200000F06CFE66
:1062000070BDC046D01A0020F81A002010B5012435
:106210000368234205D04168214202D082682242AD
:1062200003D10D20FBF744F810BD5810802801D988
:106230001520F7E74910FF2901D91620F2E752107F
:10624000FF2A01D91720EDE7FFF7C0FF0020EBE799
:10625000F7B501221400904222DD0D682A421FD0BA
:106260001D4B15411B684C68002B01D1FFF752FFF5
:10627000E9B201272500194E3D40300000F0C1FD74
:10628000002D0FD03C413000E1B200F0C1FC3000E5
:1062900000F022FE0024A04202D02320FBF708F8E1
:1062A0002000FEBD042CF2D90F2322681340092BD5
:1062B000EDD163685B100193019BAB42E7DDAB005E
:1062C000E3189968394204D04910C9B2300000F08F
:1062D0009FFC0135F0E7C046D01A0020F81A0020D4
:1062E000144B70B51B6805000E00002B01D1FFF7A1
:1062F00011FF114CEDB22900200000F082FDF1B237
:10630000200000F085FC0021200000F085FD002821
:1063100001D0404270BD01222900200000F06CFD38
:10632000200000F066FC0028FAD0200000F066FC97
:10633000F0E7C046D01A0020F81A002010B501245A
:106340000368234202D04168214203D10D20FAF7AD
:10635000AFFF10BD5810802801D91520F7E749106C
:10636000FF2901D91620F2E7FFF7BAFF40002043CA
:10637000EFE70000002370B5344D0400EB56013305
:106380000BD10D211D20FFF7ABFF5A2814D101229C
:106390002A212A703D38FFF719FF0023EB56022B04
:1063A0002AD0032B49D0012B4CD121001D200124E0
:1063B000FFF796FF644225E00F211920FFF790FFB9
:1063C000332805D102235F222B7020211A38E2E7FF
:1063D0000D211E20FFF784FFC7280AD103230022C6
:1063E0002A21A9382B70FFF7F1FE1B222A211E203B
:1063F000D1E700232B70D0E7012C13D129211920DC
:10640000FFF76EFF7F2801DD0138FF3803007F337F
:1064100001DA7F20404264237F21584302F086FE48
:10642000604370BD032C0BD12B211920FFF758FFBF
:10643000043CE7E72D211920B9E721001E20B6E72B
:10644000052CF7D0012400206442E4E72C00002052
:1064500070B50120FFF78EFF04000320FFF78AFFCD
:1064600005000520FFF786FF6D4364434043641930
:10647000201804F06BFE01F035FB04F031FE430000
:106480000120184370BD10B50120FFF773FF4300D2
:106490000120184310BD10B50320FFF76BFF430028
:1064A0000120184310BD10B50520FFF763FF43001E
:1064B0000120184310BD0000F8B501231C009842CC
:1064C00029DD0F683B4226D04E6835001D4022D1A1
:1064D000042E20D90F2231680A40092A1BD1736883
:1064E0005C10202C00DD2024134B1B68002B01D1F5
:1064F000FFF710FE7F10F9B2104F2200380000F0B5
:106500007BFCA54214DA380000F073FB002804D1AC
:1065100001246D002C432000F8BD380000F06EFB14
:106520000122AB004000F31810439860AD18E8E773
:1065300064000125EEE7C046D01A0020F81A0020BA
:1065400000207047012070470020704700207047EE
:1065500001207047002070470020704700207047DE
:1065600000207047002070470020704700207047CF
:106570000020704700207047704770477047000048
:1065800010B5034A0E210348FEF7DAFE10BDC046DF
:1065900028DB000098DB00000378013B1F2B00D9AB
:1065A00070470130F8E710B5FFF7F6FF0378002BCE
:1065B0000BD00130222B11D10378002B03D0421CC9
:1065C000222B03D11000FFF7E7FF10BD5C2B03D196
:1065D0004378002B00D0821C1000EDE73A2BF2D05C
:1065E0002C2BF0D07B2B0BD1FFF7D6FF0378002BA1
:1065F000E9D07D2B01D10130E5E7FFF7D4FFF5E7C6
:1066000020225B2B14D1FFF7C7FF0378002BDAD0D1
:106610005D2BF0D0FFF7C7FFF7E7202BD3DD2C2B46
:10662000D3D0190091435D29CFD0222BCDD001309A
:106630000378002BF1D1C6E7002210B5904216D0A6
:10664000FFF7AAFF03780422222B10D0023A7B2BFB
:106650000DD0013A5B2B0AD01900303902320929DA
:1066600005D92D2B05D14178303909290AD81000D8
:1066700010BD0522742BFAD00132662BF7D00132FF
:106680006E2BF4D0581E83415A42F0E770B5FFF7E5
:1066900083FF037801222D2B01D18018023A0023B9
:1066A0000A2502E06B430130CB1801783039CCB2B7
:1066B000092CF7D95A43100070BDF8B50C0015002D
:1066C000FFF76AFF0378222B02D000232370F8BD66
:1066D0000D236A1E210008250C260A279C4601303E
:1066E0000378222B02D100230B70F0E7002BFAD0A5
:1066F000441C5C2B0BD14378841C622B0ED0662B80
:106700000ED06E2B0ED0722B0ED0742B0ED0002A12
:10671000E9DD0B70013A01312000E1E72B00F6E7DB
:106720003300F4E73B00F2E76346F0E70923EEE7C6
:1067300010B50400FFF737FFA04202D90378202BE1
:1067400000D910BD0138F7E710B5002815D003783F
:10675000002B13D0FFF720FF2021037802008B438A
:1067600000205D2B09D01000FFF71DFF03782C3BA4
:106770005A425341C018FFF70FFF10BD1800FCE745
:106780000300002070B50C0081420EDD1A785B2AF0
:106790000BD1581CFFF700FF0125AC4205D0FFF7D5
:1067A000D3FF002801D00135F7E770BD70B50C00AC
:1067B0001500002901D000230B70002820D0037899
:1067C000002B1ED0FFF7E8FE037806002C2B03D128
:1067D0000130FFF7E1FE0600337800207D2B0FD05B
:1067E000844204D02A0021003000FFF766FF300009
:1067F000FFF7D9FE03783A2B02D10130FFF7CCFE28
:1068000070BD1800FCE7F0B50D0004009DB02E78B7
:10681000002E35D02E21280005F03EF9071E14D099
:10682000431B0193303E092E14D82800FFF72EFF9A
:1068300001002000FFF7A4FF0400002C20D0002F4F
:106840001ED0019B0133ED18E1E7280005F03CF96B
:106850000190E7E723787B2B11D1601C642203A908
:10686000FFF7A4FF041E0BD0019A290003A805F02E
:1068700032F90028E1D02000FFF795FEEEE7002472
:1068800020001DB0F0BD70B5050000200C00814255
:106890001DDD2800FFF7D0FE0300681C012B14D07B
:1068A0000020022B13D10022681C1100FFF77EFF8D
:1068B000012C0CD0FFF748FF00221100FFF776FFF4
:1068C000013CF5E7FFF740FF013C012CFAD170BD18
:1068D000F8B5050000200C0016001F0081420DDDF8
:1068E0002800FFF7A9FE03000020022B06D1681C38
:1068F0003A003100FFF75AFF012C00D1F8BDFFF735
:1069000023FF3A003100FFF751FF013CF4E710B5D7
:106910000024A04218D0FFF73FFE03787B2B0AD15A
:10692000013000221100FFF741FF00280CD0FFF7D3
:106930003AFE0134F5E75B2B06D10130FFF704FF87
:10694000002801D00134F9E7200010BDF8B5002877
:1069500016DD0D68EB0713D56D10013D0124FDF721
:10696000FDFE0026FF27644200280CD1002E21D016
:10697000300005F0A9F801003000FCF73BFFF8BD3E
:1069800001256D42EAE703681A143A40152A0BD133
:106990001B123B409C4200DA1C009D4201D10600C4
:1069A0000836FDF7CFFDDFE71D2AFAD101240026C6
:1069B0006442F6E70120013464002043DFE7000071
:1069C00010B508680C00FCF7F5FCFFF73FF900284C
:1069D00003DB6268024B8000C250002010BDC0463D
:1069E000802D002010B50868FCF7E4FCFFF72EF9B5
:1069F0000123002802DB024B8000C358180010BDA1
:106A0000802D002010B50868FCF7D4FCFFF71EF9B4
:106A1000C043C00F800010BD10B5034A04210348D5
:106A2000FEF78EFC10BDC04628DC000021DC000013
:106A300010B5FCF7EFFBFCF78FFCFEF795FC044864
:106A4000FEF774FEFDF7E8FFFEF74AFF10BDC046F3
:106A500077DC000010B5FCF7D5F810BD70B5002547
:106A600004AC24780573A94205D10A4B0A4A2321B4
:106A70000A4804F015FC01600949920052589B0035
:106A800002715B58A40083716358856043710223CF
:106A9000C37170BD8FDC0000EEDC00009DDC0000E7
:106AA0004CDD0000037B002B04D14373837303612F
:106AB00001330373704700001FB50191A02100242A
:106AC0000068C900D2B24450012A10D0A24209D0B5
:106AD000032A0AD0074A8350074B019AC250012368
:106AE00043501FBD02221343F4E70422FBE70622B2
:106AF000F9E7C046540500002405000010B5040065
:106B0000FFF7D0FFA1222368A179D20099506179C3
:106B1000064A20009950217904329950044B196893
:106B20005A689B68FFF7C8FF10BDC0460C050000FF
:106B3000EC1A00204BB2002B0FDB80233F290FD82B
:106B40001F290FD80F290FD807290FD803290FD8CD
:106B50001B060168074A8B50704780239B04F8E7A7
:106B6000DB04F6E71B05F4E75B05F2E79B05F0E7BE
:106B7000DB05EEE7240500000368074A99501A0078
:106B8000FC32D1680029FCD0A321C9005858002349
:106B9000C0B2D3607047C0461C05000007B5802214
:106BA000074BD2051A6000229A6002321A710F2335
:106BB0000C3200930349023B0348FFF74FFF07BD28
:106BC000EC1A002000300040D81A0020F8B505006B
:106BD0000E0017000024BC4208D02B68315D1B68F2
:106BE00028009847002801D00134F4E72000F8BDC0
:106BF000704710B51C3000F0A9F910BD10B51C305D
:106C000000F096F910BD10B51C3000F0A5F910BDCC
:106C100070B5437E0D00002B01D1002070BD6430A3
:106C2000040000F0A2F90028F7D12000290000F0AC
:106C300070F90120F2E70000F7B50193FA2300256F
:106C400004009B0083600D4B4560083303601C30DB
:106C50000F00160000F052F92000643000F04EF9E9
:106C6000074A2761B600B35820006375019B9B005B
:106C70009B586576A576A375FEBDC0462CDD000049
:106C80004CDD00000123A022C375837D0E49C13372
:106C9000FF33D2059B009950437DC133FF339B00E6
:106CA0009950CC220169094B5204CA50052201694E
:106CB000243BCA50827D01690833CA500269417D74
:106CC000034BD1507047C0460C060000240500005D
:106CD0000C050000A022002310B50469D200A350C7
:106CE0000A4CA1420FD90A4C8C425B4109495B42D4
:106CF0000B40CD21C9045B18046907496350052185
:106D00000369995010BDCC235B04F5E7A086010010
:106D100090D00300000098FD24050000F7B50400A2
:106D200000200D000193824265D01600402A00D950
:106D3000402627001C37380000F0F6F8B1232269FE
:106D4000DB00D55080220123216992008B50A27E66
:106D5000002A03D122691362226913600025731E81
:106D6000AB4207D1019B002B04D080220221236972
:106D700092009950012223691A622369FC33DA6870
:106D8000002A02D19A6A002AF9D09A6A002A0BD105
:106D9000DA60A3232269DB00D1583800C9B201357B
:106DA00000F0B7F8B542DAD3019B2269002B0FD16E
:106DB0001300FC339B6A002B0AD10133A376D36105
:106DC0002369FC33DA6C002AFCD00022DA640AE082
:106DD00000230121A37651611A002369FC339968CD
:106DE0000029FCD09A602369FC339A6A002A01D0FA
:106DF00000229A62E8B2FEBD10B50123FFF78EFFB4
:106E000010BD0300AC3310B504001970643000F0FD
:106E10008BF80123637610BD0023020070B5AC32FD
:106E200043760D001178B12204000069D200815030
:106E30008022216992008B502269013313622269FA
:106E4000936026006436300000F080F8002812D0ED
:106E5000300000F06DF81E4B2269D0502369FC33DE
:106E60001A6A002A02D19A6A002AF9D09A6A002A7C
:106E700001D11A62E5E723690122002D0DD1190025
:106E8000FC31896A002908D1DA612369FC33DA6CA4
:106E9000002AFCD00022DA6407E05A612369FC333F
:106EA0009A68002AFCD000229A6000202369FC33F3
:106EB0009A6A82420BD098622169064A8B588B509D
:106EC0001800022B03D0181F431E9841033070BDD9
:106ED0001C050000C404000010B50121FFF79CFF51
:106EE00010BD000010B51323142202490248FFF719
:106EF000A3FE10BD00400040F81A002010B540224B
:106F00000021040004F056FA002320002364636487
:106F100010BD10B53F24026C531C2340446C9C42AE
:106F200001D08154036410BD00230364436470479F
:106F3000436C026C934206D03F21C25C01330B408C
:106F400043641000704701204042FBE7036C406C33
:106F5000181A00D540307047436C026C934201D040
:106F6000C05C704701204042FBE73F22036C406C4D
:106F700001331340181A43425841C0B27047000011
:106F800003210A4802680A430260094802680A436A
:106F900002600849084A094B9B1A03DD043BC858A4
:106FA000D050FBDC00F012F8F9F7AEF824050040F1
:106FB000540500409CE20000000000206402002014
:106FC000FEE7FEE7FEE7FEE7FEE7FEE72D4B10B526
:106FD0001A68D2B2012A0FD12B4A126812070BD1BC
:106FE0002A4AE0241168F0220800104021422DD1E5
:106FF0002749096811422CD01A68D2B2012A12D14D
:107000002149096809070ED1F0202049096801408B
:10701000402908D11E490968014204D18020C121BC
:10702000C005C90042501B68DBB2012B0DD1164BC5
:107030001B681B0709D1154B1A68F0231A40A02AB8
:107040000FD1134A12681A420ED010BD3028CFD08B
:10705000D2E7104A104911608021104A09021160DC
:10706000CAE7D02AF1D1ECE70D4B1A68012A04D007
:107070000C4A1A601A68012AFCD1C0220A4B1A6015
:10708000E3E7C046E00F00F0E40F00F0E80F00F087
:10709000EC0F00F004050040DFFF07C0186C004053
:1070A00000EC06407593000014EC06400120704788
:1070B00010B503681322DB69984710BD70470000C4
:1070C000054B0269D1500369FC331A6A002AFCD0CF
:1070D000002201201A6270471C050000030010B551
:1070E0005C331A781F231A401E3B19009140114A45
:1070F000D167C222042104699200A1500269536041
:107100000269D360A02300220169DB00CA50012379
:107110000169094A5B428B500169084A8B50016939
:107120000C3A8B50016908328B501430FFF7FCFE8B
:1071300010BDC04604E100E00C050000140500008D
:1071400010B51430FFF702FF10BD10B51430FFF773
:1071500003FF10BD10B51430FFF7EAFE10BD0000AC
:10716000030070B55E331A780469724BE250030075
:107170005D331A780469704BE250030061331C7868
:1071800002696E4B012C00D09EE005005F352E7821
:10719000A225ED005651020060321578A122066941
:1071A000D200B5500269D4509623DB00994200D832
:1071B0008CE096231B01994200D88AE096235B015C
:1071C000994200D888E096239B01994200D885E037
:1071D000E1239B01994200D882E09623DB0199428A
:1071E00000D880E0E123DB01994200D87DE09623BE
:1071F0001B02994200D87AE0E1231B02994200D891
:1072000077E096235B02994200D874E0E1235B02A9
:10721000994200D871E0E1239B02994200D86EE0C8
:10722000474B994200D86CE0E123DB02994200D839
:107230006AE0E122002312038A425B41414A5B4239
:107240001340802252059B1801693F4A8B50A023AE
:1072500004220169DB00CA5000210369FC33D960B4
:107260000369FC331962012301690B6001698B60BA
:10727000C1210469890062501F215C3002780A40F4
:1072800093406231314AFF31535000214156002969
:107290003CDA0F230B40083B2D4C9B089B001B192D
:1072A00003242140A140FC348C40DD69A5432C001F
:1072B000C0258D4029002143D9611F230178194041
:1072C0001E3B8B40136070BD00246CE79E23DB02E5
:1072D000BAE79D231B03B7E71E4BB5E71E4BB3E789
:1072E000EC239B03B0E71D4BAEE71D4BACE71D4BFA
:1072F000AAE71D4BA8E71D4BA6E71D4BA4E71D4BB6
:10730000A2E78023DB049FE71B4B9DE78C080F4B14
:10731000A400E41803230B40FF21C025DB009940A3
:10732000AD0066598E433100C0269E4033000B43AA
:107330006351C2E70C050000140500006C05000055
:1073400090D0030000D0BEFE2405000000E100E064
:1073500000ED00E000B013000050270000A04E0038
:1073600000F0750000509D0000F0EB0000903A0125
:1073700000E0D70100B0AF0300705F07F7B50093DE
:1073800008AB1B7800250193FA2304009B0083605F
:107390000E4B45600833036014300F001600FFF7F2
:1073A000ADFD23005C3327611E70009B084A9B00E3
:1073B000995823005D331970019B20009B009A5857
:1073C00023005E33DD701A70FEBDC046D0DD0000C4
:1073D0004CDD0000036910B51A00FC32D2680400CD
:1073E000002A0AD0A322D20099581430C9B2FFF75C
:1073F00090FD00222369FC33DA6010BD10B502480D
:10740000FFF7E8FF10BDC046B01B0020162307B5EC
:10741000022200930249013B0248FFF7AFFF07BD7C
:1074200000200040B01B002010B5002801D004F05F
:107430007DFA10BD7047000010B500F011F8FFF79D
:10744000F9FF012000F000FAFFF7F2FAFFF702FB64
:10745000024B002BFAD000E000BFF7E7000000006D
:10746000C420114B80001A5810491140C02212024A
:107470000A431A50C0218022490092025A501A60D1
:107480008023A3220021DB05D20099500122F9308C
:107490009A60074BFF301950C1200231800019500B
:1074A000403019501A60704700E100E0FF00FFFF14
:1074B00000100140014B18607047C0467800002062
:1074C000F7B5002320285AD8384B8000C258042A28
:1074D0005BD007D8022A54D055D80423012A09D0FA
:1074E00000234CE0062A54D051D31A2A53D0022349
:1074F0001B2AF5D12E4A116808294ED909294FD0E7
:107500000A240226A02001252A4AC00015502A4834
:107510002A4D07681C20BF000740294801970068D2
:107520005759009027481B0207401F43C02300986B
:107530009B020340FF2057515759000207401F4349
:10754000019B1F43009B58016023184007433E43A3
:10755000565101251C4B156058680028FCD00020AE
:107560005860A1230125DB00D3585560A025ED000C
:1075700050511BB2A14202D015D2611ACB40180063
:10758000FEBD0823B6E71023B4E72023B2E740236B
:10759000B0E78023AEE70123ACE708240026B1E77B
:1075A0000C000126AEE7091B8B40E8E74CDD00002C
:1075B000740000200070004030000020040500002E
:1075C00034000020FF00FFFFFC700040F0B52028D1
:1075D0005BD8364B8000C258354B1E68002E30D128
:1075E000C227344BBF00D859334C03250440C02078
:1075F00000022043D851C02480206400800018512C
:107600002E4F18602E4B803CD859FF3CA043D851D8
:107610000437D859A8432043D8510837D8590C35D6
:10762000A8438446072065462843D851A820C000B7
:107630001E50C1208026800076021E501C601C4B0C
:107640001C60142500202B001E4C2E00464336598A
:10765000771C1BD14343E250A0230325C132FF32E4
:107660009200DB05D550184B1A68082A14D1142350
:107670004343E3189A6812485132FF32920059602E
:107680001150DA68C1239B00C250F0BD9642E1D090
:1076900001300328D9D1F8E7082A02D9083AD140A5
:1076A000E5E708239A1A9140E1E7C0464CDD000067
:1076B000141C002000E100E0FF00FFFF04050000B3
:1076C0000090004038000020780000202149F0B5EB
:1076D0004A6C2148002A14D0A025A12600230124A9
:1076E000ED05F600C258571C06D0C7187F68002F5A
:1076F00002D027009740AF5114333C2BF2D1002326
:107700004B64A0230121DB0500260F009C461423B7
:107710004B43C3181A1F1268104C0E4D92001419D7
:107720005219526C002A10D01A00143A1268551CD3
:1077300009D0103B1B68FF2B05D03B0093406546EA
:107740001A00074BEA50FC34666401310429DED18B
:10775000F0BDC046FC900040380000200090004082
:107760000C05000000B5202810D80C4A8000835872
:1077700003290BD8A0220800C133FF33D2059B0098
:1077800001F036FC020905070021D15000BD0C2193
:10779000FBE70421F9E70321F7E7C0464CDD0000D1
:1077A00020280AD8074B8000C25801239340A0220A
:1077B000D205002902D1044953507047A121C900C4
:1077C000FAE7C0464CDD00000C0500000300002075
:1077D000202B0AD8A021A222C905D2008858034A2A
:1077E0009B009B58D8400123184070474CDD000097
:1077F000F7B506000D000C008B180193019B671B69
:107800009C4207D0336821781B68300098470134C8
:107810000028F3D13800FEBD0849094A094B10B5CC
:107820001B688858FA22190A1B0618439200002385
:1078300001F0B4FD4904C00B084310BD0010014025
:1078400004050000181C002070B5041E09D0FFF7C5
:10785000E3FF050000F014F8FFF7DEFF401BA04235
:10786000F8D370BD0022044B9A60044A13680133B8
:10787000DBB213607047C046FC100140181C0020AA
:1078800070470000F0B5C64600B5CB0F9846404A99
:107890004B005B0D9A1882B00D000400132A2FDCF8
:1078A000002A49DB3B4F17413E000E40064323D0E0
:1078B0007F08390029400C430AD03749BD438C4624
:1078C00063445C425C418023DB021341E4071D43B7
:1078D0004146CE0031492B008E192200346875686C
:1078E0002000290001F000FF00900191009801990B
:1078F00022002B0003F090F802B004BC9046F0BDCB
:10790000332A08DD8023DB009A42F5D102000B0008
:1079100001F0EAFEF0E7224A944601226344524213
:10792000DA400242E8D052080242D1D09443802289
:10793000D2051A411443CBE74B005B080343DBD06D
:107940000B031B0B1C436342234380244D0C240375
:107950001B0B23406D042B4319004346DA000F4BE9
:107960009B181C685D6802000B002000290001F0D4
:10797000BBFE009001910098019922002B0003F0BA
:107980004BF842464B005B08D60733431900B3E778
:1079900001FCFFFFFFFF0F00EEFBFFFF00DE00001A
:1079A000EDFBFFFFF8B5274A4B005B0D9A180C0062
:1079B0000700132A10DC002A36DB234B13410B424D
:1079C0003AD0802424031441002064189C4306000C
:1079D000250030002900F8BD332A0EDD8023060083
:1079E000DB000D009A42F4D102000B0038002100A8
:1079F00001F07AFE06000D00EBE7144D0600AC46E0
:107A0000012563446D42DD40AC4663460D000342F0
:107A1000DFD033239A1A323B93401818874200D99B
:107A20004C1C63469843D2E7C90FCC070020531C77
:107A3000CDD1074B1C43CAE706000D000028C0D17A
:107A4000C7E7C04601FCFFFFFFFF0F00EDFBFFFF94
:107A50000000F03F30B5214A4B0087B05B089342ED
:107A60001EDD1F4A934205DD02000B0002F0D4FF29
:107A700007B030BD02AA00F095F803231840049A1D
:107A8000059B012813D002281DD0002814D002988D
:107A9000039900F06FFB80231B069C466144E7E7D7
:107AA000002300220093002301F0DEF8E0E70298B3
:107AB000039900F05FFBDBE701240298039900942F
:107AC00001F0D2F8D4E7012402980399009401F060
:107AD000CBF880231B069C466144C9E7FB21E93FA4
:107AE000FFFFEF7FF0B54746CE4680B58DB004006E
:107AF0000D0000F067FA294B06001B780F005BB2FF
:107B00009846013310D022002B002000290003F0FA
:107B1000CBFA8146002807D100220023200029004B
:107B200001F014FC002806D1300039000DB00CBC67
:107B300090469946F0BD01230293194B0694079590
:107B400003934B460A93434604940595002B15D0A6
:107B5000002300221900100002F0E2F843460890CA
:107B60000991022B0ED103F0B9FB212303600A9B7C
:107B70000193002B0CD1089E099FD5E70023002418
:107B80000893099402A801F0C1F90028EFD1EAE7AF
:107B900003F0A4FB0A9B01930360ECE77C00002048
:107BA00010DE0000F0B54E464546DE465746E0B5CD
:107BB000E14B4C008FB09046894664089C4200DC43
:107BC00087E0DE4B9C4222DCDD4A002900DC92E0AB
:107BD000DC4B02F021FFDB4B06000F009C4200D182
:107BE0007EE1D94AD94B02F017FF02000B00414653
:107BF00030000A604B60390002F00EFFD34BD24ACE
:107C000002F00AFF434601259860D9606BE0D04B33
:107C10009C4200DC8FE0CF4B9C4200DD55E1CE4A18
:107C2000231592469A4451460905631A19001D000E
:107C3000040003F055FA03F089FA02000B0020005B
:107C400029000892099302F0E7FE0022C34B02F0DC
:107C500071FC0F00060003F043FA03F077FA04000A
:107C60000D0002000B00300039000A940B9502F061
:107C7000D3FE0022B94B02F05DFC002200230C90E1
:107C80000D9101F05DFB002800D192E1002300225C
:107C90002000290001F054FB434243410133B04A24
:107CA00041460192022208A80092524600F07CFB55
:107CB0004B460500002B16DA8022434612069446F6
:107CC00042465B68454263445360D3686344D36073
:107CD00009E00B00020041460A604B6000220023CD
:107CE00000258A60CB6028000FB03CBC90469946C6
:107CF000A246AB46F0BD934B01F0F6FC914B06005B
:107D00000F009C4200D13DE18F4A904B01F0ECFC0A
:107D100002000B00414630000A604B60390002F05F
:107D20007BFE894A894B01F0DFFC012543466D4209
:107D30009860D960D7E701F049F88A4A8A4B060073
:107D40000F0002F0F7FB0022884B01F0CDFC03F09E
:107D5000C7F9050003F0FAF9794A7A4B04900591C6
:107D600002F0E8FB02000B003000390002F054FE84
:107D7000754A06000F0004980599744B02F0DAFB6F
:107D8000029003911F2D00DCC7E0029A039B300094
:107D9000390002F041FE83468A4653465B002415B3
:107DA0005B0DE31A102B6CDD04980599D322674B09
:107DB000520502F0BFFB02000B00300039000292B6
:107DC000039302F029FE0A000100130006910792B6
:107DD00002003900300002F01FFE029A039B02F0FD
:107DE0001BFE06000F0004980599614A614B02F0E2
:107DF000A1FB32003B0002F00FFE069E079F0B0026
:107E00000200390030000292039302F005FE4B009D
:107E10005B0D83468A46E41A312C32DD04980599BD
:107E2000B822544B920502F085FB03000C000200BF
:107E3000029303940B000698079902F0EDFD0200EF
:107E40000B0006000F000698079902F0E5FD029A64
:107E5000039B02F0E1FD484A0290039104980599C2
:107E6000464B02F067FB029A039B02F0D5FD02002D
:107E70000B00300039000292039302F0CDFD8346DF
:107E80008A465A465346414630000A604B603900E4
:107E900002F0C2FD029A039B02F0BEFD44460B00B5
:107EA0000200A260E3604B46002B00DB1BE75B4651
:107EB000236080231B065344636080231B069C467B
:107EC0006144A060E1606D420DE70B00020002F02A
:107ED000A3FD434600259860D9601860596002E709
:107EE000D3221A4B520502F097FD214A214B0D0077
:107EF000040002F091FD02000B00414620000A60E0
:107F00004B60290002F088FD1A4B194A02F084FDEB
:107F1000434601259860D960E5E602000B00300079
:107F2000390002F079FD6B1E154A9B009B58834671
:107F30008A46A342A5D130E7FB21E93F7BD9024025
:107F400000004054FB21F93F3163621A61B4D03D17
:107F5000FB213941FFFFEF7FEAFBFFFF000070418B
:107F600098DE000083C8C96D305FE43F0000E03F49
:107F70007370032E8A19A33BC14920259A837B394C
:107F800018DE0000D3220C4B520501F0ADFB0B4A6A
:107F90000B4B04000D0001F0A7FB02000B00414653
:107FA00020000A604B60290002F036FD034A044BB2
:107FB000B9E6032373E6C04661B4D03D7370032E67
:107FC0008A19A33BF8B54746CE46674B80B50A00F1
:107FD0000F00190005003940994200D19BE00400D0
:107FE0000100002F69DD3F1500D1B4E05F4B1203A3
:107FF0009C468023120B5B0313435B00CA0F67444C
:108000009B184A00F80703D5D20F5B009B188A0023
:1080100079108C46002180201624894680030D1893
:108020009D4202DC29185B1B8144D50F5B00013C9B
:108030005B1952004008002CF1D1002080468020BE
:1080400020250027000609E08B425CD0D40F5B009E
:10805000013DE31852004008002D16D0C4198B4290
:10806000F2DD27180E00002C49DB5B1AA242894181
:1080700049425B1A121BD40F5B00013D8044310062
:10808000E31852004008002DE8D113434ED1434677
:108090005B0837494A468846494652104244C90758
:1080A00002D5802109060B4361460F05BD18180053
:1080B00029000CBC90469946F8BD7B005B08034341
:1080C0003900002BF5D0002F3CD1E30A153A6405A6
:1080D000002BFAD08020400303423FD1002700E06C
:1080E0000F005B00791C0342FAD0250020208D4050
:1080F000401A2900D71B2200C2401A4376E7FE43EC
:10810000F60F8E19B1E79442A0D82718002CF6DBA1
:108110001E000023AEE702003B002800390002F0F9
:1081200009FA2A003B0001F0DFFAC2E743460133B7
:1081300003D0434601335B08ABE701239846002395
:10814000C144A6E73B00020002F066FC02000B00FF
:1081500001F0E6FDADE713000022BBE70127210097
:1081600020207F42C6E7C0460000F07F01FCFFFFF1
:108170000000E03FF0B54746CE4680B587B000929C
:108180000193754B4F00814688467F089F4263DC10
:1081900002F0A6FF002800D1D4E04A4643464846F4
:1081A000414602F0C7F904000D006C4A6C4B02F026
:1081B000C1F96C4A6C4B01F097FA22002B0002F0D7
:1081C000B9F96A4A6A4B02F027FC22002B0002F040
:1081D000B1F9684A684B01F087FA22002B0002F0DF
:1081E000A9F9664A664B02F017FC22002B0002F048
:1081F000A1F9644A644B01F077FA22002B0002F0E7
:1082000099F9029003910022604B2000290002F0AE
:1082100091F9029A039B06000F002000290002F04A
:1082200089F9009A019B04000D004846414602F07E
:1082300081F902000B002000290002F0EDFB020092
:108240000B003000390002F0E7FB02000B000020B9
:108250004F4902F0E1FB70E002000B0002F06AF906
:1082600004000D003D4A3E4B02F064F93D4A3E4B8E
:1082700001F03AFA22002B0002F05CF93B4A3C4B39
:1082800002F0CAFB22002B0002F054F9394A3A4BA3
:1082900001F02AFA22002B0002F04CF9374A384B41
:1082A00002F0BAFB22002B0002F044F9354A364BAB
:1082B00001F01AFA2B00220002F03CF9354B029033
:1082C00003919F429FDD344B00229F423DDC3349A6
:1082D00000207B182E4916001F0002F09DFB049021
:1082E00005910022294B2000290002F023F93200D9
:1082F0003B0002F091FB029A039B06000F00200056
:10830000290002F017F9009A019B04000D0048466D
:10831000414602F00FF902000B002000290002F094
:108320007BFB02000B003000390002F075FB0200FD
:108330000B000498059902F06FFB07B00CBC904647
:108340009946F0BD00201249F7E7154B002604922C
:108350000593144FC5E7C046FFFF3F3ED43888BEA3
:10836000E9FAA8BDC4B1B4BD9EEE213EAD529C80D9
:108370004F7E923E9015CB19A001FA3E7751C1165F
:108380006CC1563F4C5555555555A53F0000E03F33
:108390000000F03F3233D33F0000E93F0000E0FF30
:1083A0000000E73F0000D23FF0B5DE464E464546AE
:1083B0005746E0B5DC4CA5440D9114001900A49A71
:1083C0000993DA4B9200D6584D1E03901821E01EF7
:1083D0000696029500F0AAFEC3430100DB17194080
:1083E0004B1C9A009B1ADB001B190B9105934C1B2D
:1083F000771918D4A59BA5009C463F1922AE654469
:10840000013707E0286802F0A1FE013403C60435F5
:10841000BC4208D0002CF5DA00200021013403C64C
:108420000435BC42F6D1069B002B01DA00F0FDFBBF
:10843000069B03990133DB009A46099BDA009446B8
:1084400000920022914672AA0492B94A614493466E
:1084500088469AAB63449B44029B002B00DABCE144
:108460005D4600260027039C4D442A686B6803CCB8
:1084700002F060F802000B003000390001F034F91E
:10848000083D06000F004445EFD1049B4B441E609D
:108490005F6008239C46E144D145DDD10EA804214C
:1084A0008446494261448C46069A93009C44614646
:1084B00084460A910399083B63448C460C93009BC5
:1084C000009263449B46009A0498D10003008C46B6
:1084D000634408911E685F68002A33DD9549804631
:1084E0008C466244D300984470AB9A460EAB9946D2
:1084F0000022914B3000390002F01CF802F0F0FD30
:1085000002F024FE00228D4B04000D0002F012F850
:1085100002000B003000390002F07EFA02F0E0FDAC
:108520004B4601C39946434620001A685B68290000
:1085300001F0DAF808235B429C46E04406000F0095
:10854000D045D5D1059B30001A003900984600F07F
:10855000DFFCFF2300229B0504000D0001F0EAFF71
:1085600000F038FC0022764B01F0E4FF02000B0023
:108570002000290002F050FA0D00040002F0B0FDC6
:10858000814602F0E3FD02000B002000290002F00A
:1085900043FA060040460F00002800DCEEE0009B96
:1085A00018215A1E92000EAB9B58091A1D000D414E
:1085B000A9448D405D1B0EAB9D5017231B1A1D4116
:1085C000002D2DDD01239C46009BE144002B00DCA7
:1085D0001CE20E9C0123002C00D0B5E0009A012A79
:1085E00009D099000EAA54580133002C00D0ACE0F9
:1085F000009A9A42F5D1059B002B0EDD012B00D18C
:10860000A8E1022B09D1009B0EA95A1E92000EABC5
:108610009B5807939B029B0A8B50022D00D1C1E00F
:10862000002300223000390000F08AFE009B002861
:1086300000D194E2069A591E8A4210DC414A0A98F7
:1086400094460EAA6344944600229B0063441C682F
:10865000043B22438342FAD1002A00D0C0E0069BAB
:108660000EAA013B9B00D358002B00D0B3E001229F
:108670000C9B043B596801320029FAD0009B9C46B0
:108680006244110007921A0001338B4246DC0B98BA
:1086900063468046A59C4344A046099C9B00A14696
:1086A0004A449844D30022AA9146049A9944944695
:1086B000089BA59A63448446614494469A468B007D
:1086C000634400934346586802F040FD4B461860EF
:1086D0005960029B002B24DB4D46039C002600279B
:1086E00001E0286869680CCC01F024FF02000B004F
:1086F0003000390000F0F8FF083D06000F005C452F
:10870000EFD153469E60DF6004239C460433E0446F
:108710009C46009BE144E2449845D3D1079B0093DB
:10872000D1E600260027ECE794FDFFFFE0DF000024
:1087300018FEFFFFFFFFFF1F0000703E00007041AA
:1087400000002040FFFFFF3F002180225204141B45
:108750000EAA5450009999420EDD0EA884469B0043
:108760000EAA8900D25861446344CF4800E01A68D9
:10877000821A04C38B42FAD101243CE7059B002BEB
:1087800006D1009B0EAA013B9B00D558ED1517E7BB
:108790000022C64B300000F0F7FD002800D024E195
:1087A00000253DE732003B000020C14902F034F9CA
:1087B00006000F00002C00D132E7059A0020BC49CA
:1087C00000F0A6FB02000B003000390002F024F993
:1087D00006000F0024E7012250E70026002754E698
:1087E0004B46059A079388468B000EA9CB58183A3A
:1087F00008950592002B0DD18C464146AD4B434464
:108800009B006344043B58680139183A0028F9D0AA
:1088100088460592059A0020A54900F079FB434659
:1088200004000D00002B00DA05E29E000EAB9C4612
:108830004346DB0066449C46059370AB9946049F13
:1088400067440097306802F081FC22002B0001F0A1
:1088500071FE002238607960974B2000290001F0FA
:1088600069FE083F04000D00043EB945EAD14AAB59
:1088700003939B4600239A46069B424699464346ED
:108880000132029204934B46002B00DAAAE08020CA
:108890008A4B009D9846C005894900260027002480
:1088A00008E008239C460835E044544511DC434663
:1088B000186859682A686B6801F03CFE02000B00DA
:1088C0003000390000F010FF013406000F00A14510
:1088D000E7DA5B46C0C39B4601239C46009BE2440B
:1088E000083B0093029B9A45CDD1049B9846A49BDC
:1088F000022B00DD8EE0002B37DC1FD1059B00270B
:108900001D00039B00249C461E006544083E2A6807
:108910006B683800210000F0E7FE083D07000C00FE
:10892000AE42F4D1089B002B03D080231B069C464B
:1089300064443A0023000D990A604B600720079BAE
:1089400018409B239B009D443CBC90469946A24600
:10895000AB46F0BD009B0EA95A1E92000EAB9B5871
:1089600007935B025B0A8B5057E64346002B00DA05
:1089700070E100200021DB004AAAD61848AF326817
:108980007368083E00F0B0FEB742F8D1089B002B98
:1089900000D025E10B0002004A984B990D9C226003
:1089A000636002F039F8434607000C00002B13DD2A
:1089B00001254CAEB14638002E0021004C46013650
:1089C0000CCC00F091FEA146B045F7DA089B0700F9
:1089D0000C00002B00D015E13A0023000D998A60AD
:1089E000CB60ABE70026002773E701239C46009B82
:1089F000E1440225002B00DDEBE532003B000020C6
:108A00002B4902F009F806000F0009E60024F2E500
:108A10004AAB0393A49B032B00D08FE74346002B64
:108A200000DC14E1039ADB009B46130091465B4493
:108A30001E685F68234B43440293DB00994448ABB4
:108A40009A464B465C681B681800210032003B00C8
:108A50000090019100F048FE04000D0002000B00A0
:108A60000098019901F0D8FF3B00320000F03CFE75
:108A70004B469860D9601C605D6008235B429C4651
:108A8000E14426002F00CA45DBD14346012B00DC20
:108A9000E3E0039A13005B441E685F68029BDB00FF
:108AA00099464A44904610E0FFFFFF000000E03F77
:108AB0000000F03FFFFFFF3F0000703EA0DF00001E
:108AC000FB21F93FFFFFFF1F984643465C681B6888
:108AD0001800210032003B000090019100F004FEDC
:108AE00004000D0002000B000098019901F094FFB2
:108AF00032003B0000F0F8FD4346039A9860D960CD
:108B00001C605D60083B26002F009A42DCD14D4678
:108B10009446002600244746083565442A686B6859
:108B20003000210000F0E0FD083D06000C00AF42DF
:108B3000F4D1039B4A9F5D689968D868089B002B15
:108B400065D08022120694460D9B654460446444BF
:108B50001F605D609960D8601E615C61EEE69A46B8
:108B60004B460793059B30005A423900089500F0A8
:108B7000CFF900223A4B06000F0000F005FC002858
:108B800024D0384B00223000390001F0D3FC02F031
:108B9000A7FA52460400950002F0D8FA0022304BA2
:108BA00001F0C8FC02000B003000390001F034FF76
:108BB00002F096FA0EAA50510122059B5244183336
:108BC0009046059393000EAAD45023E653463000F6
:108BD00039009C0002F084FA0EAB1851D04619E619
:108BE00080230D9A1B06CB18106053600B00020007
:108BF0004A984B9901F010FF434607000C00002BE8
:108C000000DDD5E680231B069C466444E4E62B0089
:108C10003A000D9D2A606B600A000300AA60EB60B9
:108C2000320023002A616B6188E6099BDB00009318
:108C300072AB049332E4A49B022B00DDE8E6002B28
:108C400000DD92E600D079E6002700246AE60026DF
:108C500000246EE70020002198E60026340068E733
:108C6000000070410000703EF0B5CE46474680B52A
:108C700087B000920193474A4B00814688465B08C3
:108C8000934207DC4146484602F02AFA4146031E59
:108C9000484666D04A4643464846414601F04AFCAB
:108CA00004000D0002000B004846414601F042FC62
:108CB000394A3A4B06000F002000290001F03AFC27
:108CC000374A384B01F0A8FE22002B0001F032FC9D
:108CD000354A364B00F008FD22002B0001F02AFC3B
:108CE000334A344B01F098FE22002B0001F022FCA5
:108CF000314B324A00F0F8FC0E9B02900391002B9E
:108D000034D00098019900222D4B01F013FC029AF7
:108D1000039B049005913000390001F00BFC020028
:108D20000B000498059901F077FE22002B0001F05A
:108D300001FC009A019B01F06FFE224A04000D0025
:108D4000214B3000390001F0F5FB02000B00200040
:108D5000290000F0C9FC02000B004846414601F022
:108D60005BFE07B00CBC90469946F0BD02000B00BC
:108D70002000290001F0DEFB124A134B01F04CFEEB
:108D800032003B0001F0D6FB4A46434600F0ACFC03
:108D9000E7E7C046FFFF3F3E7CD5CF5A3AD9E53DD5
:108DA000EB9C2B8AE6E55A3E7DFEB157E31DC73E9C
:108DB000D561C119A0012A3F1111813FA6F81011F8
:108DC0000000E03F495555555555C53F49004B08F2
:108DD00019007047474AF0B54F4691464B005B0D6E
:108DE00099444646D6464A46C0B505000C000E00DA
:108DF00088460700132A27DC002A4BDB3E4B134131
:108E00009A460B0052461340034318D03B4A3C4B52
:108E10002800210000F068FC0022002300F0AAFADC
:108E2000002847D0002C04DA80234A465B03134114
:108E300098444646534600279E43380031001CBCE8
:108E400090469946A246F0BD332A08DD8023DB0018
:108E50009945F4D102000B0000F046FCEFE7294AE7
:108E60009446012263445242DA4092460242E6D0DE
:108E7000224A234B2800210000F036FC0022002368
:108E800000F078FA002815D0002C1EDB5346464629
:108E90009F430FE0194A1A4B2800210000F024FCE0
:108EA0000022002300F066FA002803D0002C04DB27
:108EB0000027002638003100C1E76400640825431C
:108EC0000027002DF6D0104EF4E74B46142B0BD0A4
:108ED0003422D21A012393405D19BD4208D20123E6
:108EE0009C462F00E044D1E7133B9C46E044CDE78D
:108EF0002F00CBE701FCFFFFFFFF0F009C750088F0
:108F00003CE4377EEDFBFFFF0000F0BF0020704720
:108F10004B0070B55B0D14000A00002B1AD14B00FA
:108F20005B08034315D0234B002201F003FB224BC7
:108F30009C422DDB0A004B005B0D363B1F4DE318B6
:108F4000AB422ADC002B0DDD1D4C1B0522401A43D1
:108F5000110070BD1B4DAB42F0D102000B0000F0C0
:108F6000C3FBF6E71D00353519DA174B02009C42AA
:108F700009DD0B001548164900F032F8134A144B6E
:108F800001F0D8FAE5E70B001248134900F028F881
:108F9000104A114B01F0CEFADBE70200E9E7084C7A
:108FA000363322401B051343190000220B4B01F0FE
:108FB000C1FACEE700005043B03CFFFFFE070000BF
:108FC000FFFF0F80FF07000050C300009C75008862
:108FD0003CE4377E59F3F8C21F6EA5010000903CB7
:108FE00030B54A00DB0FDB0752081A43110030BDD1
:108FF00002B4714649084900095C49008E4402BC2C
:109000007047C04603B47146490840004900095AF8
:1090100049008E4403BC7047002243088B4274D33E
:1090200003098B425FD3030A8B4244D3030B8B4269
:1090300028D3030C8B420DD3FF22090212BA030C72
:109040008B4202D31212090265D0030B8B4219D353
:1090500000E0090AC30B8B4201D3CB03C01A524173
:10906000830B8B4201D38B03C01A5241430B8B42BB
:1090700001D34B03C01A5241030B8B4201D30B03A4
:10908000C01A5241C30A8B4201D3CB02C01A5241CB
:10909000830A8B4201D38B02C01A5241430A8B428E
:1090A00001D34B02C01A5241030A8B4201D30B0277
:1090B000C01A5241CDD2C3098B4201D3CB01C01A91
:1090C000524183098B4201D38B01C01A524143099B
:1090D0008B4201D34B01C01A524103098B4201D389
:1090E0000B01C01A5241C3088B4201D3CB00C01AF6
:1090F000524183088B4201D38B00C01A524143086E
:109100008B4201D34B00C01A5241411A00D2014692
:10911000524110467047FFE701B5002000F0F0F81B
:1091200002BDC0460029F7D076E7704703460B43DF
:109130007FD4002243088B4274D303098B425FD350
:10914000030A8B4244D3030B8B4228D3030C8B427C
:109150000DD3FF22090212BA030C8B4202D3121262
:10916000090265D0030B8B4219D300E0090AC30B37
:109170008B4201D3CB03C01A5241830B8B4201D3E4
:109180008B03C01A5241430B8B4201D34B03C01ACD
:109190005241030B8B4201D30B03C01A5241C30A45
:1091A0008B4201D3CB02C01A5241830A8B4201D3B6
:1091B0008B02C01A5241430A8B4201D34B02C01AA0
:1091C0005241030A8B4201D30B02C01A5241CDD245
:1091D000C3098B4201D3CB01C01A524183098B4290
:1091E00001D38B01C01A524143098B4201D34B0179
:1091F000C01A524103098B4201D30B01C01A5241DC
:10920000C3088B4201D3CB00C01A524183088B4262
:1092100001D38B00C01A524143088B4201D34B004B
:10922000C01A5241411A00D20146524110467047BD
:109230005DE0CA0F00D04942031000D340425340C2
:1092400000229C4603098B422DD3030A8B4212D382
:10925000FC22890112BA030A8B420CD389019211B4
:109260008B4208D3890192118B4204D389013AD0F1
:10927000921100E08909C3098B4201D3CB01C01AC6
:10928000524183098B4201D38B01C01A52414309D9
:109290008B4201D34B01C01A524103098B4201D3C7
:1092A0000B01C01A5241C3088B4201D3CB00C01A34
:1092B000524183088B4201D38B00C01A5241D9D24C
:1092C00043088B4201D34B00C01A5241411A00D2CD
:1092D0000146634652415B10104601D34042002BC9
:1092E00000D54942704763465B1000D3404201B548
:1092F000002000F005F802BD0029F8D016E77047FD
:109300007047C046D0400B1C1141203A03D49C4604
:109310001341184363465242934018437047C04676
:109320008446101C62468C46191C634600E0C04609
:109330001FB501F097F8002801D40021C8421FBDD5
:1093400010B500F0EFFF4042013010BD10B501F044
:1093500089F8002801DB002010BD012010BDC046A7
:1093600010B501F07FF8002801DD002010BD0120BC
:1093700010BDC04610B501F011F8002801DC002036
:1093800010BD012010BDC04610B501F007F800283F
:1093900001DA002010BD012010BDC046F0B5CE4658
:1093A000474615042D0C2E0080B50704140C3F0C05
:1093B0009946030C7E435D43674363437F19340C36
:1093C000E4199C46A54203D980235B029846C44415
:1093D0004B4643435143250C36046544360C240464
:1093E000A4195B19591820000CBC90469946F0BD91
:1093F000F0B54E4657464546DE46E0B543025B0AA9
:10940000450083B00F1C99462D0EC60F002D57D076
:10941000FF2D24D08020DB00C004184300238146A8
:109420009A469B467F3D7C027A00FB0F640A120E2F
:10943000984623D0FF2A4BD0E30080240020E40488
:109440007F3A1C43AD186B1C474601935346774047
:109450003A000F2B48D87D499B00CB589F46002BE4
:1094600000D085E008339A46063B9B467C027A0092
:10947000FB0FFF25640A120E9846DBD1002C00D0AA
:1094800090E0524601231A4392460120DBE74C4606
:1094900058461700022824D0032800D1CFE000222C
:1094A000002301284DD15802D205400AFF0710437E
:1094B000384303B03CBC90469946A246AB46F0BD4B
:1094C000002B5BD104239A46033B00259B46AAE769
:1094D000FF35002C60D1524602231A4392460220E7
:1094E000B1E7FF220023DEE74B461B0C9C464B46B0
:1094F0002604360C180461463300220C6446000C26
:1095000043434E435043544380191A0C1218964259
:1095100003D9802149028C4664441B041B0C1004AF
:10952000C01883015E1EB341800E1843130C1B1933
:109530009B0103431C00230179D5012362081C40D1
:109540001443019A7F32002A4DDD630704D00F23B4
:109550002340042B00D00434230103D53C4B019A53
:109560001C408032FE2ABCDCA3015B0AD2B29AE71F
:109570000C239A46093BFF259B4654E7180001F04F
:1095800071FE4A46431F76259A4000236D4291465C
:109590002D1A9A469B4646E7524603231A439246A3
:1095A000032050E7200001F05DFE431F2D1A9C4070
:1095B000763D002047E780230027DB03FF2272E788
:1095C000424666E74C463200584662E780234A46E8
:1095D000DB031A4222D01C4220D123435B025B0AE8
:1095E0004746FF225FE701239A1A1B2A21DC23004A
:1095F0000199D3409E318C401A0023005C1EA34188
:1096000013435A0704D00F221A40042A00D004330F
:109610005A0111D49B015B0A002244E780234A4689
:10962000DB0313435B025B0A3700FF223BE7019534
:1096300087E70022002336E70122002333E7802357
:10964000DB0323435B025B0AFF222CE7F0DF000011
:10965000FFFFFFF770B500283DD0C317C5185D4068
:10966000C40F280001F0FEFD9E22121A962A07DC84
:10967000D2B2082833DD083885406802400A23E06A
:10968000992A0BDD052329001B1AD94003001B333F
:109690009D402B005D1EAB4119430D00052801DDE7
:1096A000431F9D402B000F490B406E0709D00F262A
:1096B0003540042D05D004335D0102D59F220B40B7
:1096C000121A9B01580AD2B24002D205400AE4079E
:1096D0001043204370BD002400220020F4E76802FC
:1096E000400AF1E7FFFFFFFBF0B54F464646D6467E
:1096F0000C000903C0B5490A470F5E0039431F0338
:10970000DB0F9C4665007B0A570F1F436D0DE40F6E
:10971000760DA146C000B846D200AB1B64457BD095
:10972000002B5FDD002E00D0A4E03E00164300D1E8
:1097300012E15E1E002E00D09EE1871A4346B84219
:1097400080410125C91A4042091A0B0200D431E1B7
:1097500049024E0A002E00D16EE1300001F082FD78
:109760000300083B1F2B00DD61E120223900D21AE3
:109770009E40D1409F400E439D4200DD51E15D1B64
:109780006B1C1F2B00DD7CE12021C91A3D0030003D
:109790008F408840DD40791E8F41310007222843E9
:1097A000D940002507433A40002A09D00F233B4007
:1097B000042B05D03B1DBB42BF417F42C9191F008E
:1097C0000B0200D426E26A1CC64B55056D0D9A4269
:1097D00000D106E1C44AFF080A40530752023B4346
:1097E000120B8EE0002B00D0B8E06B1C5B055B0D0C
:1097F000012B00DC30E1871A4346B842B641CB1A50
:1098000076429E1B330200D54CE13B003343A1D18D
:1098100000220024002570E0002B00DCE5E0002E93
:1098200000D183E0AF4EB54260D080263604374386
:10983000B846382B00DC3EE1434613431F007A1E36
:1098400097413F1887428041404209180B0200D4DB
:10985000B0E0A44B01359D4200D1C3E0A24A7B0891
:109860000A4001210F401F435108D30707221F431D
:109870003A4099E79B4EB54238D0802636043743AC
:10988000B846382B00DDDCE01F2B00DC30E11E0089
:109890004746203EF740BC46202B04D04026F31A12
:1098A00046469E403243170063467A1E97411F4347
:1098B000CCE0002B00D104E24346134300D159E130
:1098C0004B07C00818438023C9081B03194208D05E
:1098D0004546ED081D4204D14346D00859070843C8
:1098E0002900420FC9007F4D1143C0004B07CA0831
:1098F0007C49C00803438D4268D012036D05120BEA
:109900006D0D002112031800130B0A0D12051A43E6
:10991000764B2D0513402B435B00E4075B08234384
:1099200019001CBC90469946A246F0BD3E00164365
:1099300012D05E1E002E00D000E1871887428041C1
:1099400041444042091801250B0233D5022585E721
:1099500064463300414610001D00C7E7002D00D0CB
:10996000DAE00C000443F3D05C1C00D19FE15D4CB5
:10997000A64200D12FE1DB43382B00DD66E11F2B2F
:1099800000DD83E120240500E41A0F00DD40D9400A
:10999000A0404346A7405B1A441EA04198462F436F
:1099A0003843171ABA42924143465242991A6446C2
:1099B0003500CAE607223A40002A00D0F6E64B07F7
:1099C000CA084849FF083B438D4296D1190011430C
:1099D00000D19EE1802109030A431203120B414D7D
:1099E0008FE71500002200238BE7002B00D0C7E093
:1099F0006B1C5F057F0D012F00DCF1E0394DAB42A0
:109A000000D1B9E085180A008542894142444942A3
:109A100051180722CF076D082F4349083A401D000F
:109A2000C2E607223049ED1A31403A40BCE63E001A
:109A30002838864000279FE6380001F013FC2030CC
:109A40008EE6434613431F007A1E9741C71BB84258
:109A500080414042091A78E60E003B00064313435A
:109A6000002D61D1002E00D0F4E0002B00D11BE1CD
:109A700064463900100039E71A4FBB427AD03300F0
:109A8000FFE630001F3DE840202B03D04021CB1AD9
:109A90009E4037437B1E9F41072207433A400021E7
:109AA000002589E7171A4346BA42B641591A764249
:109AB0008E1B64464EE61F2B00DDADE02026474698
:109AC000F61AB740B9461700B246DF404E463E434D
:109AD00037005646B240561EB24117434246DA405E
:109AE0008918AEE6FF070000FFFF7FFFFFFF0F8032
:109AF00020264746F61AB740B9461700B246DF405F
:109B00004E463E4337005646B240561EB2411743BA
:109B10004246DA40891A99E77F4CA6425BD08024FE
:109B200024045B42214327E7002E0CD1002B00D1F7
:109B3000CBE0644639001000774DD7E6764FBB4244
:109B400018D0330075E6002B14D04B07C00818431B
:109B50008023C9081B03194207D0FC081C4204D10A
:109B60007907D0080843E14621004C46420FC9005E
:109B70001143C000684DB9E61D0000220023C0E675
:109B8000002D5BD10D00054300D1E2E65D1C00D144
:109B9000B0E0614DAE421FD0DB43382B71DC1F2B90
:109BA00000DD96E020250F00ED1AAF40B946070012
:109BB000AA46DF404D463D432F005546A840D940B8
:109BC000451EA84188440743BF189742924151421D
:109BD000414435003AE6644635004146100085E6CA
:109BE0000B000343002D00D063E6002BF5D0434665
:109BF000134300D17AE68718874280410722414407
:109C0000404209183A400B0200D4D5E6434B0135D7
:109C10001940C9E5380069E61E004746203EF74076
:109C2000BC46202B04D04026F31A46469E403243C1
:109C3000170063467A1E97411F4302E6364DAE4237
:109C4000CAD080252D045B422943A6E70843411E64
:109C50008841A6E6002B00D148E6871A4346B84261
:109C6000B641CB1A76429E1B33024BD5171A434698
:109C7000BA429241591A5242891A072264463A401E
:109C800092E501430F00791E8F419DE71C000F00F4
:109C9000203CE740202B03D04024E31A994008439E
:109CA000411E884138437CE60022002425E6171A2D
:109CB0004346BA429241591A5242891A64463500C3
:109CC00043E541461000144D10E6802200241203A3
:109CD00080E61D000F00203DEF40BC46202B03D046
:109CE0004025EB1A9940084307006346781E8741D8
:109CF0001F4369E7871897429B4141445B42C9185B
:109D00003500A3E53B003343CED0072231003A4073
:109D100052E600231A00F4E5FF070000FFFF7FFF73
:109D2000F0B55746DE464E464546E0B58346070049
:109D30000E03480085B092461C00360B400DCD0F37
:109D4000002800D19DE0954B984239D08023F60041
:109D50001B041E43924A7B0F3343994694460300EB
:109D60006344009300230026FF00029323031B0B90
:109D700098466300E40F52465B0D019400D1B3E0B6
:109D800086498B4200D19EE04246D10080221204D7
:109D90000A435146490F11438B46814952468C462E
:109DA00000996344CB1A0021D20000932B0063403A
:109DB0009A460F2E00D905E17A4BB6009B599F4673
:109DC0005B463343994600D0B8E0022308260027BB
:109DD00000900293CAE7CB463A0002990195019B95
:109DE0009A46022927D0032900D180E2012944D0D4
:109DF0006D49009B8C4663441C00002C38DD5307E2
:109E000000D013E2D2085B46DB0109D55946674B07
:109E100019408B468021C9008C46009B63441C007E
:109E2000634B9C4207DC5B4664055F075B0217439C
:109E30001B0B620D02E000230027584A00211B0380
:109E40001C0B0B0D1B05234314055A4A3800134005
:109E50001C4353466400DB0764081C43210005B023
:109E60003CBC90469946A246AB46F0BD0122524208
:109E700001231B1B382B00DCADE10022002300274F
:109E8000DCE75B46334399465ED0002E00D18AE181
:109E9000300001F0E7F903000B3B1C2B00DD7BE1F8
:109EA0001D22D31A5A460100DA4008398E401300A9
:109EB0005F46334399468F403F4B00261B1A009361
:109EC0000023029352E7414653460B433B499B46CE
:109ED0008C46009B634400935B46002B3BD10223DE
:109EE00000221E43022161E7434613439B4637D0BD
:109EF0004346002B00D162E1404601F0B3F9030074
:109F00000B3B1C2B00DD53E102004146083A914017
:109F100088461D21CB1A5146D9400B0041460B43C0
:109F20009B46534693401A00009B25499C4660443B
:109F300003008C4663440093002137E70323B146B6
:109F400000900C26029311E70023009301330426AE
:109F5000002702930AE70323C3461E43032125E794
:109F600001331E430022012120E700239A4680236B
:109F700000271B03094A61E7802349461B03194256
:109F800000D1E2E05946194200D0DEE00B431B034A
:109F900017001B0BA246014A50E7C046FF0700000E
:109FA00001FCFFFF30E00000FF030000FFFFFFFEA9
:109FB000FE070000FFFF0F800DFCFFFF01F8FFFF11
:109FC000F3030000D94500D9CBE000D1C6E03C0046
:109FD00048460027009B013B00935B46160E1B0280
:109FE0001E431302984633041B0C9946310C019111
:109FF000FFF798F84A4642430B04210C0500194329
:10A000008A4207D98919013D8E4203D88A4201D973
:10A01000851E8919881A0199FFF784F809048C466E
:10A020004A46210464464243090C030021438A4204
:10A0300004D98919013B8E4200D8F1E02D041D435B
:10A04000AB464346891A4246280C12041D0C5B4657
:10A05000140C22001B041B0C5A4303946B4344430F
:10A06000029568431B19150CEB189C4203D98024F8
:10A070006402A44660441C0C15041B042D0C20181B
:10A080005D19814277D373D00C1AA24A7D1BAF426F
:10A09000BF419446009B7F426344E01B1C00864204
:10A0A00000D1DBE00199FFF73DF84A4642430B043B
:10A0B000290C070019438A4207D98919013F8E42AA
:10A0C00003D88A4201D9871E8919881A0199FFF796
:10A0D00029F809044A46894629044D464243090C99
:10A0E000030029438A4207D98919013B8E4203D8CC
:10A0F0008A4201D9831E89193F04891A3A00039FB5
:10A100001A43380013041B0C584381460298150C5F
:10A110006F43434345434846000C8446DB19634480
:10A120009F4203D9802040028446654448461F0C64
:10A1300000041B04000C7D191818A94200D284E009
:10A1400000D17FE001231A4357E680234A461B03D0
:10A1500013431B031B0BAA466F4A6FE6BA4200D992
:10A1600035E74B46DC0758087B081C43FF0734E7FC
:10A170000024AF4289D247444745A4415B4664422C
:10A18000A4196418013BA6421ED2A0426DD800D18A
:10A19000B6E0241A9B4678E703005A46283B9A40CB
:10A1A0000027914688E6584601F05CF8203072E6B8
:10A1B00003005246283B9A4093460022B4E650469C
:10A1C00001F050F820309AE6A642E2D1B845DCD939
:10A1D000341A9B4659E71F2B65DC504C0099A44666
:10A1E0005C46614408008C4011008240D940501EFA
:10A1F00082410C4314435A46DA401300620709D0E7
:10A200000F222240042A05D02200141D94428941C5
:10A2100049425B181A0262D50122002300270DE68D
:10A220008A4200D80AE7831E891907E70F231340E3
:10A23000042B00D1E6E5171D9742924153429B44FF
:10A24000FA08E0E5002800D1D7E57118531EB142A5
:10A2500027D3A94215D358D01A0073E7002B00DC8E
:10A2600004E6012300229B44CDE5022347444745F1
:10A2700089415B429C46494289190C19E344241ADE
:10A2800003E743465F0047459B41B8465B429E1942
:10A29000023A8919A94200D054E7404500D051E75D
:10A2A000ABE51A00F6E71F215F4649420C1BE74069
:10A2B000202B07D01A49009B8C46634418005B464C
:10A2C00083401A43501E82413A4307270023174018
:10A2D00009D00F21002311401400042995D1220038
:10A2E0005F075B021B0BD20817430022A6E5802301
:10A2F00059461B030B431B0317001B0B064A9DE526
:10A30000BD42B2D89B460024BFE68045B9D31A00AF
:10A31000C3E7C046FF030000FF0700001E04000063
:10A320003E040000F0B54F464646D6468446C0B5CA
:10A330008046194E18030F034D00000B5C00824647
:10A340003F0B6D0DC90F9146640DDB0F0120B54227
:10A350000AD0B44203D0A54201D157450CD01CBC51
:10A3600090469946A246F0BD66463E43F7D1AC42C0
:10A37000F5D154461443F2D10120C845EFD199429A
:10A3800007D0002DEBD163461F433800471EB8416C
:10A39000E5E70020E3E7C046FF070000F0B54F46C1
:10A3A0004646D6464D00C0B50E03C90F8A462C4915
:10A3B0001F035C008046360B6D0D91463F0B640D0C
:10A3C000DB0F8D421ED08C4216D0002D1ED13043A3
:10A3D0008446002C01D13A4323D06246002A1AD089
:10A3E0009A4529D0514602200139084001381CBC49
:10A3F00090469946A246F0BD39001143E5D00220AF
:10A400004042F4E73043FAD1AC420FD0002C0FD1D8
:10A410003A43E7D00CE00122013B9343180001309E
:10A42000E5E763460020002BE1D0DBE73A43E6D1C5
:10A430009A45D7D1A542D5DCA54205DBBE42D1D88D
:10A4400008D00020BE42D2D25046012301389843A2
:10A450000130CCE7C845C5D80020C845F4D3C6E7CD
:10A46000FF070000F0B54F464646D6464D00C0B542
:10A470000E03C90F8A462E491F035C008046360B27
:10A480006D0D91463F0B640DDB0F8D4218D08C4251
:10A4900011D0002D18D130438446002C1ED13A43F0
:10A4A0001CD163460020002B30D0514602200139D8
:10A4B000084001382AE039001143EAD0022025E0A3
:10A4C0003043FBD1AC4226D0002C26D13A4324D1D4
:10A4D0005146022001390840013817E06246002A3F
:10A4E0000FD09A45E1D1A54205DBBE42DDD819D097
:10A4F0000020BE420AD25046012301389843013061
:10A5000004E00122013B9343180001301CBC90463B
:10A510009946A246F0BD3A43D0D19A45C5D1A5424D
:10A52000C3DCE0E7C845C0D80020C845E3D3EDE769
:10A53000FF070000F0B55746DE464E464546E0B5FB
:10A54000834606000F03480087B092461D003F0B6C
:10A55000400DCC0F002800D16FE0DE4B984238D080
:10A560008023FF001B041F43730F3B430193DA4B0F
:10A570000027994600239B46F60081442B0369007F
:10A580001B0B52469846490DED0F002900D185E07E
:10A59000D04B994200D173E04346DA0080231B047C
:10A5A00013435246CC48520F844613435246002070
:10A5B0006144D20089442100694000918C46012108
:10A5C00049448A460F2F00D990E0C449BF00CF59B3
:10A5D000BF465B463B43019300D06AE10223082754
:10A5E000002681469B46C9E732005846019B6146DA
:10A5F0000091022800D175E0032800D1FEE1012876
:10A6000000D02CE100230027002600253F032A0D5F
:10A610003F0BB34812053A4302401B051343009A0F
:10A620005B00D1075B080B433000190007B03CBC4E
:10A6300090469946A246AB46F0BD5B463B4301932C
:10A6400000D12FE1002F00D1A5E1380000F00AFE73
:10A6500003000B3B1C2B00DD96E11D22D31A5A464A
:10A660000100DA405E4608398F4013008E403B43BC
:10A6700001939C4B00271B1A994600239B467DE7BC
:10A68000414653460B4393498C46E144002B00D08E
:10A690001AE102220220174300228CE7134300D163
:10A6A0000DE14346002B00D181E1404600F0DAFD88
:10A6B00002000B3A1C2A00DD72E101004346083912
:10A6C0008B4098461D239A1A5346D3401A0043469E
:10A6D000134352468A404946081A824989468144B2
:10A6E000002068E77B4B002700268EE7140C12043D
:10A6F000120C1100370C3604350C794328008C46B7
:10A700002E0060436044834656432100300C80464F
:10A710005846794340440291844506D988468021B1
:10A7200049028C46E044414602913604010C360C45
:10A7300000048B4681191E0C1B041B0C039119008D
:10A7400079438C46280075436544A8465843050C58
:10A7500045447743A94203D9802149028C46674486
:10A76000290C8C4639000004000C2D042D1861447E
:10A77000AB4405915946049101990F043F0C080C14
:10A78000390051434243904602008C46090C8B46E7
:10A7900062437C4344445C44A04503D98021490280
:10A7A00088464244210C884661460904090C8C46BF
:10A7B00039005943434370437E430F0CF618240479
:10A7C000BE19644442448C46B34203D980235B02E1
:10A7D00098464044029B61469846049B3704434494
:10A7E0009B46AB45AD416B420D0405992D0C8C4643
:10A7F0007F196744FD18A8465D462D19A542A4415E
:10A8000093466442A446C344DC448F42BF4198450A
:10A810009B4193459241A445A4415B427F421F4323
:10A82000360C52426442BF192243BF1862463818A0
:10A830004302D20D039913436A020A43501E824118
:10A840006146ED0D2A434E023243D90100D4B3E0F4
:10A850000126500832400243DE0732435B08224C97
:10A860005444002C62DD510709D00F201040042809
:10A8700005D0101D9042924152429B180200D9010E
:10A8800004D580241948E400034054441848844205
:10A8900000DD27E75E075B02D2081F0B6305164346
:10A8A0005B0DB2E6002399460133042700269B4640
:10A8B00064E60323019781460C279B465EE601224E
:10A8C00001201743002276E6032303201F4343465B
:10A8D00071E6C046FF07000001FCFFFF70E00000CA
:10A8E000FFFF0F800DFCFFFFFF030000FFFFFFFED7
:10A8F000FE0700000023802700933F030026434B00
:10A9000083E6019B3200A446584670E6AC466EE6EC
:10A91000802701993F0339422DD03B422BD11F4361
:10A920003F033F0B00951600384B6EE601252D1BAB
:10A93000382D00DD66E61F2D40DC35481C005044F4
:10A94000160082408440EE40501E8241344314433E
:10A95000EB40620709D00F222240042A05D02200D2
:10A96000141D9442804140421B181A023ED5012317
:10A970000027002649E68027019B3F031F433F0332
:10A980003F0B0094214B40E603005A46283B9A4077
:10A99000002601926DE6584600F064FC203057E630
:10A9A00003005246283B9A401300002293E650468B
:10A9B00000F058FC20307BE6CA4650E71F201E00FE
:10A9C0004042041BE640202D03D0124C5444A340C7
:10A9D0001A43501E8241324307260027164009D0F1
:10A9E0000F200023104014000428B9D122005E0774
:10A9F0005B021F0BD2081643002306E680273F03A5
:10AA00001F433F033F0B1600004BFEE5FF0700000E
:10AA10001E0400003E040000F8B557464E46454669
:10AA2000DE460C000903E0B5490A460F5F003143DA
:10AA30001E03DB0F760A9B46530F3343C84E650057
:10AA4000C000E40FD2006D0DA24681467F0D9C46EA
:10AA50009046B74200D1B9E05B46012673409B4661
:10AA6000EE1BA34500D183E0002E63DD002F00D054
:10AA7000B1E06346134300D123E1731E002B00D0E5
:10AA8000BAE1861A6346B04280410125C91A4042A4
:10AA9000091A0B0200D447E149024B0A9846434683
:10AAA000002B00D189E1404600F0DCFB0300083BAD
:10AAB0001F2B00DD7CE120223000D21A4146D0401D
:10AAC000994002009E400A439D4200DD6AE15D1B01
:10AAD0006B1C1F2B00DD94E1202110003500C91AEA
:10AAE0008E40DA408840DD40711E8E411100072201
:10AAF0002843002506433240002A09D00F23334063
:10AB0000042B05D0331DB342B641764289191E008D
:10AB10000B0200D43DE26A1C914B55056D0D9A4223
:10AB200000D119E18F4AF6080A405707520237430D
:10AB3000120B9BE0002E00D0C5E06E1C7605760D52
:10AB4000012E00DC48E16746861ACB1BB042BF41AC
:10AB50007F42B8461F004346FF1A3B00B8461B021F
:10AB600000D55FE137439AD100220024002579E027
:10AB7000002E00DCFAE0002F00D18DE0784B9D42E2
:10AB800067D0802367461B041F43BC46382E00DC79
:10AB900052E1634613435A1E93411E188642804178
:10ABA000404209180B0200D4BEE06D4B01359D42B6
:10ABB00000D1D2E06B4A73080A4001210E401E43C7
:10ABC0005108D30707221E43324095E71E00164363
:10ABD00000D045E740E7624B9D423AD0802367466C
:10ABE0001B041F43BC46382E00DDEBE01F2E00DCAB
:10ABF0003AE133006746203BDF403B00202E05D082
:10AC00004027BF1B6646BE40324390464646721EF2
:10AC100096413343DAE0002B00D114E2634613433C
:10AC200000D168E180234E07C008C9081B03064312
:10AC3000194208D06046C008184204D1634601009A
:10AC4000D2085E071643F3009946C900720F444DBF
:10AC500011434B46DE08424B4F073743CA089D421B
:10AC600000D16EE012036D05120B6D0D0021120371
:10AC7000130B0A0D12051A433B4B2D0513402B43B2
:10AC80005B00E4075B082343380019003CBC904696
:10AC90009946A246AB46F8BD6346134311D0731ED6
:10ACA000002B00D007E18618864280416144404273
:10ACB000091801250B0237D502257BE73E006146C6
:10ACC00091463500C5E75C46002D00D0E1E00B0061
:10ACD0000343F3D0731C00D1ACE1214B9F4200D160
:10ACE0003AE1F343382B00DD6FE11F2B00DD8CE1EF
:10ACF00020250E00ED1AAE40B0460600AA46DE4002
:10AD0000454635432E005546D940A8406346451E6A
:10AD1000A8415B1A9C463043161AB24292416346E0
:10AD20005242991A3D00B4E607223240002A00D070
:10AD3000E4E60B4BF6084F073743CA089D4200D0A4
:10AD400090E73B00134300D1A6E180231B031A4385
:10AD50001203120B024D89E715000022002785E738
:10AD6000FF070000FFFF7FFFFFFF0F80002E00D0D6
:10AD7000C7E06B1C5E05760D012E00DCF0E0C84DCF
:10AD8000AB4200D1B9E085180A008542894162448E
:10AD9000494251180722CE076D082E434908324018
:10ADA0001D00A9E6BF49ED1A114007223240A3E673
:10ADB000320028388240002686E6300000F052FA41
:10ADC000203073E6634613435A1E9341C61AB042BD
:10ADD00080414042091A5CE60E006746064317436D
:10ADE000002D5ED1002E00D0F3E0002F00D11EE137
:10ADF0005C46614691462CE7A94FBE427BD01E00BF
:10AE0000F1E610001F3DE840202B03D04021CB1A73
:10AE10009A401643731E9E4107220643324000218A
:10AE2000002583E7161A6346B2428041591A404210
:10AE30000B1A98465C4632E61F2E00DDABE0202759
:10AE4000BB1B9A4663465746BB40994613004F4684
:10AE5000F3401F433B005746BA40571EBA411343C5
:10AE60006246F240891898E62027BB1B9A46634643
:10AE70005746BB40994613004F46F3401F433B00E3
:10AE80005746BA40571EBA4113436246F240891AE8
:10AE90009CE7834B9F425FD080252D04734229435A
:10AEA00020E7002E0CD1002F00D1D0E05C46614697
:10AEB00091467B4DCDE67A4FBE421CD01E0065E622
:10AEC000002F18D0C0084E0706438020C908000391
:10AED000014208D06346DC08044204D12100DA466E
:10AEE000D2085E071643F300994601245346C90071
:10AEF000720F11431C406A4DABE61D000022002773
:10AF0000B4E6002D59D10B00034300D1D6E6731CE3
:10AF100000D1B2E0624B9F421ED0F343382B6FDC6E
:10AF20001F2B00DD97E020250E00ED1AAE40B04645
:10AF30000600AA46DE40454635432E005546A84049
:10AF4000D940451EA8418C440643B618964292410A
:10AF5000514261443D0025E63D006146914678E658
:10AF60000B000343002D00D055E6002BF5D06346BF
:10AF7000134300D16DE68618864280416144404209
:10AF8000091800220B0200D4D0E6464B01351940C7
:10AF9000B2E5B1465DE633006746203BDF403B004B
:10AFA000202E05D04027BF1B6646BE403243904648
:10AFB0004646721E96413343EFE5394B9F42CBD054
:10AFC00080252D0473422943A8E70843411E884188
:10AFD000A2E6002F00D13CE66346861ACF1AB042A3
:10AFE0009B415B42FB1A98461B024ED5161A6346DC
:10AFF000B2429241591A5242891A5C4600227BE5BC
:10B0000001430E00711E8E419FE71D000E00203D82
:10B01000EE40B046202B04D04025EB1A994008435F
:10B02000814648464346411E8841184374E6002243
:10B03000002417E6161A6346B2429241591A524248
:10B04000891A3D0025E561469146154D01E68022AD
:10B050000024120379E61D000E00203DEE40B046AC
:10B06000202B04D04025EB1A9940084381464E46D8
:10B070004346711E8E411E4367E7861896429B41E8
:10B0800061445B42C9183D008CE547463743CED04A
:10B0900007224146324049E600273A00E6E5C0462D
:10B0A000FF070000FFFF7FFF70B50C4E0D031C0370
:10B0B00049005B002D0B490D240B5B0DB14208D0FC
:10B0C000064900208B4203D114432000441EA041B6
:10B0D00070BD05430120002DFAD1F1E7FF07000004
:10B0E00030B5144D0A034B00120B5B0DC90F002441
:10B0F000AB4211DD104CA34210DC802464032243D8
:10B100000E4CE41A1F2C0CDD0D48C31ADA40130054
:10B110005C42002900D11C00200030BD094BCC1836
:10B12000FAE7094DE040AC4663449A4013000343FC
:10B13000EEE7C046FE0300001D04000033040000DB
:10B1400013040000FFFFFF7FEDFBFFFF70B5002839
:10B150002DD0C317C5185D40C40F280000F082F839
:10B16000154B1B1A5B055B0D0A2815DD0B38854056
:10B1700000222D032D0B002110002D030A0D2D0B95
:10B1800012052A430D4D1B052A4013435B00E407BB
:10B190005B082343190070BD02002900153291405D
:10B1A0000A000B21081AC5402D032D0BE3E70024EC
:10B1B000002300250022DEE71E040000FFFF0F80B1
:10B1C0004100090E4B1C70B5DBB24602750AC40F74
:10B1D000012B14DDE0239B006D07360BCB180021FB
:10B1E0000A0D280012051C4D32435B052A405B08FE
:10B1F00013435B00E4075B082343190070BD00297B
:10B2000014D1002D1ED0280000F02CF80A281CDCD8
:10B210000B232A001B1ADA40030015339D400F4B05
:10B2200012031B1A5B05160B5B0DD8E7002D06D029
:10B23000320B802636036D071643094BCFE7084BC8
:10B240000026CCE700230026C9E703002A000B3BB9
:10B250009A400025E3E7C046FFFF0F808903000006
:10B26000FF0700001C2101231B04984201D3000C9E
:10B2700010391B0A984201D3000A08391B09984269
:10B2800001D30009043902A2105C40187047C0467F
:10B29000040302020101010100000000000000009F
:10B2A00030B51C00094B05001B6885B0D868084BF9
:10B2B000002A01D1074B1A000292019300912B0042
:10B2C0002200054900F026F800F0A6FD80000020CD
:10B2D000B0E00000E8CE0000BDE00000014B1868BF
:10B2E0007047C04680000020084B10B50400002BBA
:10B2F00002D0002100E000BF054B1868836A002BD4
:10B3000000D09847200001F05DFBC046000000001F
:10B31000ECE000000EB403B5010003AB044804CB1D
:10B320000068019300F076F802B008BC03B018473B
:10B330008000002070B500260C4D0D4C641BA4103D
:10B34000A64209D1002601F03FFB0A4D0A4C641BBE
:10B35000A410A64205D170BDB300EB589847013642
:10B36000EEE7B300EB5898470136F2E750020020B1
:10B37000500200205002002060020020002310B57F
:10B380009A4200D110BDCC5CC4540133F8E710B52B
:10B39000884202D98B18984203D3002307E08B5CC4
:10B3A0008354013AFBD210BDCC5CC45401339A42A1
:10B3B000FAD1F8E703001218934200D170471970D0
:10B3C0000133F9E7936810B5013B9360002B04DA71
:10B3D0009469A34207DB0A2905D01368581C106042
:10B3E0001970080010BD00F04BFC0100F9E7F8B53A
:10B3F00006000F001400D518AC4201D1002007E070
:10B4000021783A003000FFF7DDFF0134431CF3D10F
:10B41000F8BD0000F0B59FB002900F001600059334
:10B42000002805D083690493002B01D100F0F4FDBE
:10B430007B4B9F425BD1029B5F68BB891B0762D538
:10B440003B69002B5FD0002306AC63612033637639
:10B450001033A37635002B78002B01D0252B5CD13F
:10B46000AB1B04930CD0320039000298FFF7BFFFEA
:10B47000431C00D1C4E06269049B94466344636149
:10B480002B78002B00D1BBE00122002352426260E6
:10B4900002A9543252186E1C2360E360A36013703B
:10B4A000A365317805225F4800F0D4FE751C0028A2
:10B4B00035D12268D30604D5532302A95B18202175
:10B4C0001970130704D5532302A95B182B21197097
:10B4D00033782A2B2CD0350000210A20E3682A7803
:10B4E0006E1C303A092A64D900292ED026E04E4B32
:10B4F0009F4202D1029B9F689FE74C4B9F429CD189
:10B50000029BDF6899E73900029800F00FFC0028E1
:10B5100099D0012040421FB0F0BD01359BE7414B5F
:10B520002268C01A01238340134323602E00B8E72A
:10B53000059B191D1B680591002B01DB099304E095
:10B540005B42E3600223134323602B782E2B0AD146
:10B550006B782A2B35D1059B02351A1D1B68059285
:10B56000002B2BDB0793324E29780322300000F0AA
:10B5700071FE002806D04023801B834022680135DD
:10B5800013432360297806222A486E1C217600F096
:10B5900061FE00283AD0284B002B25D10722059BBD
:10B5A00007339343083305936369039A9B186361D8
:10B5B00050E7434301219B18350090E701235B428C
:10B5C000D0E700230A201A000135636029786E1C39
:10B5D0003039092903D9002BC5D00792C3E742436C
:10B5E000012352183500F1E705AB00933A00134BE5
:10B5F0002100029800E000BF0390039B0133D3D1E8
:10B60000BB895B0600D584E70B9884E705AB009304
:10B610003A000A4B2100029800F080F8ECE7C0469F
:10B6200044E10000F0E0000064E1000024E10000DB
:10B63000F6E00000FAE0000000000000EFB30000B8
:10B64000F7B5150001938A680B6900900C009342CE
:10B6500000DA130022002B6043321278002A01D056
:10B6600001332B6023689B0602D52B6802332B60C5
:10B67000062723681F4027D0230043331B785A1E18
:10B6800093412268920630D42200019943320098F7
:10B69000089EB047431C25D0062320682A68E1682D
:10B6A00003400025042B03D18D1AEB43DB171D400B
:10B6B000A3682269934201DD9B1AED180027BD4261
:10B6C00020D1002010E00137E3682A689B1ABB42B2
:10B6D000D2DD22000123193201990098089EB0475B
:10B6E000431CF0D101204042FEBD3020E11843311F
:10B6F000087021005A1C45310978A21843320233E0
:10B700001170C1E7220001231A3201990098089EA6
:10B71000B047431CE6D00137D1E70000F0B589B04F
:10B7200004920A0043320593039002920A7E0C00B1
:10B730000E9B6E2A00D186E01FD8632A33D008D82A
:10B74000002A00D18CE0582A4DD0250042352A70BD
:10B7500030E0642A01D0692AF7D1196825680A1DEA
:10B76000280629D508681A60002803DA2D23029AD2
:10B77000404213706B4E0A274FE0732A74D008D8EA
:10B780006F2A1FD0702AE0D1202209680A43226064
:10B7900003E0752A16D0782AD7D1220078214532C5
:10B7A0001170614E22E025001A684235111D1960A2
:10B7B00013682B70012365E008681A606906D3D509
:10B7C00000B2D1E719682568081D186008682E06C0
:10B7D00005D5544E08276F2A1BD00A2719E06D069D
:10B7E000F7D580B2F5E745314E4E0A7018682268E9
:10B7F000011D00681960150621D5D30702D5202345
:10B800001A4322601027002803D1202322689A437C
:10B8100022602300002243331A706368A360002B68
:10B8200058DB0422216891432160002854D1029DF5
:10B83000002B5AD02500337842352B7055E0550641
:10B84000DBD580B2D9E71A680D68101D4969186008
:10B8500013682E0601D5196002E06D06FBD519802C
:10B860000023029D23614FE01A68111D19601568BD
:10B8700000216268280000F0EDFC002801D0401B88
:10B880006060636823610023029A13703CE02369BF
:10B890002A0004990398059DA847431C3ED02368BD
:10B8A0009B0715D4079BE068984239DA180037E007
:10B8B00022000123193204990398059EB047431CC6
:10B8C0002CD00135E368079A9B1AAB42F0DCE9E71C
:10B8D0000025F7E70028ADD0029D3900FDF722FCD6
:10B8E000735C013D2B700028F7D1082F09D1236824
:10B8F000DB0706D563682269934202DC3023013DF1
:10B900002B70029B5B1B2361059B07AA0093210000
:10B91000049B0398FFF794FE431CB8D101204042DA
:10B9200009B0F0BD01E1000012E100000D4B70B55F
:10B930001C680500A36B002B0FD1182000F06EFCD3
:10B94000094BA0630360094B01224360084B8360ED
:10B950000B2383810023026143610022A36B1D61DD
:10B960005A6170BD800000200E33CDAB34126DE6FD
:10B97000ECDE0500124B10B51C68A36B002B0FD139
:10B98000182000F04BFC0F4BA06303600E4B01220C
:10B9900043600E4B83600B2383810023026143616C
:10B9A000A46B0B4A206961690A4BFDF7F7FC012281
:10B9B000002380185941206161614800400810BD92
:10B9C000800000200E33CDAB34126DE6ECDE0500B6
:10B9D0002D7F954C2DF451580CB430B5164B9DB0BD
:10B9E0000C1E1D6808DA8B2301202B6040421DB01D
:10B9F00030BC08BC02B01847822302A99B008B818F
:10BA00000023029008619C4200D0631E8B604B6152
:10BA100001235B42CB81209A21AB2800019300F0E7
:10BA200055FD431C01DA8B232B60002CDFD0002353
:10BA3000029A1370DBE7C046800000200EB400B508
:10BA40000B499CB01DAB02900690079104910948E8
:10BA5000094904CB0591006802A9019300F036FD65
:10BA60000023029A13701CB008BC03B01847C046EC
:10BA7000FFFFFF7F800000200802FFFF020010B5DB
:10BA80001378541C002B05D1CC5CD4540133002C0A
:10BA9000FAD110BD2200F3E7C9B20378002B04D01D
:10BAA0008B4200D170470130F7E74B425941494280
:10BAB0000840F7E702780B78002A03D00130013103
:10BAC0009A42F7D0D01A70470023C25C0133002A93
:10BAD000FBD1581E7047002330B59A420AD0013A74
:10BAE000C45CCD5CAC4204D1934202D00133002C43
:10BAF000F6D1631B180030BD30B50500002A00D117
:10BB000030BD0C78013A6B1C2C700131002C05D132
:10BB10009A189A42F4D01C700133FAE71D00EDE741
:10BB200010B50378002B0FD10B785A4253415B427A
:10BB3000184010BD0023CA5C002AFAD0C45C9442AD
:10BB400001D10133F7E701300378002BF2D118005F
:10BB5000EFE70000F0B51F000E0087B005900191DF
:10BB600002920C98347800F0EAFA0822001943781F
:10BB7000751C134036D12D2C36D1B51C7478012696
:10BB8000002F62D0102F09D1302C07D120222B7822
:10BB90009343582B54D110276C7802352D4B390024
:10BBA000F31818000393FDF7BDFA04910121002357
:10BBB000494202008C4618002100303909291AD860
:10BBC0000C00A74223DD591C09D06346824206D3EC
:10BBD00002D10499A14202DB0123784320182C787A
:10BBE0000135E9E72E00BCE72B2C01D01E00C7E78A
:10BBF000B51C7478FAE721004139192901D8373C7E
:10BC0000DFE721006139192901D8573CD9E75A1CCF
:10BC100008D1059A23331360029B0398002B09D1A6
:10BC200007B0F0BD002E00D04042029A002AF7D0A3
:10BC3000002B01D06B1E0193029B019A1A60EFE763
:10BC40003024002FAAD10827A8E7302C9ED00A273D
:10BC5000A4E7C046FFFFFF7F37B51300064A050083
:10BC60001068046A002C00D1044C0A0000942900DA
:10BC7000FFF770FF3EBDC04680000020E4000020BA
:10BC8000F8B505000E001400002804D08369002BCD
:10BC900001D100F0C1F9224B9C422DD16C68A369FF
:10BCA000A360A3891B0731D52369002B2ED02368FD
:10BCB0002269F7B2981A6369F6B2834205DC210063
:10BCC000280000F03BF9002826D1A3680130013B91
:10BCD000A36023685A1C22601F706369834204D0EA
:10BCE000A389DB071AD50A2E18D12100280000F0FD
:10BCF00025F9002812D00FE00A4B9C4201D1AC6814
:10BD0000CDE7094B9C42CAD1EC68C8E72100280066
:10BD100000F00CF80028CAD0012676423000F8BDA9
:10BD200044E1000064E1000024E10000364B70B5FE
:10BD30001D6806000C00002D05D0AB69002B02D158
:10BD4000280000F069F9314B9C420FD16C680C233C
:10BD5000E25E93B219072DD4D90611D4092301202C
:10BD6000336037331343A381404270BD284B9C425C
:10BD700001D1AC68EBE7274B9C42E8D1EC68E6E7E1
:10BD80005B0713D5616B002908D023004433994227
:10BD900002D0300000F06AFA002363632422A389F2
:10BDA0009343A38100236360236923600823A2894E
:10BDB0001343A3812369002B0BD1A0218022A389E7
:10BDC000890092000B40934203D02100300000F024
:10BDD000E1F90123A289134011D00023A360636914
:10BDE0005B42A361002023698342BED10C23E25E43
:10BDF0001306BAD540231343A3810138B5E7920750
:10BE000000D46369A360EDE78000002044E10000F6
:10BE100064E1000024E1000010B5062000F090FC71
:10BE2000012000F0CFFD0000F7B58A8905000C0065
:10BE3000130760D44B68002B04DC0B6C002B01DC77
:10BE40000020FEBDE76A002FFAD000232E682B6089
:10BE500080235B01216A1A4034D0606DA3895B079F
:10BE600006D56368C01A636B002B01D0236CC01A1F
:10BE70000200216A00232800E76AB847A189431C11
:10BE800006D12B681D2B30D82B4ADA40D3072CD58E
:10BE90000023636023692360CB0405D5431C02D1D2
:10BEA0002B68002B00D16065616B2E600029C7D024
:10BEB00023004433994202D0280000F0D7F9002033
:10BEC0006063BEE701232800B847431CC6D12B6836
:10BED000002BC3D01D2B01D0162B01D12E60AFE754
:10BEE0004023A2891343A381ABE740230B430120E6
:10BEF000A3814042A5E70F69002FA1D00B680F6016
:10BF0000DB1B01930023920700D14B69A360019BC7
:10BF1000002B00DC94E7019B3A00216A2800A66A06
:10BF2000B047002803DC4023A2891343DFE7019BCD
:10BF30003F181B1A0193EAE7010040200B6970B516
:10BF400005000C00002B01D1002070BD002804D09A
:10BF50008369002B01D100F05FF80B4B9C4209D1A3
:10BF60006C680C22A35E002BEED021002800FFF7A6
:10BF70005BFFEAE7054B9C4201D1AC68F1E7044B5B
:10BF80009C42EED1EC68ECE744E1000064E1000083
:10BF900024E10000002310B50400036043608360C7
:10BFA00081814366C2810361436183611900082274
:10BFB0005C30FFF7FFF9054B24626362044BA36218
:10BFC000044BE362044B236310BDC04681C70000ED
:10BFD000A9C70000E1C700000DC8000010B5024964
:10BFE00000F08CF810BDC0463DBF000070B568255C
:10BFF0004A1E55430E002900743100F081F9041ED9
:10C0000008D000212A00016046600C30A060683230
:10C01000FFF7D0F9200070BD836913B50400002B31
:10C0200028D18364C3640365134B144A1B6882627E
:10C030000193984201D101238361200000F020F890
:10C040006060200000F01CF8A060200000F018F8EC
:10C050000022E06004216068FFF79CFF01220921B3
:10C06000A068FFF797FF02221221E068FFF792FF16
:10C070000123A36113BDC046ECE00000DDBF00005A
:10C08000F8B51C4B07001E68B369002B02D13000C5
:10C09000FFF7C2FF4836B4687368013B04D53368C4
:10C0A000002B07D03668F6E70C22A55E002D0DD0D8
:10C0B0006834F2E704213800FFF798FF3060002869
:10C0C000F0D10C2304003B602000F8BD20000A4B97
:10C0D000656625606560A560E36025616561A561B1
:10C0E000082229005C30FFF765F96563A563A56444
:10C0F000E564E9E7ECE000000100FFFFF7B50400AC
:10C100000700002601914834002C01D13000FEBD0B
:10C110006368A5680093009B013B009301D52468E8
:10C12000F2E7AB89012B08D90E22AB5E013304D0B4
:10C1300029003800019B984706436835EBE7EC304F
:10C140000068704770B50E001D000E23C95E96B0E2
:10C150001400002907DA00232B60B3891B0611D4D1
:10C160008023DB000FE06A4600F088FB0028F2DB4A
:10C17000F022019B12021340054A9B185A42534178
:10C180002B60EDE740230020236016B070BDC04651
:10C1900000E0FFFFF7B502268B8905000C00334253
:10C1A00006D0230047332360236101236361F7BD79
:10C1B00001AB6A46FFF7C6FF00990700280000F0B0
:10C1C0009FF8002808D10C22A35E9A05EFD4032221
:10C1D00093431E43A681E4E70F4BAB628023A28901
:10C1E00020601343A381009B20616361019B002BAE
:10C1F0000DD00E23E15E280000F052FB002806D08F
:10C200000322A38993431A0001231343A381A08926
:10C210003843A081CBE7C046DDBF000010B5034B1B
:10C220000100186800F06CF810BDC04680000020C6
:10C2300082B0002900D101A9101E06D0002B06D023
:10C2400013780B601078431E984102B070470220AB
:10C250004042FAE7C9B28218904201D100207047EB
:10C2600003788B42FBD00130F6E7000070B5050083
:10C27000002910D00C1F2368002B00DAE4182800D6
:10C2800000F034FB1D4A1368002B05D16360146075
:10C29000280000F02CFB70BDA34209D9216860186A
:10C2A0008342F3D118685B6841182160EEE7130000
:10C2B0005A68002A01D0A242F9D919685818A04238
:10C2C0000BD120680918581819608242E0D1106813
:10C2D0005268411819605A60DAE7A04202D90C236B
:10C2E0002B60D5E721686018824203D1106852683C
:10C2F0004118216062605C60CAE7C0461C1C0020D7
:10C30000032370B5CD1C9D43083506000C2D1ED2AD
:10C310000C25A9421DD8300000F0E8FA254A14681F
:10C320002100002919D1244C2368002B03D13000AF
:10C3300000F0CAF920602900300000F0C5F9431C64
:10C340002BD10C233000336000F0D1FA03E0002D34
:10C35000DFDA0C233360002070BD0B685B1B19D43F
:10C360000B2B03D90B60CC18256003E04B688C4283
:10C370000DD11360300000F0BAFA200007220B3014
:10C38000231D9043C31AE7D05A42E250E4E76360AA
:10C390000C00EFE70C004968C3E70323C41C9C436F
:10C3A000A042E1D0211A300000F08EF9431CDBD10D
:10C3B000C7E7C0461C1C0020201C0020F8B5070061
:10C3C0000D001600002905D11100FFF799FF0400A8
:10C3D0002000F8BD002A03D1FFF748FF3400F7E73B
:10C3E00000F086FA2C00B042F2D231003800FFF79C
:10C3F00087FF041EECD029003200FEF7BFFF2900A2
:10C400003800FFF733FFE3E7F0B58E6885B007002B
:10C410000C00039201939E423CD890238A89DB0052
:10C420001A4234D00325096923685B1A02936369B1
:10C4300002985D43EB0F5D19019B6D1001331B18D2
:10C44000AB4200D91D00530532D529003800FFF753
:10C4500057FF061E09D10C233B6040230120A2890F
:10C4600040421343A38105B0F0BD029A2169FEF753
:10C4700085FFA389144A1A4080231343A381029B9A
:10C480002661F61826606561019EED1AA560019B84
:10C490009E4200D9019E320003992068FEF777FF83
:10C4A000A36800209B1BA36023689E192660DAE71F
:10C4B0002A003800FFF782FF061EE0D1216938000C
:10C4C000FFF7D4FEC7E7C0467FFBFFFFF0B59FB084
:10C4D000029005938B890F0016001B0611D50B697E
:10C4E000002B0ED14021FFF70BFF38603861002888
:10C4F00005D10C23029A013813601FB0F0BD402310
:10C500007B61002306AC6361203363761033A3762E
:10C5100035002B78002B01D0252B46D1AB1B049383
:10C520000CD0320039000298FFF76EFF431C00D197
:10C53000AEE06269049B9446634463612B78002BF0
:10C5400000D1A5E0012200235242626002A95432C8
:10C5500052186E1C2360E360A3601370A3653178EA
:10C5600005225448FFF776FE751C00281FD122686B
:10C57000D30604D5532302A95B1820211970130791
:10C5800004D5532302A95B182B21197033782A2B69
:10C5900016D0350000210A20E3682A786E1C303A54
:10C5A000092A4ED9002918D010E00135B1E7414BD6
:10C5B0002268C01A01238340134323602E00CEE774
:10C5C000059B191D1B680591002B01DB099304E0F5
:10C5D0005B42E3600223134323602B782E2B0AD1A6
:10C5E0006B782A2B35D1059B02351A1D1B680592E5
:10C5F000002B2BDB0793304E297803223000FFF706
:10C6000029FE002806D04023801B83402268013584
:10C61000134323602978062228486E1C2176FFF7F1
:10C6200019FE00283CD0264B002B25D10722059B64
:10C6300007339343083305936369039A9B18636137
:10C6400066E7434301219B183500A6E701235B42BF
:10C65000D0E700230A201A000135636029786E1C98
:10C660003039092903D9002BC5D00792C3E74243CB
:10C67000012352183500F1E705AB00933A00114B46
:10C680002100029800E000BF0390039B0133D3D147
:10C69000BB890B985B0600D42FE7012040422CE7B2
:10C6A00005AB00933A00074B21000298FFF736F8DC
:10C6B000EAE7C046F0E00000F6E00000FAE0000023
:10C6C0000000000009C40000002370B5064C0500FE
:10C6D0000800236000F060F9431C03D12368002B9D
:10C6E00000D02B6070BDC046B02F002070B5040094
:10C6F0000D001F2904D9162303600120404270BD9C
:10C70000436C002B04D08A009B181A68002A08D1B9
:10C71000200000F031F82A000100200000F01AF893
:10C72000EDE70020012AEAD0511C03D11623013085
:10C730002360E4E7002428001C6090472000DEE727
:10C7400010B5034B01001868FFF7D0FF10BDC046BD
:10C7500080000020002370B5064C05000800110081
:10C76000236000F001F9431C03D12368002B00D0A3
:10C770002B6070BDB02F002010B500F0E5F810BDA3
:10C7800070B50C000E25495F00F0BAF8002803DBF5
:10C79000636D1B18636570BDA389024A1340A381B2
:10C7A000F9E7C046FFEFFFFFF8B51F008B890500D2
:10C7B0000C001600DB0505D50E23C95E00220223FE
:10C7C00000F080F8A389054A28001340A3813200B5
:10C7D0000E23E15E3B0000F02BF8F8BDFFEFFFFFFA
:10C7E00070B50C000E25495F00F06CF8A389421C5F
:10C7F00003D1054A1340A38170BD80225201134327
:10C80000A3816065F8E7C046FFEFFFFF10B50E2378
:10C81000C95E00F021F810BD0B1E04D0FF2A04D918
:10C820008A2303608B3B180070470A700123FAE7E4
:10C8300070B50500080011000022064C22601A00A5
:10C8400000F0B8F8431C03D12368002B00D02B6004
:10C8500070BDC046B02F0020002370B5064C050007
:10C860000800236000F060F8431C03D12368002B0C
:10C8700000D02B6070BDC046B02F0020002370B5E3
:10C88000064C050008001100236000F055F8431C19
:10C8900003D12368002B00D02B6070BDB02F002087
:10C8A000002370B5064C05000800236000F054F822
:10C8B000431C03D12368002B00D02B6070BDC04601
:10C8C000B02F002070B50500080011000022064CB2
:10C8D00022601A0000F050F8431C03D12368002B9B
:10C8E00000D02B6070BDC046B02F0020704770474D
:10C8F0000B1F1B68181F002B01DA0B58C01870475C
:10C9000070B50500080011000022064C22601A00D4
:10C9100000F03AF8431C03D12368002B00D02B60B1
:10C9200070BDC046B02F002058220120014B40426C
:10C930001A607047B02F002058220120014B40425E
:10C940001A607047B02F002058220120014B40424E
:10C950001A607047B02F00205822024B00201A6046
:10C960007047C046B02F002058220120014B4042A2
:10C970001A607047B02F002058220120014B40421E
:10C980001A607047B02F002058220120014B40420E
:10C990001A607047B02F0020044A1368002B00D1A2
:10C9A000034B1818106018007047C046241C002064
:10C9B000B82F002058220120014B40421A607047D6
:10C9C000B02F0020FEE7C046F8B5C046F8BC08BC52
:10C9D0009E467047F8B5C046F8BC08BC9E467047F6
:10C9E000646174610000000064CA0000EF0100008F
:10C9F0006DCA0000E302000075CA000009090000CA
:10CA00007CCA0000190A000081CA0000310500003C
:10CA10008CCA00005303000091CA0000710C000092
:10CA20009DCA00001F020000A7CA000011080000F4
:10CA3000B5CA0000BD060000C2CA0000F104000033
:10CA400072616E646F6D00616C6C006C6173740078
:10CA500066616C7365007472756500252E313573DF
:10CA60002E2E2E006D616B654C69737400616464D9
:10CA70004C6173740064656C657465006A6F696EFF
:10CA800000636F707946726F6D546F0066696E64F3
:10CA9000006A6F696E537472696E677300756E69B0
:10CAA000636F6465417400756E69636F6465537488
:10CAB00072696E67006E6577427974654172726162
:10CAC0007900667265654D656D6F727900000000D2
:10CAD00035CB0000D91000003ACB0000E510000073
:10CAE00075CA0000E910000040CB0000ED10000006
:10CAF0004ACB0000F110000053CB0000F5100000FD
:10CB00005DCB0000F910000068CB0000FD100000B4
:10CB100074CB0000011100007DCB00000511000066
:10CB200087CB0000DD10000092CB0000E110000078
:10CB300066696C65006F70656E00636C6F7365008D
:10CB4000656E644F6646696C6500726561644C6928
:10CB50006E6500726561644279746573006170701E
:10CB6000656E644C696E6500617070656E644279D3
:10CB70007465730066696C6553697A6500737461E6
:10CB800072744C697374006E657874496E4C697385
:10CB9000740073797374656D496E666F00000000F0
:10CBA00030130000401300005A130000D813000097
:10CBB00010140000461400007E140000A4140000AD
:10CBC000E01400002215000078150000BC150000DC
:10CBD000281600007016000096160000CE16000001
:10CBE000141700003A17000068170000961700009D
:10CBF000CE170000521800001A190000901900000A
:10CC0000FE1900004A1A00006A1A00008C1A00007F
:10CC10003E1B0000841B0000FC1B000030130000C2
:10CC2000301300002A1C0000921C0000FA1C0000B7
:10CC3000581D0000A01D0000161E00008C1E0000E4
:10CC4000D41E00001A1F0000501F0000961F000095
:10CC5000DC1F00002420000078200000CC20000011
:10CC6000142100007E210000B4210000FC210000FE
:10CC7000442200008C220000C62200000E23000087
:10CC800056230000B82400003013000030130000C9
:10CC9000BE23000030130000F42300002024000015
:10CCA00056240000822400003013000030130000DE
:10CCB00030130000301300003A2500007C250000EE
:10CCC0003013000030130000C225000012260000BF
:10CCD000382600003013000030130000301300002D
:10CCE0006626000096260000C6260000FC260000EE
:10CCF000262700005C27000086270000AE270000E2
:10CD0000D627000006280000362800006028000012
:10CD10008A280000E82800001229000030130000D3
:10CD200030130000301300003013000030130000F7
:10CD3000422900006E2900009A290000C62900003F
:10CD4000F2290000282A00005E2A0000942A000030
:10CD5000CA2A0000F62A0000222B0000582B0000EF
:10CD600030130000301300003013000030130000B7
:10CD700030130000301300003013000030130000A7
:10CD80003013000030130000301300003013000097
:10CD90003013000030130000842B0000BA2B000079
:10CDA0005B2564206974656D206C6973745D00286F
:10CDB00025642062797465732900286F626A65634F
:10CDC0007420747970653A20256429005374616376
:10CDD0006B20756E646572666C6F7700626F6F6C46
:10CDE00065616E006E756D62657200737472696E56
:10CDF00067006C6973740062797465206172726196
:10CE00007900000007000000030000005ECE000073
:10CE1000DD2C000066CE00008D2D00006FCE0000DE
:10CE2000372E000078CE0000E12C000081CE0000FB
:10CE30003B2E000089CE0000252E000000000000DF
:10CE400001000000020000000300000004000000D8
:10CE50000A0000006D6963726F3A6269740068616C
:10CE600073546F6E6500706C6179546F6E65006805
:10CE70006173536572766F00736574536572766F74
:10CE800000646163496E6974006461635772697418
:10CE90006500474320746F6F6B20256420757365B0
:10CEA00063733B206672656520256420776F72642A
:10CEB00073003C496E74656765723E003C4C697353
:10CEC000743E003C4F626A6563743E003C42797474
:10CED0006541727261793E000D0A564D2050616EB7
:10CEE00069633A2025730D0A006D697363000000C1
:10CEF00025CF0000013B00002ECF0000913A00003A
:10CF000032CF0000E53900003ACF00008B39000035
:10CF100044CF00002139000050CF0000233800002A
:10CF20006E756C6C00686578546F496E7400736937
:10CF30006E006A736F6E476574006A736F6E436F3D
:10CF4000756E74006A736F6E56616C75654174001E
:10CF50006A736F6E4B65794174000000B8CF0000B2
:10CF60006D3B0000C0CF0000713B0000CACF000045
:10CF70008F3B0000D3CF0000993B0000DECF0000C4
:10CF8000A33B0000EACF0000AD3B0000FFCF000054
:10CF9000B73B000014D00000C13B000020D00000CF
:10CFA000CB3B000030D000007B3B00003CD00000B9
:10CFB000853B00006E6574006861735769466900BF
:10CFC0007374617274576946690073746F7057693E
:10CFD00046690077696669537461747573006D7989
:10CFE000495041646472657373006874747053656A
:10CFF00072766572476574526571756573740072F7
:10D000006573706F6E64546F487474705265717597
:10D010006573740068747470436F6E6E656374003A
:10D02000687474704973436F6E6E656374656400F1
:10D030006874747052657175657374006874747087
:10D04000526573706F6E7365001A1B1C030406072C
:10D05000090A171819000000000008080800080A4B
:10D060004A4000000A5FEA5FEA0ED92ED36E1932F9
:10D070004489330C924C924D080800000004880843
:10D0800008040804848488000A448A4000048EC48A
:10D0900080000000048800000EC0000000000800AE
:10D0A00001224488100C9252524C048C84848E1CB1
:10D0B000824C901E1EC244924C06CA525FE21FF080
:10D0C0001EC13E02448ED12E1FE24488100ED12E86
:10D0D000D12E0ED12EC48800080008000004800460
:10D0E000880244880482000EC00EC008048244886E
:10D0F0000ED126C0040ED135B36C0C925ED2521CF8
:10D10000925C925C0ED010100E1C9252525C1ED09B
:10D110001C901E1ED01C90100ED013712E12525E49
:10D12000D2521C8808081C1FE242524C1254981418
:10D1300092101010101E113B75B131113935B371B9
:10D140000C9252524C1C925C90100C92524C861CC9
:10D15000925C92510ED00C825C1FE4848484125243
:10D1600052524C1131312A44113135BB7112524C9B
:10D170009252112A4484841EC488101E0EC80808C6
:10D180000E10080482410EC242424E048A40000042
:10D19000000000001F0804800000000ED2524F1053
:10D1A000101C925C000ED0100E02424ED24E0C9219
:10D1B0005C900E06C81C88080ED24EC24C10101C83
:10D1C00092520800080808024002424C10149814B9
:10D1D000920808080806001B75B131001C925252D3
:10D1E000000C92524C001C925C90000ED24EC20079
:10D1F0000ED010100006C8049808080EC8070012C8
:10D2000052524F0011312A4400113135BB00124CEB
:10D210008C9200112A4498001EC4881E06C48C8477
:10D2200086080808080818080C881800000C836095
:10D2300000000000010000000200000003000000E8
:10D2400004000000050000000600000007000000C8
:10D2500008000000090000000A0000000B000000A8
:10D260000C0000000D0000000E0000000F00000088
:10D270001000000012000000140000001600000062
:10D28000180000001A0000001C0000001E00000032
:10D2900020000000230000002600000029000000FC
:10D2A0002C0000002F0000003200000036000000BB
:10D2B0003A0000003E00000042000000460000006E
:10D2C0004B00000050000000550000005A00000014
:10D2D00061000000680000006F00000076000000A0
:10D2E0007D000000840000008B0000009200000020
:10D2F00099000000A0000000A7000000AE000000A0
:10D30000B5000000BC000000C3000000CA0000001F
:10D31000D1000000D8000000DF000000E60000009F
:10D32000ED000000F4000000FB000000FF00000022
:10D3300080D30000ED3B00008BD300003D41000096
:10D3400095D30000A93D0000A2D30000AD3F00002E
:10D35000A9D30000FD3F0000B2D300004D40000003
:10D36000BED30000453F0000CFD30000193E0000AF
:10D37000DCD30000D53E0000646973706C617900F5
:10D380006C696768744C6576656C006D624469739E
:10D39000706C6179006D62446973706C61794F667D
:10D3A00066006D62506C6F74006D62556E706C6FCC
:10D3B00074006D62447261775368617065006D62DC
:10D3C0005368617065466F724C6574746572006E67
:10D3D000656F506978656C53656E64006E656F505B
:10D3E0006978656C53657450696E004E6F74206582
:10D3F0006E6F75676820726F6F6D206576656E2041
:10D40000616674657220636F6D70616374696F6EBD
:10D4100000436F6D70616374656420466C6173686E
:10D4200020636F64652073746F72650A25642062DF
:10D430007974657320757365642028256425252912
:10D44000206F6620256400426164207265636F72FC
:10D450006420666F756E6420647572696E672069FA
:10D460006E697469616C697A6174696F6E002564B4
:10D470002025642025642028256420776F7264733A
:10D4800029002564207265636F7264732C20256403
:10D4900020776F7264732C206D6178494420256475
:10D4A0002C20636F6D70616374696F6E20637963A4
:10D4B0006C657320256400526573746F7265642017
:10D4C000256420736372697074730053746172749D
:10D4D000656400726164696F000000006CD5000033
:10D4E000054B000079D50000A14D000089D5000052
:10D4F000214D000097D50000354F0000A2D5000057
:10D500002D4B0000B2D50000B54B0000C6D5000081
:10D510009D4B0000D5D5000017510000E1D500005B
:10D5200095500000EAD5000039500000F5D5000004
:10D53000814F000000D60000BD4F000009D600005A
:10D54000F14F000012D600003D4B000021D6000034
:10D550001D4B00002AD600004D4B00006E6F6E651B
:10D56000006F74686572007061697200646973614C
:10D57000626C65526164696F006D657373616765A4
:10D580005265636569766564007061636B657452AA
:10D59000656365697665007061636B657453656E7C
:10D5A00064007265636569766564496E7465676574
:10D5B000720072656365697665644D657373616752
:10D5C0006554797065007265636569766564537446
:10D5D00072696E670073656E64496E746567657223
:10D5E0000073656E64506169720073656E64537494
:10D5F00072696E67007365744368616E6E656C0076
:10D6000073657447726F757000736574506F7765DA
:10D6100072007369676E616C537472656E677468CB
:10D62000006465766963654944006C6173744D6597
:10D630007373616765494400556E6B6E6F776E203A
:10D640007072696D6974697665205B25733A25731C
:10D650005D00000000000000963007772C610EEEA0
:10D66000BA51099919C46D078FF46A7035A563E939
:10D67000A395649E3288DB0EA4B8DC791EE9D5E060
:10D6800088D9D2972B4CB609BD7CB17E072DB8E75F
:10D69000911DBF906410B71DF220B06A4871B9F3B4
:10D6A000DE41BE847DD4DA1AEBE4DD6D51B5D4F4ED
:10D6B000C785D38356986C13C0A86B647AF962FD52
:10D6C000ECC9658A4F5C0114D96C0663633D0FFA9F
:10D6D000F50D088DC8206E3B5E10694CE44160D5A5
:10D6E000727167A2D1E4033C47D4044BFD850DD28F
:10D6F0006BB50AA5FAA8B5356C98B242D6C9BBDBA2
:10D7000040F9BCACE36CD832755CDF45CF0DD6DC9C
:10D71000593DD1ABAC30D9263A00DE518051D7C843
:10D720001661D0BFB5F4B42123C4B3569995BACFCE
:10D730000FA5BDB89EB802280888055FB2D90CC6EF
:10D7400024E90BB1877C6F2F114C6858AB1D61C168
:10D750003D2D66B69041DC760671DB01BC20D29887
:10D760002A10D5EF8985B1711FB5B606A5E4BF9F14
:10D7700033D4B8E8A2C9077834F9000F8EA8099607
:10D7800018980EE1BB0D6A7F2D3D6D08976C649172
:10D79000015C63E6F4516B6B62616C1CD83065858B
:10D7A0004E0062F2ED95066C7BA5011BC1F4088268
:10D7B00057C40FF5C6D9B06550E9B712EAB8BE8BA9
:10D7C0007C88B9FCDF1DDD62492DDA15F37CD38C32
:10D7D000654CD4FB5861B24DCE51B53A7400BCA330
:10D7E000E230BBD441A5DF4AD795D83D6DC4D1A462
:10D7F000FBF4D6D36AE96943FCD96E34468867AD39
:10D80000D0B860DA732D0444E51D03335F4C0AAAD7
:10D81000C97C0DDD3C710550AA41022710100BBEDA
:10D8200086200CC925B56857B3856F2009D466B921
:10D830009FE461CE0EF9DE5E98C9D9292298D0B056
:10D84000B4A8D7C7173DB359810DB42E3B5CBDB703
:10D85000AD6CBAC02083B8EDB6B3BF9A0CE2B60384
:10D860009AD2B1743947D5EAAF77D29D1526DB0439
:10D870008316DC73120B63E3843B64943E6A6D0D84
:10D88000A85A6A7A0BCF0EE49DFF099327AE000ACF
:10D89000B19E077D44930FF0D2A3088768F2011E62
:10D8A000FEC206695D5762F7CB67658071366C19F9
:10D8B000E7066B6E761BD4FEE02BD3895A7ADA101A
:10D8C000CC4ADD676FDFB9F9F9EFBE8E43BEB717FB
:10D8D000D58EB060E8A3D6D67E93D1A1C4C2D83885
:10D8E00052F2DF4FF167BBD16757BCA6DD06B53FEB
:10D8F0004B36B248DA2B0DD84C1B0AAFF64A03362A
:10D90000607A0441C3EF60DF55DF67A8EF8E6E31A8
:10D9100079BE69468CB361CB1A8366BCA0D26F25F1
:10D9200036E2685295770CCC03470BBBB91602223E
:10D930002F260555BE3BBAC5280BBDB2925AB42B53
:10D94000046AB35CA7FFD7C231CFD0B58B9ED92C68
:10D950001DAEDE5BB0C2649B26F263EC9CA36A75CD
:10D960000A936D02A906099C3F360EEB8567077284
:10D9700013570005824ABF95147AB8E2AE2BB17BEB
:10D98000381BB60C9B8ED2920DBED5E5B7EFDC7C72
:10D9900021DFDB0BD4D2D38642E2D4F1F8B3DD68C9
:10D9A0006E83DA1FCD16BE815B26B9F6E177B06FC4
:10D9B0007747B718E65A0888706A0FFFCA3B0666B1
:10D9C0005C0B0111FF9E658F69AE62F8D3FF6B613E
:10D9D00045CF6C1678E20AA0EED20DD75483044EE0
:10D9E000C2B30339612667A7F71660D04D4769496E
:10D9F000DB776E3E4A6AD1AEDC5AD6D9660BDF4081
:10DA0000F03BD83753AEBCA9C59EBBDE7FCFB24733
:10DA1000E9FFB5301CF2BDBD8AC2BACA3093B35318
:10DA2000A6A3B4240536D0BA9306D7CD2957DE5421
:10DA3000BF67D9232E7A66B3B84A61C4021B685DFA
:10DA4000942B6F2A37BE0BB4A18E0CC31BDF055A73
:10DA50008DEF022D416C6C207461736B73207374B5
:10DA60006F70706564007630383200202573202591
:10DA700073004D656D6F727920636C6561726564CA
:10DA8000004E6F2066726565207461736B20656E51
:10DA90007472696573000000E0DA000051640000F0
:10DAA000EDDA0000DD600000F9DA000087640000B4
:10DAB000FFDA00009764000005DB0000A7640000A7
:10DAC0000BDB00001161000015DB0000B9640000F1
:10DAD0001DDB00005162000073656E736F7273008E
:10DAE000616363656C65726174696F6E0074656D06
:10DAF00070657261747572650074696C7458007435
:10DB0000696C74590074696C745A00746F75636839
:10DB10005265616400693263526561640069326311
:10DB200057726974650000009CDB000041650000CD
:10DB3000AADB000045650000B3DB00005165000072
:10DB4000BDDB000055650000C6DB00005965000024
:10DB5000CBDB00005D650000D0DB000061650000EC
:10DB6000DCDB000065650000E3DB000069650000A8
:10DB7000ECDB00006D650000F1DB0000716500006A
:10DB8000FCDB00007565000006DC00004965000054
:10DB900010DC00004D65000074667400656E616203
:10DBA0006C65446973706C6179006765745769646A
:10DBB00074680067657448656967687400736574A4
:10DBC000506978656C006C696E65007265637400FD
:10DBD000726F756E64656452656374006369726325
:10DBE0006C6500747269616E676C65007465787449
:10DBF00000746674546F7563686564007466745469
:10DC00006F7563685800746674546F756368590063
:10DC1000746674546F75636850726573737572655A
:10DC2000007661727300000048DC0000056A0000A5
:10DC300052DC0000E56900005BDC0000C169000007
:10DC400067DC00004D690000766172457869737485
:10DC500073007661724E616D656400736574566120
:10DC6000724E616D6564007661724E616D65466FDE
:10DC700072496E6465780057656C636F6D652074DA
:10DC80006F204D6963726F426C6F636B732100701C
:10DC90005F73706920213D204E554C4C002F686FFA
:10DCA0006D652F6769742F2E706C6174666F726D6D
:10DCB000696F2F7061636B616765732F6672616D49
:10DCC00065776F726B2D61726475696E6F6E6F72BE
:10DCD0006469636E7266352F6C6962726172696520
:10DCE000732F5350492F5350492E63707000535077
:10DCF00049436C6173733A3A535049436C6173738F
:10DD0000284E52465F5350495F547970652A2C2043
:10DD100075696E74385F742C2075696E74385F7421
:10DD20002C2075696E74385F7429000000000000B3
:10DD300000000000116C0000CD6B0000F36B0000D0
:10DD4000FD6B0000076C0000F16B00000300000099
:10DD500002000000010000000400000005000000B7
:10DD6000110000000C0000000B0000001200000079
:10DD70000A000000060000001A0000001400000065
:10DD80001700000016000000150000001000000041
:10DD9000FFFFFFFFFFFFFFFF000000001E0000006D
:10DDA0001900000018000000070000000800000033
:10DDB000090000000D0000000E0000000F00000030
:10DDC0001C0000001B0000001D00000013000000EC
:10DDD0000000000000000000C1700000F1770000AA
:10DDE00041710000557100004B710000BD700000D2
:10DDF000B170000061710000DD700000AD700000C6
:10DE0000000000000000304300000000000030C3AC
:10DE10007371727400000000FB21F93FFB2109407F
:10DE20007CD91240FB2119407A6A1F407CD92240DC
:10DE3000BBFD2540FB2129403A462C407A6A2F4001
:10DE40005C4731407CD932409C6B3440BBFD35404F
:10DE5000DB8F3740FB2139401BB43A403A463C4007
:10DE60005AD83D407A6A3F404C7E40405C47414032
:10DE70006C1042407CD942408CA243409C6B444091
:10DE8000AC344540BBFD4540CBC64640DB8F4740E8
:10DE9000EB584840FB21494083F9A200444E6E00F4
:10DEA000FC291500D1572700DD34F50062DBC000E6
:10DEB0003C999500419043006351FE00BBDEAB00EE
:10DEC000B761C5003A6E2400D24D42004906E00019
:10DED00009EA2E001C92D100EB1DFE0029B11C00A6
:10DEE000E83EA700F535820044BB2E009CE9840083
:10DEF000B4267000417E5F00D6913900538339000B
:10DF00009CF439008B5F840028F9BD00F81F3B00AA
:10DF1000DEFF97000F980500112FEF000A5A8B00C3
:10DF20006D1F6D00CF7E360009CB2700464FB7002E
:10DF30009E663F002DEA5F00BA277500E5EBC7003B
:10DF40003D7BF100F739070092528A00FB6BEA0033
:10DF50001FB15F00085D8D00300356007BFC46005A
:10DF6000F0AB6B0020BCCF0036F49A00E3A91D0093
:10DF70005E619100081BE60085996500A0145F00B2
:10DF80008D40680080D8FF0027734D0006063100E1
:10DF9000CA561500C9A873007BE260006B8CC000F4
:10DFA00000000040FB21F93F000000002D44743EBA
:10DFB000000000809846F83C0000006051CC783B9F
:10DFC00000000080831BF0390000004020257A38D3
:10DFD000000000802282E336000000001DF3693556
:10DFE0000200000003000000040000000600000022
:10DFF000E89400009294000092940000C095000004
:10E000008E9400008E940000B6950000C09500002C
:10E010008E940000B69500008E940000C09500001C
:10E02000C4950000C4950000C4950000CC95000084
:10E03000C49F0000369E00007A9E0000DE9D000016
:10E040007A9E00006A9F00007A9E0000DE9D00001C
:10E05000369E0000369E00006A9F0000DE9D000094
:10E06000D69D0000D69D0000D69D0000789F000040
:10E07000ECA60000EEA50000EEA500000CA9000033
:10E08000E8A50000E8A50000F4A800000CA9000025
:10E09000E8A50000F4A80000E8A500000CA9000015
:10E0A00002A9000002A9000002A9000010A90000B6
:10E0B0002C2066756E6374696F6E3A20006173730D
:10E0C000657274696F6E2022257322206661696C07
:10E0D00065643A2066696C6520222573222C206CC9
:10E0E000696E65202564257325730A00840000206D
:10E0F000232D302B2000686C4C0065666745464731
:10E1000000303132333435363738394142434445B3
:10E110004600303132333435363738396162636422
:10E120006566000000000000000000000000000024
:10E1300000000000000000000000000000000000DF
:10E1400000000000000000000000000000000000CF
:10E1500000000000000000000000000000000000BF
:10E1600000000000000000000000000000000000AF
:10E17000000000000000000000000000000000009F
:10E18000000000004300504F534958000020202059
:10E190002020202020202828282828202020202057
:10E1A0002020202020202020202020202088101027
:10E1B0001010101010101010101010101004040483
:10E1C0000404040404040410101010101010414141
:10E1D000414141410101010101010101010101012F
:10E1E0000101010101010101101010101010424243
:10E1F00042424242020202020202020202020202FF
:10E20000020202020202020210101010200000009E
:10E2100000000000000000000000000000000000FE
:10E2200000000000000000000000000000000000EE
:10E2300000000000000000000000000000000000DE
:10E2400000000000000000000000000000000000CE
:10E2500000000000000000000000000000000000BE
:10E2600000000000000000000000000000000000AE
:10E27000000000000000000000000000000000009E
:10E28000000000000000000000000000000000008E
:04E29000000000008A
:08E29400741EFF7F0100000071
:10E29C00FFFFFFFF4006000001000000E803DC0563
:10E2AC00DC05DC05DC050000FFFFFFFFFFFFFFFFC7
:10E2BC001800000019FCFFFFFFFFFFFFFF0000002C
:10E2CC000200000003000000FFFFFFFF0000000041
:10E2DC00010000000000020001000000FFFFFFFF32
:10E2EC00000000000200000000000400020000001A
:10E2FC00FFFFFFFF0000000003000000000008000B
:10E30C00030000000A0000000800000001000000EB
:10E31C00840000200000000044E1000064E10000E3
:10E32C0024E10000000000000000000000000000DC
:10E33C0000000000000000000000000000000000D1
:10E34C0000000000000000000000000000000000C1
:10E35C0000000000000000000000000000000000B1
:10E36C0000000000000000000000000000000000A1
:10E37C00000000004300000000000000000000004E
:10E38C000000000000000000000000000000000081
:10E39C00000000004300000000000000000000002E
:10E3AC000000000000000000000000000000000061
:10E3BC00000000004300000000000000000000000E
:10E3CC000000000000000000000000000000000041
:10E3DC0000000000430000000000000000000000EE
:10E3EC000000000000000000000000000000000021
:10E3FC0000000000430000000000000000000000CE
:10E40C000000000000000000000000000000000000
:10E41C0000000000430000000000000000000000AD
:10E42C0000000000000000000000000000000000E0
:10E43C00000000004300000000000000000000008D
:10E44C0000000000000000000000000000000000C0
:10E45C000000000019C8000031C2000000000000DC
:10E46C008CE1000062CA0000E8CE0000E8CE00009B
:10E47C00E8CE0000E8CE0000E8CE0000E8CE0000B8
:10E48C00E8CE0000E8CE0000E8CE0000FFFFFFFF62
:10E49C00FFFFFFFFFFFFFFFFFFFF000001004153E5
:10E4AC00434949000000000000000000000000008B
:10E4BC0000000000000000000000000000004153BC
:10E4CC00434949000000000000000000000000006B
:10E4DC000000000000000000000000000000000030
:10E4EC00E90000009D6B0000E56E00000D7400005B
:04E4FC00C10000005B
:0400000300006F8109
:00000001FF
